:20000000004B00204D3E0100FDC90110FDC90110FDC90110FDC90110FDC90110FDC90110DF
:1C002000FDC90110FDC90110FDC90110FDC90110FDC90110FDC901103BCA0110A4
:20003C00FFFFFFFFFFFFFFFF9A100000000000000000000000000000000000000000000002
:20005C000000000000000000000000000000FAFA1400000000000000000000010000010179
:20007C00000000000000000000000000000000000000000000000000000000000000000064
:20009C00000000000000000000000000000000000000000000000000000000000000000044
:2000BC000000007800080230000800000000000000000804FA000000FFFFFF000C1100004A
:2000DC000000000000001D1100000000000000002E010F000000FA0000002F010F0000005F
:2000FC00FA000000300100000000FF000000310100000000FF000000320100000000030053
:20011C0000003301000000000300000034010000000001000000350200000000FFFF000021
:20013C00370200000000FF000000390200000000FF0000003B0200000000FFFF00003D01B8
:20015C0000000000FF0000003E0100000000010000003F01000000000100000040010000C2
:20017C0000000700000041200000000000000000610200000000FFFF00006308000000002F
:20019C00000000006B080000000000000000730800000000000000007B08000000000000D2
:2001BC000000830205000000580200008501000000001000000086010000000032000000F0
:2001DC0087010000000032000000000038C40D00C8000000810000320F01000000C50D00E3
:2001FC00900100004000009605010000952B0D00C8000000220000320F0200003600010045
:20021C000600000000000000000F000000000000000000000000000000000300FFFF0000AC
:20023C000403FFFF0000FFFF0F00F4010005401F0320000100000000FF3F0F0008000E00B0
:20025C0000000000000000000300010F000009010000000000000000000000000000000065
:20027C0000000000000000000000000000000000000000000000000000000000AD000000B5
:20029C000001363601010001020100010301000104010606080400000C0100340D01000F4E
:2002BC0010040101140100FF1608000020020000220100FF23010001240100FE2501000820
:2002DC002602000028010001290100012A0200002C01000F2E020000300100013101000881
:2002FC00320200FF3401000735010240360100003701000138010001390100FF3A01000FCE
:20031C003C0200FF3E01010F3F0100014001041F41010001420100FF4301008044080000FB
:20033C004E0100084F01000F50010001510100FF5201090A53010185540100015804000056
:20035C005C0400006004000064040000680400006C04000070040000740400007804000011
:20037C007C040000800100FF81010001000120181A18182C34041E000C0E020B040B0A0792
:20039C000800110F00000500B900B300AD00B8001C00300038000800340102000304710404
:2003BC0002046004110470040204020401040204000410046104000414046304730472042A
:2003DC0062044304000413040604000400040404120400040004000400045104640000043C
:2003FC0000040004440400040004000400046504000435048104640005040004830400045A
:20041C00660400040004010171010101010111010101310101010101800100011001610197
:20043C003B001400630173017201620143010001130106013D0135000401120100010001B6
:20045C000001000104010401330133013C0144013201360000010001650100013500810101
:20047C00000105018201830100016601000100010302710230016002110270020102020251
:20049C00020280020002100261023A00410063027302720262024302000213023800000280
:2004BC00000204021202000200020002000204020402370037003C024402000239000002C1
:2004DC00000265020002350281020002050282028302000266020002000200000001000258
:2004FC000101000302010002000000000301000704010003050800000D0101FF0E08000092
:20051C0016080000200200000000000000FFFFFFFFFFFFFFFFFFFFFFFFFFFFFFFFFF000090
:20053C000000000000000300FFFF000000000000000000000000000000000000000000009E
:20055C0000000000000000000000000000000000000000000000000000000000000000007F
:20057C0000000000000000000000000000000000000000000000000000000000000000005F
:20059C0000000000000000000000000000000000000000000000000000000000000000003F
:2005BC0000000000000000000000010403040104030400000000FFFF000000000000000009
:2005DC000000000000000000000000000000FFFF0000000000000000000000000000000001
:2005FC00000000000000FFFF000000000000000000000000000000000000000001040501D6
:20061C0003040501009133010000A92E0100024B2D0000004F700100014B2D0000004F70A2
:20063C0001000355E10000004F70010004ED6F0100004F70010001E16F010001DB6F0100E5
:20065C00014F700100014F700100014F70010000A9440100014F700100014F700100014F7B
:20067C00700100014F70010002E16F010002DB6F0100024F70010000A9440100024F70011A
:20069C0000024F7001000241330100024F700100046B3C0000004F70010003E16F01000381
:2006BC00DB6F0100034B2D0000034B2D0000034F7001000355E10000034F70010000A94431
:2006DC000100034F700100034F70010004E16F010004DB6F0100044B2D0000044B2D0000DB
:2006FC00044B2D0000046B3C0000044F700100044F70010004E76F010000A94401000104E1
:20071C00E9FA01000300000000040000EDF701008BF90100DFF90100F9F301005DF4010050
:20073C00D5F8010061FA0100C7F90100B1FA0100F9F2010019F501006DF9010001F90100A9
:20075C006DF50100BDFA0100D5FA01009DFA010089FA010043FA010035FA0100D5F601003C
:20077C006FFA0100ADF9010015FA01009DF60100DFFA010011150100A151010001F00100C2
:20079C00C1F5010029F10100FDF9010021450100A966010091660100BDF40100B16D010034
:2007BC00A36D010059F601000000000000000000236F0100C56C010015F7010000000000EA
:2007DC000000000000000000000000000001040000333333333333333333333333333333FB
:2007FC003303010F00000000000000000000000000000000FFFFFFFFFFFFFFFFFFFFFFFFA3
:20081C00FFFFFFFFFF46485465737400000000000000000000000000000000000000000093
:20083C000000000000000000F507000001000000BC0B0000080000001A0700000112345612
:20085C00789ABCDEF000000000000000000000000000000002040201010101090200A2A681
:20087C00A8A0A5A59F95AD96B8B2A4313117191A21241B1D1F31313331313118191A223137
:20089C001C1E2031313431000000000002000000020000000A000000020000000200010008
:2008BC00000000000000000000000000000000000000000000000000000000000E0000000E
:2008DC0003007100300160001100700031022003500480000700100061000000140063005D
:2008FC0073007200620043000000130006000000000004001200000000000000000004001F
:20091C000400370037003C02440000000000000000006500000035008100000005000000A7
:20093C008300000066000000000001037103010301030103010301032203020301030003F5
:20095C001003000300030003000300030003000342030003240306030003000304031203B9
:20097C002503230325032303040304030003000300034403000300032303000365032100A9
:20099C0035038103000305030003000300030003250323038F0000008F0001008F0002006A
:2009BC008F000300900000018F00010190000002900000038F0001048F0000058F0008047F
:2009DC008F0000048F000006510000007F0001003F0004003F0002003F0001007F000200BD
:2009FC007B756E6B6E6F776E2D696E7374616E63652D6E616D657D007B656D7074792D6943
:200A1C006E7374616E63652D6E616D657D00C0467B7374617469632D696E7374616E6365F8
:200A3C002D6E616D657D00C0000000000800000000000000200000004000000060000000C7
:200A5C00000000000600000002000000860000008200000000000000080000001000000052
:200A7C001800000020000000C003000080070000000F0000001E0000003C000000780000F7
:200A9C0000F0000000E0010000C003000080070000000F0000001E0000003C00000078003E
:200ABC000000F0000000F00006088080070880800D2007C00E2007C01400C080024000801E
:200ADC000300C0800108C0801E08C08009400080084000800A400080FE00000009050100A0
:200AFC006D260100396701007D93000059BB000005700100B51D0100D5C400000B70010023
:200B1C009505010000000000FFFFFFFFFFFFFFFF00000000000000000101010100C201005F
:200B3C0003000000000000007BC80110C5BC0110D9B2011033C20110BDAD0110C1B1011010
:200B5C006DBA011065BB01101DC00110001000400600000015000000FF00000000000000B8
:200B7C000302FFFF082D002020000000FFFFFFFFC409000000000000C782000001003A0193
:200B9C000000000000000000F80A000008250020680B000000000000000000000000000077
:200BBC00000000000000000000000000000000000000000000000000C33B3D3A5D3A713A62
:200BDC00A10A8F3A0F3BB309495E850A2F3B853B001610160E18151C0212032418580302DC
:200BFC0010025800010000000000000000000000000001000000FF7F142B0020340C000050
:200C1C0000000000000000000000000055D90000691A010001010100004002400B00000076
:200C3C0027000000FF00000000010509000408100004081041B5011095A6011015B80110FA
:200C5C0000BE040A00BE0208FFFFFFFFFFFFFFFFFFFFFFFFFFFFFFFFFFFFFFFFFFFFFFFFFC
:200C7C00FFFFFFFFFFFFFFFF3545251502030504FF0000000000000021670100FD2F0100E9
:200C9C00060005000000FFFF000000400F000000AD9600000A000000041B00209556010068
:0F0CBC0097700100C1C70000BB6F01000102016A
:201000003C000000000000000000000034100000000000000000000001000000000000004F
:1C10200000000000000000000000000001000000000000000800000000000000AB
:20103C003400000000000000000000006810000000000000000000000100000000000000E7
:14105C00010000000000000000000000080000000000000077
:2010700030000000000000000000000098100000040000000000000001000000FFFFFFFF87
:10109000FF00000001000000080000000000000048
:2010A0002C0000000000000000000000C4100000040000000000000001000000FFFFFFFF2F
:0C10C000FFFFFFFF080000000000000020
:2010CC0038140000E410000095A1011091A70110A1C2011009B2011041B8011000000000EA
:0810EC00000000002D000000CF
:2010F400280000000000000000000000141100000000000000000000FFFFFFFF0000000093
:081114000800000000000000CB
:20111C00341400003011000065C2011069C101101BC2011091BA011000000000000000006D
:04113C002F00000080
:20114000341400005411000071C20110A5B6011099BF011045B601100000000000000000BD
:04116000300000005B
:201164002400000000000000000000008011000000000000000000000000000008000000AE
:041184000000000067
:20118800240000000000000000000000A41100000000000000000000000000000800000066
:0411A8000000000043
:2011AC00240000000000000000000000C8110000000000000100000000000000080000001D
:0411CC00000000001F
:2011D00000000000C81B002004000000000000000000000020000000701000003000000028
:2011F0001C110000D01B00200400000000000000000000000C00000030130000180000003C
:2012100040110000D81B0020040000000000000000000000240000004813000018000000BF
:2012300000000000E01B002004000000000000000000000010000000A01000002C00000093
:20125000CC100000E81B0020040000000000000000000000200000006411000024000000C2
:20127000FFFFFFFFF01B00200400000000000000000000002800000088110000240000004E
:20129000FFFFFFFFF81B0020040000000000000000000000580000003C1000003400000033
:2012B000FFFFFFFF001C002004000000000000000000000010000000601300001800000047
:2012D000FFFFFFFF081C00200400000000000000000000001C000000AC11000024000000BD
:2012F000FFFFFFFF101C002004000000000000000000000038000000F4100000280000002E
:20131000FFFFFFFF181C002004000000000000000000000054000000001000003C000000C9
:1813300018000000000000000000000040130000080000000000000032
:1813480018000000000000000000000058130000080000000000000002
:18136000180000000000000000000000701300000800000000000000D2
:0813780002000000940C0000CB
:041384000100000064
:0413880000000E0053
:04138C0000000F004E
:041390003200000027
:041394000100000054
:041398003C1B0020DA
:04139C00000200004B
:0413A000F36F0100E6
:0413A400FDC901106E
:0413A8000000000041
:0413AC00000000003D
:0413B0000800000031
:0413B4000000220013
:0413B8005C1900209C
:0413BC00010000002C
:0413C000541B00209A
:0413C400080000001D
:0413C8000000000021
:0413CC00000000001D
:0413D0000000000019
:0413D400080000000D
:0413D8000000000011
:0413DC00000000000D
:0413E0000100000008
:0413E400841A002047
:0413E80006000000FB
:0413EC0001000000FC
:0413F000FC170020C6
:0413F40000000000F5
:0413F80000000000F1
:0413FC0000020000EB
:0414000000000000E8
:021406002900BB
:021408000100E1
:02140A002500BB
:02140C002F00AF
:02140E003000AC
:021410002D00AD
:021412000100D7
:0114140001D6
:0814180003000000500C00006D
:081420000000000000000000C4
:0414280000000100BF
:04142C0000000300B9
:0414300083C4011060
:041434003C14000064
:041438003C14000060
:04143C0000000000AC
:041440008000000028
:041444008000000024
:0414480000000000A0
:04144C00541B00200D
:04145000516C0100DA
:041454002000000074
:04145800000C000084
:04145C00440B00003D
:0414600009C30110AB
:041464006B400100D8
:041468006B440100D0
:04146C0095C801100E
:0414700097C8011008
:041474000000000074
:04147800FF0B000066
:04147C00140A00004E
:041480002C0A000032
:04148400FC0900005F
:0214880008005A
:02148A00090057
:02148C0001005D
:02148E0000005C
:01149000015A
:041494000000000054
:041498000000000050
:04149C00000000004C
:0414A0000000000048
:0414A4008B70010048
:0414A8002D4C0100C6
:0414AC001D5E0100C0
:0414B000E14F010007
:0414B400DF50010004
:0414B800A15401003A
:0414BC0055170100BF
:0414C000F76D0100C3
:0414C400D92A010020
:0414C8000DC801103A
:0414CC001DC8011026
:0414D0000800000010
:0414D40024000000F0
:0414D80018000000F8
:0414DC0028000000E4
:0414E00020000000E8
:0414E4003C000000C8
:0414E8000C000000F4
:0414EC0034000000C8
:2014F000CA482DE9F04F0C4601210170DFF82493DFF82483DFF824A3DFF824B3C4494FF0EC
:20151000000C2027ADF14C0D65461F4081F800C0C7490E9391F838600D9205EA020008BF05
:2015300000287AD10D984FF0E047194662460F4002EA000008BF002843D10E9E0D9B4FF441
:201550008601B9F8B200DFF80CC3CDF8289012EA060701EA030108BF002919D1BC4912EA9B
:20157000060701EA030108BF00296FD0374643460D9E1C8103F130015881002F81E8C0008C
:2015900004BF311CB1F1806F60D102285ED111E0374643460D9E1C8103F130015881002FA4
:2015B00081E8C00004BF311CB1F5803F4ED1B0F5505F4BD1186A674643693868214698472D
:2015D00042E04646C449B6F9087091F90000BC42A0F10100087017D1728906F1300003C8B2
:2015F000002904BFB0F5803FB2F5505F08D0002904BFB0F1806F022A02D010F037FF03E0CA
:2016100012F0BCF815F02CF9524692F90000401E10706FF00101318114E043466FF00100E9
:2016300003F1080108806EB1B4480078832802D08120594608704646316919B160468847E8
:201650002146E8E7CDF82890B9F8B2000D9A0E9E02212F461140374008BF002900F07C83D2
:20167000A84A43F201418142119200F04F83C91C814200F04B8398490A4691F9001047460B
:20169000491E1170B7F908108C4205D043F60401814240F04A8346E3654890F838C007F19B
:2016B000300090E800034FF482062F4617EA090706EA080008BF002810D15748303003C88C
:2016D0004FF400322F4602400F4008BF002A02D110F0CCFE29E312F051F826E30020BCF1C4
:2016F000010F4FF081045D460F9003D0287808B115F0D8FA2C70824C002067786081119EC8
:20171000E770054635702069DFF8FC91017A457A05F0070201EB022135F07F05A1F10401FE
:201730001FFA81F840F0D982B8F5006F80F2D5820A3041460FF08EF9E16904F114000522D6
:20175000083115F0C9F8A8F1030305201FFA83F8E27DA57D6081217E354B0C96C2F3011039
:20177000109093F83800617105EB022518B91099022900F0B2821099022900F3AE8260B13C
:2017900015F0070F00F0A9825C480078862804D105F00700022840F0A082281300F0020AB5
:2017B000BAF1020F58DAA37805F00700022841D14E46D6F804B0002B3CD1E16909A801226C
:2017D0000D3115F089F806206081D84780460B96C24F4A48B6683A680078862822D122B951
:2017F00015F060FA48463A6886689DF9240015F03CFC9DF924705077002090774046D77779
:20181000B04705F0100010F07FF80DE0A21B0020981B0020D8120020001700209E1B00208E
:20183000902D00204046B04714F0B6FE59E2C04614150020314800780026862808BF012649
:20185000CDF82C905EB1002012F00AF8E77805E000000C8CD0190020CDF82C90A37887B10B
:201870007BB9012F00F03682022F03D115F0070F40F03082032F04D105F00700032840F0EC
:201890002982280908D315F4405F00F02382C2480778002F00F01E82BAF1020F02DAA80AB2
:2018B00080F01882BE480078C0F3810B8611BBF1010F00F00F82012E00F00C821099B74828
:2018D00002290BD010F80B10805D4018C7B20EB3E8091FD3BF1E0EE09F1B002000EB0B01E1
:2018F0008019097900794018C7B2E8090ED25BEA06030FD0BF1CFFB20CE0C046942D002016
:20191000E42C0020922D0020B41500205BEA060308BF0227C5F30029A7EB09008045C0F28E
:20193000D981A8EB07002909484480B2208124BF25210F910F994018743080B215F0AAF8CC
:2019500094F80280E060002800F0C481002174220FF0C1FB0020B8F1000F207103D10C9978
:2019700005F0200008700C9803784FF00008002B53D0B9F1000F50D1D548008805F007019A
:2019900003291ED18108424609D3544991F82E30A3B90B681BB15B7E33F07F030ED16AB990
:2019B0008008C24607D3D6498B68887813B1984794F8048010B9BAF1000F02D004202071DE
:2019D0008046D14890F8383013B11098022824DACC490220002301F10A0AB8F1000F8AF8FA
:2019F00000006279CB72AAF1020007D000F1020A9AF8001041F010018AF8001002710A9AC1
:201A10000521A2F87810C2F8840014F081F9504603210FF01FF894F80480E16801F1740023
:201A30004860886523890B812089A1F85C0028090ED3C9F1030082B2A1F85C20886DD54900
:201A500014F04AFFE1688A6DB1F85C00801888655348D04B0078C0F3011218788D81B9F123
:201A7000000F00F0780040EA020048EA00050D744FF0FF038B730CBF6079002081F83060EF
:201A900081F83AB081F849006089002FA0EB090085B2658100F01381E0693A46E780291853
:201AB0000831684614F018FF3D48EE19B5B26581E16800780A7C6E46C0F38103C0F3011A3B
:201AD000C0F38108002B02F0400949D0C0F301100023022804D1D0090ED201E0700D00201E
:201AF0009DF801209DF8000000EB0220A1F844000DF10206A1F84200AE4AB1F84400B2F831
:201B10005220824203D04FF6FF72824222D1B8F1030F12D072783078A64B00EB022082B2DE
:201B30004A86B3F85010B61C0120914211D04FF6FF71914218BF00200BE0E0683146323088
:201B500015F073FAE0689B493230473114F032FD08360346002B00F0B5802046E168C07D07
:201B7000831125D0BAF1020F03D0087CC00903D309E059EA080206D172783078B61C00EBBE
:201B90000220A1F84200032B0CD07078327802EB00220A850CE0C0466C0F00205C0C000009
:201BB000FB2C0020E0683146283015F03EFAE16888890009C0F08380886D3A46694614F03C
:201BD0008BFEE068816D79188165E669B0F85C1001227F18A919A0F85C7008310DF1250020
:201BF00014F07AFE6F1CBDB26581E1689DF82500896D0870E2689DF825609DF82530906DBD
:201C1000401C9065B2F85C00401CA2F85C0006F0070082F82400C3F3C10182F825102089A0
:201C300092F824708046002F4CD0604F7F183E78361D8642E68045DCE0692918324608318C
:201C500005A814F049FE3A789DF817C0111D481980B29DF81450608105EB0C60E3689DF887
:201C7000165000EB05409DF81550042900EB052098610BDDE06806A9521E1C3014F02CFEC5
:201C90003878E3686844C07D83F82600986D05A9324614F021FEE068816D71188165B0F814
:201CB0005C10A8EB06077118A0F85C10791E89B22181B0F85C2001818918A0F85C1000F0CC
:201CD00083F80EE015F0F6F810F0D0FB09E0C0464816002014F042FF03E014F03FFFCDF831
:201CF0002C90DDF82C80D8F804008047E1690A68002313710968E161D8F80810884714E03B
:201D1000A41B0020F41900201415002040462A4F80784146401C887097F900003946401E1F
:201D3000087010F0A3FB14F0B7F926480A99214F00226FF0010690F83800A1F8B2203E81D6
:201D500010B11198007808B914F08AFD1B481B4990F90000401E0870174890F9000010B96E
:201D7000134800210170154890F90000A0B10D9A0E9F02214FF0E0401140384008BF0029A0
:201D90000ED00E4890F90000002809DC14F08AFF06E0C046FA2C00200020014604F008FF48
:201DB0000749002013B00870BDE8F08F440C0000961B0020001700209F1B00209E1B002039
:201DD000A21B0020141500202DE9F04FB94C0C3CE0686189E2692589806DADF13C0D0E46D8
:201DF000891808312A4614F077FDA81986B2E068816D6D188565E0690122311808310EA8CF
:201E100014F06AFDE069761CB5B2042265812918083104A814F060FD9DF813109DF8100015
:201E300000EB0160E3689DF812102D1D00EB01409DF81110658100EB0120049014F048FE48
:201E5000D863049814F02AFBA3F84000EA2014F0CCFB0221B648E2680170117C2079084375
:201E700010749DF9380015F000F982F846009DF93800118982F84800002082F8470002F144
:201E900074009065B2F85C00401A5168091851609089830A18D2030957D310F0070F07D02B
:201EB00000F00700032812BF081C5068401C48E05068C17801F00703491001F0380101EB64
:201ED00043014018001D3CE0171C02D114F0EAFEE268B889800A2ED379684878C6112AD1A2
:201EF0003E89796600204D780B7805F07F056D0005EBE3157E2D0DD07F2D09D003F07F0374
:201F10001818801C5B1880B2991C8642EBDC08E0002100E00121801C87F8601080B286426C
:201F300001DA002005E07968411879603989091A3981A7F86800506E10B1B2F86800B0B106
:201F5000506850619089000916D292F86000002800F0FC80104611F045F9E268D06C00283D
:201F700000F0F480B2F85000002840F0EF8014F08FFF0020E06024E24FF0000B1546104639
:201F900005A9CDF814B007ABCDF818B095F82470CDF81CB006AA04F004FD002840F0CB80C1
:201FB000059A6E6968682B89311A581A1FFA80F80AB914F077FEB5F85C0000900196CDF898
:201FD00008800698001D03900598A969AB6D3A4615300AF0E1FC002840F0AD80AD4895F8B1
:201FF00060302E89C15D701A288113B1284611F0F9F8AE8906F00706032E02D1686800788F
:20201000E87395F80F90732009A913F08FFC83200DF13A0108F08CFADFF8D082DA4651461C
:202030000AE0C278012A03D1002F08BFDC2027D0001D491C0990C9B29DF83A00884279DDFF
:2020500009988278032E07D00378B3420DD098F800300BB1022E08D0032EE9D10378032B68
:20207000E6D103465B784B45E2D1BB10B3EBA20F05DA02F0030207F003039A42D1DD50462D
:202090008146059895F80FC090F814E0514601E0491CC9B28E4549DD07694B00032E03EBC9
:2020B000070209D1FB5C032BF2D152786245EFD10BE0C046F02C00201278B24205D098F8A4
:2020D0000020002AE4D0022EE2D10698077D002F08BFB9F1DC0F2DD0A869B0F1FF3F23D082
:2020F000712008A913F022FC5346089AA9690598824206D106989A4600EB8A00C068884203
:2021100010D85B1C2C32022BF1DB0698491CB1F1FF3F00EB8A00C16002D1079801218170FB
:20213000584608E0DB2007E0DB2004E0DC2002E0902D0020DD206870E268507090695778E6
:2021500050651FB1F22014F050FAE2689F4DDFF8849295F83810002900F0AD8090899C4E49
:20217000DFF874B200F00700022858D1A078002855D15078002852D1E1684FF000080CA84B
:202190008DF83980283114F050FF06F11C01E7680888EB6D401C0880786E0DF139020421D2
:2021B000984704F10C0A30B94846006818B19DF8391080F8681014F0FFFA90B1E76897F893
:2021D000300002280ED1DAF80000594602222031283013F0E5FD28B90BF116010CA814F0E7
:2021F00024FFE7680DF12E0000906D6E786E0CA942460BABA84779480078862808D1F08BC3
:20221000E768401CF083B88900F010000FF07CFB14F03EFE4046E06014F0BEF9D3E0704BAA
:202230001A78002702B101277248026827B16F7817B114F0C1FA28B91878002831D014F0F2
:20225000BBFA70BB53782779002B40F0BA809DF83800318C02F12803002F207002F11C0216
:2022700001F10100308414BF082600265D490020086014F0ADFA0146009658460192263043
:2022900006881A460D20334605F094F920B913F03FFD03E0480C000014F01CF91348E2680B
:2022B000017841B1D5F880702FB13946104688470E48E26801780A9251B1907BFF287AD02F
:2022D0001046C17B042976DC40680078072872D0938913F0070040D0401E56D0801E6AD1B9
:2022F000C3F30130022808D102E0C0464C1500205068007807282ED0FFE7108900285AD04D
:20231000104641684A1C42600F788446C7739CF824607EB9002F4ED00A2F4CDA0189324E16
:20233000F01910F8010C884209D0082F43D1082905D040E0C07B00283DD00A283BDA6046FE
:202350000189491E0181C17B0B3101700A99C87B401CC8731BE0322018E0244E96F8A100AE
:202370000F280CD014F0D2FB48B9181300F00200022804DA0A984D462D1D2968884796F8D6
:20239000D7000A9A1074152000E0162010700A994D4605F1280012F001FE154E706880470C
:2023B00095F83010491C85F83010B1688847202014F0B0FC02E00AA811F0D0FF4FF000089B
:2023D00028E710F053F80FB0BDE8F08F14150020241A0020700D0020340F0020942D002028
:2023F000922D0020F819002070080000A00E0020B4150020F02C00202DE9FE4FE5498046FB
:202410000122A1F130000260DF480768002FFCD0DE4ADF4EC027E048E04B1760326892089A
:2024300008D2324652F8042C03F14104120C42F0F00222704FF0000A8346C1F800A0DFF871
:2024500064C3DBF80810D64D0191880E43D2480E41D3802018744FF6D802A3F851201870B1
:202470002868C0F30464162CA8BF203C1F460F3F387800F01F001628A8BF2038844223D074
:20249000624602F1980EDA4ACEF800A0261A022E05DC16F1020FB8BF6FF0010600E0022613
:2024B0003018166800F01F06844246F4F856A7F866604FF001061660E8D11068374617609D
:2024D0001068CEF80060106828460068C0F30420162808DB06E0A5F1D0000068C0F304603D
:2024F000162800DB203800EB2170401C162805DA10F10A0FB8BF6FF0090000E01520DE4F2B
:2025100000F01F0040F4F850A3F85900386880083ABFEA48C0F800A041F04061019E624668
:20253000A5F13804C80E8F0E80F0010000F00100106087F0010000F0010090602068C0F3E0
:202550008367C0F38F21B00C23D2304640F3072000280BD542425046490805D17F0806BF08
:202570000127391C4FF6FF71521EF5D1002810DD4FF6FF72490041F001018A4207D27F0078
:2025900047F001070F2F92BF01210F27111C401EF0D141EA0741182012F0E2FB2068D24E87
:2025B0002768C94CA6F10409C0F3870107F0030041EA0021D9F8040040F2FF3253468FB230
:2025D0002C21466800972746A7F14000B0470C3D2868C0F30D011C2012F0C2FBB84955F83A
:2025F000080C014000F07C400143142012F0B8FB55F80C1C01F47C000904090C0143102021
:2026100012F0AEFB624955F8042C0968C2F30350C2F30345490813D2DBF800100B0510EB3D
:20263000237003D41028A8BF0F2000E05046090415EB217503D4102DA8BF0F2500E055460F
:2026500045EA001502F47F4002F0FF01B8F1220F40EA054041EA000124BF02F0804211431F
:202670000C2012F07DFB974DB8F1220F32BF01202868C0F30070B8F1220F4FEA400040F09E
:20269000200084F8090126BF2868C0F3407001208E4EB8F1200F40F0100084F8090138BF1A
:2026B000514606D33168C80C00F44070C1F384510143282012F054FBB8F1200F26BF3068CE
:2026D000C0F301505046B8F1220F4FEA400040F0600084F80C0126BF2868C0F3C060504606
:2026F000B8F1220F4FEAC00040F0800084F8010126BF2868C0F345505046B8F1200F4FEA65
:20271000800040F47C40A4F89C0138BF70490AD3306801038A15920501F47C1100F00F0020
:20273000114341EA0031082012F01AFB4FF48000A5F1D0012060674A886D40F21E236FF375
:202750001F40834216D90868030E13F00F0F03F00F01C0F3034018BF491E072805D006284B
:202770000EBF0720801C00F00F0041EA0011A2F108000170DDF804C0CCF381477F1E13D0D2
:202790007F1E3BD036E0C0469402224300600C40B03F005040100940AC3F005015620840EC
:2027B000881300500000204328460068810C21D24FF480412160D2F80210430AC0F30337CA
:2027D00003F0800321F08F010B4347EA0301C2F80210D2F80130060A66F30303C2F801302E
:2027F000116800F0E70721F0E70147EA010004E02C2009404FF00040224610603B4800688C
:20281000C0F3C0070FB94020A0624FF40070206428684027C0F3C14040F0300084F8C8007E
:20283000CCF3815050B3401E03D0401E1FD002211EE0012012F0CEFE0646042031460FF081
:20285000DDFE042012F0C6FE8642FAD12248066826F07F4012F0FCFCD9F8140003680721F1
:202870004FF06022300E98474FF480602060032104200FF0C3FE08E0000009400420012148
:202890000FF0BCFE154812F0E3FC203D2868144947F6180600F03F0084F8CB0F144B0E801A
:2028B000D9F800201868D1680220884711480D4D076001212960BDE8FE8FC04694042A436B
:2028D000FCFCFC008C13005040A00C409813005000803F400A600840A83F0050BD3786007C
:2028F00070B00C4094046042A4010010B03F00502C20094000600C402DE9F04FADF18C0D61
:202910001C911E93CC491D920A6806460DF156000260496841603046694612F0B7F90028C0
:202930001F9004BF0020229000F0F78102200027B61CDFF84CB32090D34D2297304602A940
:2029500010F0CDFC5FEA000900F0E48122990EA816220EF0C0FB9DF809707F1E00F08280F8
:202970007F1E40F0CF81B9F10A0F40F3D681B61C316804A80160361D318805AF42F20B0066
:2029900039800DF1160110F087FEBDF81600BDF81410884200F3C181B61C16F8010B16F837
:2029B000017B16F8014B8DF8380016F8011B8DF839700EAA8DF83A40304605F03BFEBF49B9
:2029D00009780028064400F0A8811F9C012904F1020400F091814FF400500DF14E0110F019
:2029F0005BFE0DF14E000DF15601082213F0D8F940B11C990DF14E00082213F0D1F90028BE
:202A100040F07A8142F2010004A906F015FB42F20B0005A906F010FB42F205000EA906F0BF
:202A30000BFB0DF1390142F2060006F005FB0DF13A0142F2070006F0FFFA0DF13B0142F247
:202A5000090006F0F9FA9DF83B0028B1022840F0538142F2030001E042F20D000FA906F096
:202A7000EBFA49E1B9F1040F40F35781B61C16F8010B16F8017B16F8014B8DF8380016F8D4
:202A9000011B8DF839700EAA8DF83A40304605F0D1FD0028064400F040811C9806A906F070
:202AB00055F89DF83600002840F00A819DF83B0000287AD195F83170002F00F0FD8095F871
:202AD0003300874207D095F88C000A2801D10AF0B9FCA86B1EE0AF6B4FF400500DF15E012C
:202AF00010F0DAFD13F048FA4FF0FF08229C2190A24695F83100A04240DCA86BB8F1FF0F87
:202B100008D008EB88040019007912F011FBA86B071923D195F831300746002B08BF229C9C
:202B300019D05846229C40681946D8467F1F7F1DFA782AB1491E04F10104F8D17F1D0AE0E4
:202B5000804795F83310491C85F83310D8F80810884795F83130A34200F094801C980CF06B
:202B700077FA38710120F870FC788DF8364038798DF83700229B8DF82330A1E0387911F0FE
:202B9000D5F8014608220DF15E0013F009F940B138880104219814F054FA82453CBF82463B
:202BB000A046641C7F1DA4B2A3E795F83070002F00F0828095F83200874207D095F88C005D
:202BD0000A2801D10AF03EFC686B1EE06F6B4FF400500DF1660110F05FFD13F0CDF94FF0A6
:202BF000FF08229C2190A24695F83000A0424DDC686BB8F1FF0F08D04FEA48140019C07F50
:202C100012F096FA686B071925D195F830300746002B08BF229C1CD0DBF80400229C19465F
:202C3000D846203F2037BA7F42B1491E04F10104F8D120370DE0C0466C0C0000804795F844
:202C50003210491C85F83210D8F80810884795F83030A34216D02299384620220EF03BFAE1
:202C70001C980CF0F5F9F8770123FF2039462022BB770446787206A8FC720CF0FBFE1FE0BD
:202C9000B4150020612055E0CC100020F87F11F04DF8014608220DF1660013F081F838B192
:202CB0007968219814F0CDF982453CBF8246A046641C2037A4B297E764203BE0151500209C
:202CD0009DF836000EA9162240F004008DF8360008A80CF0CFFE1F9C9DF83B00A41C40B186
:202CF0009DF84D700FA839460FF04AFF3F1A8DF8357006A80FF02AFA20984844801C80B28E
:202D1000209003E01F9C4E44B61CA41C209884423FF714AE2098022803DC229A6720114660
:202D300004E01F9A911C121A2298921C1D9B19801E990A8023B0BDE8F08F70472DE9F84314
:202D5000C74C0F460646F80B80F0DD81E07AB90F80F06B81B80880F05881F80A80F0318133
:202D7000207A10B1380980F02981206C002840F093803809C0F09380002501262570B948B0
:202D9000A67114F03DF8284613F036F9B64904F170002A4614F04CF904F1580090E800034E
:202DB00013F050FE2379B0EB08004FEA103071EB09010905012B40EA0100606606D194F806
:202DD0006810B0EBC12F01D8E07860B340F60900A08294F82100267100F0F00040F00100E6
:202DF00084F8210094F82000E57000F0F00084F82000A56114F0FCF9D14A131D196821F0CD
:202E1000020119606FF00203136004F1140642F8106C11688908FCD31360516841F0020151
:202E3000516014F0E1F92E4604F1580080E86000666611F003FC6078012803D0E068403012
:202E500014F0CEF9C6480660022011F0D7FF11200BF05AFBE068007C10B90E200BF054FBA4
:202E7000A07A18B1A572052011F0C8FFBD49A5710878E57128B10D7004F1EC00042113F00A
:202E90007FFDB4F95000B4F95210884214BF022007200CF031F98EE0380980F08C80B80BA0
:202EB00077D2780B29D2380CC0F0518104F13C0014F0D1F8F0B1C16849680978022919D166
:202ED00090F82700400915D2206C90F82700400910D3206C806840880028FAD0206C8068FA
:202EF00040880128F5D0206C0026A0641920266413F020FF27F4004729E110F0D7FD38B148
:202F1000B56930466FF4807100224FF00073A847954904F17000002214F08AF8B1680025CD
:202F30004FF0010840F602026572088884F8008082420AD0B0F5C15F07D00A8B4FF61F6009
:202F5000104040F43470088306E00A8A4FF61F60104040F434700882757413F073FDD4F896
:202F70005421E36804F5AA719A4208BFA846266E46B1864226BF301A401E801B01EB8801EC
:202F9000000B88602566192013F0D4FE27F48057DDE004F1400014F05EF8061C08D0706885
:202FB00030B17568F068B6F9241000222023A84727F40057CBE027F00807C8E00020207217
:202FD000F9E714F015F9054604F13C0014F043F8061C15D0E06810B1783013F0BDF8F0686C
:202FF000E060284614F000F913F02CFD20665F4813F006FF4FF4006104F1EC0013F0C0FC71
:20301000002027F480672072A1E004F14C05284614F021F807F0E0FB284614F01CF827F02B
:20303000020708B147F0020791E020B1042011F0E5FE0020E07214F0DBF8B168804608887C
:2030500040F60202824211D0B0F5C15F0ED00A8B4FF61F60104040F4347008830DE0C046DF
:20307000A00A0020CDB600001DFE00000A8A4FF61F60104040F43470088204F1580090E809
:203090000C00002B08BF002A18D0042012F0A2FAA0B1A56D13F0D6FC854226BF401B401EB1
:2030B000401B000BF060F168708A401840F6C411F06081422CBFB0F5FA7FF160404614F09D
:2030D00093F810F0F3FC98B1B56930466FF4807100224FF00073A84704F13C0013F0BBFF84
:2030F000002808BF47F0020702D0192013F022FE75692DB1002130464FF080630A46A847AF
:2031100027F0005723E014F073F8014604F1440013F0A1FF0646B569A80813D296B125EA47
:203130000500B061084614F05FF8706868B165B12A46F068B6F9241075680023A84704E03B
:2031500010100440084614F04FF827F4804727B104F1EC00394613F013FCBDE8F883C04610
:20317000000004608B2D0020A5BF00008DAA00002DE9F04F0320ADF1540D12F081F8CA4C60
:203190000025022004F11C0141F80C5F401E8D60FAD104F14000A946062701467F1E21F8BE
:2031B0000C9BFBD14FF0080AC049A0F800A0C04A8160C049121D22F00303CF1A2762A36149
:2031D000E361A66904F11C08944618460A46B14200F29581B910E82700EB810121F8049CF2
:2031F0004FF6FC761F8006EA0C033746D21A00F1E80607EA02012661EC39A0F8E810284684
:203210001CF030F86061C249D8F80000DFF82C8320610A6808F10C00026049684160BD4996
:203230008346524612F0BCFD28B9BB4801685A46116040685060B948B94FC0F8B070C0F813
:20325000B850C0F8C850B74EC0F8CC50B64BC0F8B460B64AC0F8BC30B54FD0F8B010C0F8F8
:20327000C020C0F8C47009B1284688471CF076F8B04ECDF8389029460C2206F120000DF0C5
:203290002AFFAD4F0222ADF820A041F270737762708CADF82220616AB3621027099740F0B7
:2032B0001900708408A8884700280CBF0A9F2F1C0120ADF82CA0616AADF82E000BA88847D9
:2032D0009DF83000444620700D99616077B1D021397087F80190B87087F8039087F8049079
:2032F0003946BD600220FD6011F030F99449182001221BF06DFFE220594613F0C3FC18202F
:203310001CF052FA60706068B046C8F808000BF02DFB944F08F17000A060D8F80850894C83
:2033300049466762F520A56013F092F9864D05F1180005F10C010CF0D1FCA8600D2013F098
:203350008BFB00B1CA460E2013F086FB08B94AF0100A7E49A86813F071FD7D49C82205F161
:20337000240010F0C7FB7B48BAF1100F686011D1606A78B1C2686AB1FF204FF6FC778DF88C
:203390001000F81CADF8120004AEADF8140096E803009047704F07F1140007F108010CF0B7
:2033B0009DFC7860484613F067FD4E46BD1E824605F8029F02206870304613F0C3FD014648
:2033D00078685246C9B211F02DFB761C022EEFDB624907F120004FF4FA7210F08BFB606A73
:2033F000002845D00769DFF878A16FB10094514612A80A688988026012AE818096E80300F4
:2034100001234A46B847606A002831D0C26852B1514612A80B688988036012AF818097E850
:2034300003009047606A18B307690FB306208DF80800ADF80A0010AEADF80C9002AD009635
:2034500095E803004A460223ADF84020B847666ABDF840007769A08057B1BDF8400002AEB1
:20347000401CADF8400096E80300022210ABB84724A013F0A5FB606A062668B307695FB3A2
:203490008DF818600425ADF81A500EA8ADF81C9006AB009093E803004A462B46B84758B910
:2034B0000E981930814617E0B41500204DF90100952D0020004B00208DF818604846676A76
:2034D000ADF81A5006AE0F907C69ADF81C9096E803002A460FABA047CDF8389048460DF09A
:2034F00083FCE0200E2113F0B3F812F067FF08F10200012112F08CFF00F00AFFFCE726F854
:20351000029B64E654492053656E736F7200C046C8FF01007C0C0000F012005008020020AB
:20353000AD4101008946010021580100FD4901005DE40000B813002020BF02006C1B002047
:20355000AD890000D411002048180020754E01006967010001690100D81800203507010053
:203570009C0C0000B80200202DE9F04FDFF8E0C292F808B009AF88460646ADF1240D049371
:2035900038F07F05039206BF604600884FF6FF700590F08A800934BF002008203076F08A40
:2035B000C00834BF102080207076F08A400903D260460E30007800E00020B076F08A4108AD
:2035D0002CBF20240024000928BF44F010047568002108F07F08307D06916D1E02280EDBF1
:2035F0000C2808DC0C2803D1022044F40854069044F0030404E00D280CBF022001200443A6
:2036100096F8880008B144F00804210900D328B1DFF8C89299F8CC3013B908B1DF2051E141
:2036300021096DD396F88950DFF8B4A206F1240133891AF8052007910AEB000109790890C5
:203650008918491DC9B2C918B1F5006F80F23C8100284CD0049A039906F180000AF0DEFBEB
:203670000799002808603FD0806AB0F1FF3F39D070680023401E8DB196F88A10524600F8DA
:203690000119515D491EC9B241B1721892F87F20491EC9B2002900F80129F6D10799706661
:2036B0000968896AB162090E00F8011996F82A1000F8011996F82910089A00F8011996F877
:2036D000281005F0030500F8011902F0070141EAC501017071683289091AC9B27060891894
:2036F000318105E0DB2700E0F3277770EDE00023F08A7370C00828BF44F0100475686D1E94
:20371000336DA3B9B36D93B999F8E510012903D13089B0F5EE7F06DA200904D202290AD1FD
:2037300044F4005401E044F48054012002E044F4085402200690DFF8ACA19AF801000128D1
:203750000FD013F039F860B19AF8380048B196F86B00042805D1022024F48054069044F49B
:20377000005444EA8834B8F1020FA4B20AD0B8F1030F10D1ED1F09F1D801284613F055FCD4
:203790006D1E08E0B9F8BE00001205F8010999F8BE0005F80109069802280CD0B8F1000F6C
:2037B00015D0BBF1000F0CD004990598814208D144F040040BE0BBF1000F08D1B8F1000FF8
:2037D00005D00599081205F8010905F8011944EA8B24BBF1020FA4B209D0BBF1030F0ED1C8
:2037F0000399ED1F284613F020FC6D1E07E003990888001205F80109087805F80109BBF19A
:20381000000F05D00498011205F8011905F801093878F8B934480178307D0D2814D068B9AA
:20383000306D28B999F8A800411C89F8A8100AE099F8CD00411C89F8CD1004E099F8B600FD
:20385000411C89F8B610014605F8011904E0C0465A0F002044F48074201205F801092C70E2
:2038700070683189401B7560C0B240183081200927D3B06D00B130629AF8380010B1307D40
:203890000D281ED1726A12F1150002D113F00AFA726A916A481C9062306A3289B162471B2F
:2038B0000092D21B019090B20290706A96F888202B46153008F0D4F900281CBF7070071C83
:2038D00007D10020707005E0E5277770F32012F08CFEF8B209B0BDE8F08FC046A00E00202E
:2038F000440C000014150020E92C0020B0B50446BC480768ADF1480D002F00F0AC812078F1
:20391000401E112800F2A781DFE810F06E0156013C0127011F010801F100E300C300B20082
:203930008D005D0053004200A5012A001C001200F86B002800F08F81684621460CF068FEF8
:20395000F96B86E1386C002800F085816846002101220DF0C0FB60788DF80000396C78E1C5
:20397000F86A002800F07781684600210E220DF0B2FBA11C684612F007FFA57BA18900223D
:20399000ADF80A1005B101228DF80C20F96A61E1B86B002800F05F816846002102220DF01E
:2039B0009AFBA5788DF8015060788DF80000B96B4FE1786B002800F04E81684621460CF0E3
:2039D00027FE796B45E1386B08B36846002114220DF081FBA5788DF80150A3680193A2890F
:2039F000ADF80820A17B8DF80A1060788DF80000E57B8DF80B50237C8DF80C3094F9112074
:203A10008DF80D2061690491396B684688476068002800F020810146F2200870002048703A
:203A300010F094FD17E1B86A002800F014816846002124220DF04FFB6078A11C8DF80000A8
:203A50000DF1020012F0A0FE04F10C0103A812F09BFE257EE08A04F119018DF818500B2238
:203A7000ADF816000DF119000CF004F8B96AF0E0786A002800F0EF806846002102220DF020
:203A90002AFBA5788DF8015060788DF80000796ADFE0386A002800F0DE80684600211222E4
:203AB0000DF019FB658862796078ADF8025023798DF80520E11D8DF80000A5798DF80430AE
:203AD0000B220DF107008DF806500BF0D3FF396ABFE0F869002800F0BE8068460021012211
:203AF0000DF0F9FA60788DF80000F969B1E0B86910B120460FF0A0FBA07D002800F0AB8034
:203B1000A07820B9A069002800F0A58003E0A069002800F0A08012F0DFF99CE078690028DB
:203B300000F099806846002113220DF0D4FA6D46A01C0168406829600B22686004F10A019F
:203B500002A80BF097FF796983E03869002800F0828020460BF0D0F97DE0F86800287AD0C1
:203B7000684600210E220DF0B6FA6078A11C8DF800000DF1020012F007FEA089ADF80C008E
:203B9000F96866E0B868002865D06846002114220DF0A1FAA01C01686D4629604068686083
:203BB000A07A0B2204F10B018DF808000DF109000BF060FFB9684CE0786800284BD06846A1
:203BD000002110220DF087FA60786588211D8DF800000B22ADF8025001A80BF04BFF796889
:203BF00037E0C046741B00203868A0B36846002119220DF070FAA01C01686D46296040687C
:203C10006860A07A410824BF01218DF80810810824BF01218DF80910C10824BF01218DF848
:203C30000A10010924BF01218DF80B10C10924BF01218DF80C1030F07F001CBF01208DF81B
:203C50000D000B220DF10E0004F10B010BF012FF39686846884712B0B0BD70472DE9F04FA8
:203C7000C34E37688246ADF12C0D17B913F01AF83768DFF80C8308F10300DFF80C9305780C
:203C9000002D3FD0002538897968BA4B0795C400097818781034890906D340F6485191FB91
:203CB000F0F1091901F5AF743B7D60438400352B0CBF2F1C4FF4FA570DF12601E8200FF0C3
:203CD000ADFE9DF82600032808BF44F620673068007D3C19352807D111F02CFF0146306811
:203CF0006C300EF04DFF444302204F468DF8200007F10C000068069406A909F097F8AC48BA
:203D10000C3805709C4901209C4F08703978012902D0002102F04CFF30680489456813F091
:203D30007EF9DFF860822888000932D398F83870316877B34A6A4F6E906A4646B0F1FF3FB4
:203D500022D00FB3431C93628862030E07F8013991F82A0007F8010991F8290007F80109A0
:203D700091F828003870086A00940190401B201A80B2029091F88820486A8B6A153019466E
:203D90002B4607F06DFF00E0DB20F16F002840F0E380214628460CF05DFE642009A90FF0E8
:203DB0003DFE494698F83870087837B9774800780AF046FF012805D0CAE00AF041FF012800
:203DD00040F0C680DFF8C8C1A01C241D6D1EA1B2ACF87800C1F3022040F0080005F80109F1
:203DF000002629700227CCF884509DF82450ACF86A60002D0CBF674867486446C4F8C00040
:203E1000664DC4F8800068688047AB460A90BAF1010F54D0BAF1040F51D0BAF1000F4ED0EB
:203E300094F84000BAF1050F04F13005C0F3C0002CD0E8200DF125010FF0F0FD98F838006E
:203E500000B39DF8250003281CD1687B2B7C00F0F00005F1110140F00300687343F0180002
:203E70002874F4200FF0DAFDD8F89C00804704968DF814706686A064B0468DE88001D9F829
:203E90000C004EE0464B04F168050EE028B9687B00F0F00040F0010004E0687B00F0F0007B
:203EB00040F003006873404B6686049638468DF8147031468DE80300D9F80C0032E094F8E2
:203ED0003D0000F0F00040F0030084F83D0094F8400004F130010D46113140F0180084F87E
:203EF0004000F4200FF09AFD98F83800002808BF4FF4FA5002D0D8F89C008047A0640496E1
:203F10001F498DF81470D9F80C008B78002B06BFA4F84E6004F14C056686324639468DE868
:203F300006001F4B294604AA01F090FD1D490880DBF80810002809D41C4A92F900001C4F2C
:203F50006834401C10700A983C600DE00A9888471A200CF03BFD08E0002908BFE420F8D02B
:203F7000144A00201070E42088470BB0BDE8F08F700D0020241B0020971B0020A21B0020D6
:203F9000241A002014150020C4190020770F0020D81200204E9055550E7A5555B41500201A
:203FB00031A10000F419002099CA00009E1B00200C170020942D00202DE9F04FC24D4FF0EF
:203FD000000AADF1140DDFF81C83E868CDF808A000288DF80CA040D1CC4CBC49843C206806
:203FF000814210D0BA4981420DD0BA4981420AD0B949814207D0B949814204D0B8498142D2
:2040100001D012F04FFE12F069F921684FF0FF32012805D1C1F30330083806D0C01F01D067
:20403000012A02D10120E87001E085F803A011F06BFB4446206A00F1200118B912F032FE68
:20405000216A2031096805F1140088474FF4FA70E884A54FAF620626EE624446E26992F831
:204070002670E7B9A14892F8257001788F4216D05046342404FB002C9CF8267037B99CF8FB
:204090002530401C9942C0B2F4D103E09CF82500884204D1604610F04DFFD8F81C20DFF83D
:2040B00050B2D8F824001BC88BE81B00E878012814BF50460520DFF83C928F4C8BF800006F
:2040D00099F8157127B990690068C4F8A40005E0D0690068C4F8A40012F0EEF9632004A919
:2040F0000FF09CFC99F8E720104611F059F9B4F896C007462CF0070C4CF0010CA4F896C01F
:20411000D4F8980004F18806812A40F00F00C4F8980001DB842A05DB397B052914BF242106
:20413000292100E0212184F89C10717D812A01F03F01717501DB842A18DBBB7A6BB99DF8C0
:2041500010203F3262F305017175F28A4FF6C07303EA020141F0180113E09DF8102001F096
:20417000C00102F03F020A43114603E021F03F0141F002017175F28A4FF6E071114041F0B5
:204190002001F182FA7A397B491D5143D8F81C200A230CF0010C91FBF3F1C9044CEA114152
:2041B000F181F97A1923890391FBF3F161F31C203061308B92F824104FF6F77361F3020033
:2041D00003EA0001308392F8240000F008000843308399F9D6000EF0A1FAA4F8A20079686A
:2041F0003B68D8F81C203889401E414303EB51004FF47A71B0FBF1F0A4F8A800106A00782E
:20421000A4F88AA084F8AC00C4F88CA0707B00F0F00040F00100707312F040FEA0B9F87ACE
:20423000364A99F8E740B1FBF0F01070F87A022CB1FBF0F0C0B2B1FBF0F0687004D13048DB
:2042500002214170A8270770EF68D8F820402FB350460FF0BBFC287999F8E710884211D1AA
:20427000697999F81521E86891420CD10221524653468DE80600314602AA01F0E7FBC8F800
:204290000C6017E0E868D8F8201049688847D8F8207001201B493C68087000E024681A480C
:2042B00005F1140359463246A047E860D8F82400C8F8280099F8E70099F81571287105B0E2
:2042D0006F71BDE8F08FC046C419002000F0022000F0012000F00020008002200080012051
:2042F0000080002000170020D95C0100870F0020582D0020A00E0020D8120020241B00200F
:20431000241A0020A31B002040280020181300502DE9F041CA4CCB4DDFF830836088ADF1C9
:20433000600D4108C0F08B800CA808A90DF006FD012878D1404624300068D8B10769CFB16A
:20435000062002268DF808000022ADF80A600FABADF80C2002AE009396E803000C23B847C4
:2043700040B9BDF83C006084109F67621198A06212F054FB9DF82D00012805D00220207772
:20439000BDF82210A1820AE0032009AF20773A6804F114010A6078684860BDF82210BDF86D
:2043B000200009AA0EF0AAFA011C02D0A0A012F01EFE022010F026FEBDF830009DF82C70CF
:2043D00028870DA985F83A7005F1480012F0B5FDBDF8320005F13E0609A9A5F84600304623
:2043F00012F0ABFDBDF82200298FA887502012F023F9B5F84610532012F01EF94A20314647
:2044100012F040FC95F83A10E12012F021F9A98F4B2012F011F905F10800102111F0F8FF84
:204430000120207005E0012010F0ECFD002012F0B3FBA01C012111F0DDFF2046408880088B
:204450000DD3606A10F04CFF11F084FA00B2A081E08101F041FDA01C022111F0CBFF28891A
:20447000410805D305F10800012111F0C3FF2889810805D305F10800022111F0BBFF288989
:2044900001094BD395F8540005F1080600283DD0401E39D0401E02D0401E33D039E095F82C
:2044B0005010472012F0D4F895F85110542012F0CFF8A98F4B2012F0BFF8298F502012F0A6
:2044D000BBF80927032395F83A008DF8597016AA8DF85A305C498DF8580001278DF85B70E5
:2044F00018201AF075FEB4F84E00B4F84C1088420FD195F8520001280BD13046202111F0AF
:2045100087FF06E0032002E0022000E001200DF0B5FD3046082111F06DFF2889410911D35D
:2045300095F8520005F10806032818BF042802D1A86D10F0BDFE10F0ADF93046102111F069
:2045500059FF2889810907D30CF0B2FE05F10800202111F04FFF2889C10907D30CF040FB18
:2045700005F10800402111F045FF2889400A0DD395F8550012F010FB41F2883010F0C8FE0C
:2045900005F108004FF4807111F034FF4546E88840080DD368780026000904D3A878012853
:2045B00001D110F00FF86E70A81D012111F022FF6088002839D10A200825254CADF8120092
:2045D0004FF0FF37ADF81050616A059704A8884700282AD10720ADF84850616AADF84A002E
:2045F00012A88847149E1596F8B91A499DF84E20087890420ED19DF84C004A78824206D040
:2046100089684B6C33B100213246984702E03046FFF76CF9159840B1ADF818500320ADF860
:204630001A00616A079606A8884718B0BDE8F08141757468204572726F723A20307800C00F
:20465000B813002070140020836F0100D4110020B41500206C1B00202DE9F04F09AFADF188
:204670003C0D08900A92388809911E46ADF81800101C08BF002000F08481002700F1010908
:204690004FF0FF3A4FF0010BB8466CE1252940F063811078521C0A922D2818BFADF80680B1
:2046B00005D15846551CADF8060010780A9530281CBF4246434605D10A9908785A465B46B5
:2046D000491C0A912A28CDF80080554616D1306804930A99CDF808A0C01C4B1C20F003001C
:2046F000001D306050F8044C0A93002C0878009418D5ADF806B06442009413E044460AE09F
:20471000610001EBC40140180A99A0F1300408780094491C0A91302801DB3A28F0DBCDF87D
:2047300008A004932E282BD10A9908782A2801F101010A9111D13068CDF80880C01C20F021
:204750000300001D306050F8045C002D48BF454608782B46491C0A9111E0454643460AE052
:20477000690001EBC50140180A99A0F1300508782B46491C0A91302801DB3A28F0DB029366
:204790000AB1224604926C2804D04C2818BFADF8048005D10A990878ADF804B0491C0A9122
:2047B0000BA9CDF80C800FAB07916428059300F08B80692800F08880BDF818C0752872D07E
:2047D00078286ED06F286AD0702850D063283DD073281ED009980A990128A1F101010A91A5
:2047F00015D96B490C68B5F1FF3F03D0A84288BF6D1C00D8099D029508A80AA932466B4681
:20481000A047C7190A99039801F1010974E040462AE030680A99C01C20F00300001D3060CC
:2048300050F8040CBCF1000F01F10109014608B955A00146079112F087F90390B5F1FF3F83
:204850005BD0A842C4BF281C039056E03068C01C20F00300001D306010F8040C5D468DF82F
:204870002C000A990395584601F1010945E0082035680490E81C20F00300001D306050F89D
:20489000041C082210230FA80DF0AEF8401E0790402101700A99079801F1010929E00823F8
:2048B00002E0102300E00A230A99306801F10109C01C20F00300001D306050F8041CAA429F
:2048D000BCBF2A1C049210E00A99306801F10109C01C20F00300001D306050F8041CAA425A
:2048F000BCBF2A1C04926FF009030FA80DF07CF80790059D281A0390009C241ABDF80650CB
:2049100000945DB906E008A8202109AA10F095FF009C7F1C641E0094F5D503980546401E64
:20493000039075B9BDF80600E8B10098401E009019D408A8202109AA10F07FFF00987F1C8A
:20495000F4E70798411C0791017809AA08A810F074FF03987F1CE1E708A809AA10F06DFFBC
:204970007F1C09F101094A460A9812F8011C401C00290A907FF48AAE089808B14146017014
:2049900038460FB0BDE8F08F286E756C6C2900C0C00C00002DE9F04F002898461546ADF1BA
:2049B0002C0D00F0158111F47C1F40F00E8111F00F0F00F00D8107460591002006900A90F9
:2049D0004FF0000A0990544608944FF0010BCDF810B0044650460790059805990BEA000038
:2049F00021EA0B014FEA4B0B401E059100F0CD80401E7BD0801E68D0001F40F0E08005B1EC
:204A10002F660720152642F2D002022307F8010B01A907F8016BA2F1CF0007F8013B0EF0A9
:204A30003BFE684603A90AF0A7FD9C4801783E46812907DB9848B0F8B600842905DA49F6BF
:204A5000D05104E09448B0F8B60042F2D00108180099019A4FF47A6390FBF3F04018009038
:204A7000824206D8801ABDF80C300090581CADF80C00009B50085146814609041804030CBB
:204A900019430004534610EB090041EB0A0102F08DFEBF1D0090BDF80C309DF80C009DF8C2
:204AB000002006F8010B181206F8010B9DF8011006F8012B9DF8023006F8011B9DF803201F
:204AD00006F8013B0934327078E00220152607F8010B042307F8016BB8F1000F07F8013B68
:204AF0000CBF099898F80000241D65E01DB1EF6595F86B0006900520152642F2D002049B6F
:204B100007F8010B0DF10E01DDF8189007F8016BA2F1CC0007F8013B0EF0BEFD02A80FF089
:204B3000D9FC5E4801783E46812907DB5A48B0F8B600842905DA49F6D05104E05648B0F84B
:204B5000B60042F2D001081802994FF47A6390FBF3F09DF80E209DF80E3040183F1D029065
:204B7000000206F8019B00EB6300B0FBF2F002909DF808009DF8091006F8010B9DF80A30F8
:204B900006F8011BE41D337018E00320152607F8010BB8F1000F07F8016B034607F8013B3F
:204BB00004BF0A9807F8010B05D098F8000007F8010B98F80100641D07F8010BA4B20598F5
:204BD00000287FF409AF264661E011F00F0F01D000205DE080468A4602264FF4803908F1C5
:204BF000020509EA0A002AEA090A4FEA4909B0F580301AD0B0F5803014D0B0F500300ED0C4
:204C1000B0F5802009D0B0F5002004D0B0F580102AD1072404E0062402E0052400E0042451
:204C3000002704E00224012701E001242746A81C214600F073FC47B104F00F04C0F30A0151
:204C500041EAC42141F4004105E004F07F0400F0FF0141EA042105F8011B36180912B61CCE
:204C70002970B6B245196D1CBAF1000FB9D1022ED8BF00260BDDB01E4FF6FE7708F8010B8F
:204C9000B819C0F3022040F0A00088F8000030460BB0BDE8F08FC046D0290020870F0020E4
:204CB000BA482DE9F84F0025B94CB749056094F8E200002800F06381012800F02F81B54EC0
:204CD00002283CD0032840F05A8151F8250CD4F8B8100029A0F5C060C4F8D400B8BF4942DA
:204CF0000028B8BF4042814226DA4FF08057D7F8A4014568B4F8BC0030214FF47F420823A1
:204D100000903046A847D7F8A4014568B4F8C00004214FF4F802122300903046A847D7F8A6
:204D3000A401B4F8D070456820214FF440620A2330460097A847012584F8D8501AE151F8C8
:204D5000258C12F069F82F4600B901273946924F38680028FCD0B146012609F10409D9F8EF
:204D70002CA03E6009B112F05DF8CAF30720C4F8BC0012F051F8AA4600B9B2463B68002B92
:204D9000FCD0D9F800B0BAF1000F3E6001D012F049F8CBF38440C4F8C00012F03DF8AA4625
:204DB00000B9B2463B68002BFCD0D9F81C90BAF1000F3E6001D012F035F8C9F38120C4F8AA
:204DD000D000B8F5C061C4F8B81000F09C8094F8D80068B9C4F8D410D4F8C000C4F8C80060
:204DF000D4F8BC70C4F8C470D4F8D030C4F8CC30D4F8D410D4F8BC30002954BF02206FF012
:204E1000010004F1C802176801EB41014018411000EB917107EBA1001060D4F8C810C4F81C
:204E3000C43000291CDD1E293CDDD4F8CC0030B93429B4BF15391E21C4F8C81025E02A2922
:204E5000BABFD4F8C8000B381E20C4F8C800D4F8C4003F28B4BF401C3F20C4F8C4001FE08C
:204E7000D4F8CC00032812D011F10B0FC6BFD4F8C8000B30301CC4F8C800D4F8C400002885
:204E9000C4BF401E051CC4F8C450032508E011F1150FC6BFD4F8C8001530301CC4F8C800CC
:204EB000C4F8CC504FF08057D7F8A401B4F8C43030214FF47F424568364800930823A847B3
:204ED000D7F8A40104214FF400321123456831480096A847B4F8C860D7F8A40104214FF425
:204EF000F802122345682B480096A847D7F8A40120214FF440620A23B4F8CC604568254815
:204F10000096A84701E084F8D85040F2FF50404502D8801C40452DD208202EE051F8251CB7
:204F30001E4F4BF2F5204843060A3868C0F3814001280AD110F00EFD0FF062FB11F078FF10
:204F50003111C010484306EBE03694F8E50030B91348006820F07F408019460801E084F86D
:204F7000E5501048310C0660012741600E4D8760287808B90B2000E0052084F8E40004F001
:204F900029F9BDE8F88FC0462D400C402C500C40B80F002000A00C4000800C40B43F00504A
:204FB000102009403C600C40320C00002DE9F04FAC4C04F128000068ADF1240D0FF08EF81C
:204FD00008B111F06FF9A248DFF89CA2DFF888B20068A24E089010F099FD10F08DFFE5692F
:204FF000A769B5F57A7F13D0C01B4FF47A720023A5FB000102F0DAFB80464FF47A7200235E
:2050100011F08EFC2A46002302F0D0FBC01901E0A0EB0708A0618D488C49006820F002002C
:20503000086070688047DBF80010DBF8043045466918B1F57A7F0DD34FF47A72B1FBF2F225
:20505000D2184FF47A73CBF804201F46B1FBF7F25A43891ACBF80010B168884770688047AB
:20507000DAF8041002466818B168CAF8040010468847DAF8000000285FD007464FF00009B0
:20509000706880474FF000081FFAA5F3079083B95FFA95F36BB93979E8B2884204DD7968B9
:2050B0002846884209D20AE03879E9B2401A387108E079682846884201D3414601E0796876
:2050D000091A7960B88878B9FB8853B9FB6843B13B8933B1B87A19460AF0ACF9F86878605D
:2050F000B88808B9FB880BB13B896BB9B9F1000F04BF3868CAF8000003D03868C9F8000066
:205110003868B846074601E0B9463F68B16807988847B8F1000F0ED0B8F8043043B9B8F860
:2051300006302BB998F80A00B8F808100AF082F9404610F0C1FE002FA2D144484349006807
:2051500040F002000860E06828B3804723E015F8060C2169A5F10C07032819D0E16A9DF872
:2051700016000978884210D115F8080C10F030F9B979012903D0022908BFA87000E02870E2
:20519000002029460DF08AFB05E011F08BF802E009B12846884708200727ADF81000716AC6
:2051B000ADF8127004A88847069D0028CFD0294800680088C8B17068804726490968002258
:2051D0000D880A80B1688847089A00202946207090470546FF202070706880471D490968B0
:2051F0000A8815430D80B168884710F08FFC0746B7F1FF3F1CD0706807B9194F216AB94210
:2052100038BF0F1C80471C230546626AADF802300820ADF80000716A019268468847A16AA5
:205230003846491CA1620FF0AFF9B1682846884708200A27ADF808004FF0FF35ADF80A70E3
:20525000716A039502A88847C5E6C04610E000E0AC0C0000842D0020B01B0020B415002074
:205270008EC2F52894190020682D00202DE9F04FA54C064600200F46ADF13C0DDFF8909248
:20529000ADF80C002068A44D017D252900F010816C3005A903F05AFC002818BFC0B240F053
:2052B000308120460068C18AC9080DD3007D03280AD09DF81F0038B99DF820004C4638704D
:2052D000B534207000201CE101A804A90AF054F9A5F12F018B4691F82F30019A3468DBF802
:2052F00008104FF47A7A504641F208155843891A0AFB12000AFB01F1001B091B8D42C8BF88
:20531000002965DC854205DD002803DD346804F5915434609DF81F00002857D042F2040019
:205330000DF135010EF0B8F910F036FE044606980DA9241A42F206000EF0AEF99DF83410B2
:205350009DF81D00FF2904BF0A218DF83410FF2808BF0A209DF834206C499DF81C30D046FF
:20537000B4FBF1F1801880B24843991008FB01F1814298BF081C2D1805A810F0EEFB9DF8EB
:205390001C203468B0FBF2F15143411A8BB251464B4308FB02F1CA1AC91A121B091B8D4269
:2053B00001D9002908D56942914216D2002A14D5B5FBF8F109B203E06900B1FBF8F189B214
:2053D00032684FF4916303FB012405E0002004E0306841F630342418346005460DF1120181
:2053F00002A80AF0C9F80298DBF80810B4FBFAF210180290814203D99BF82F30834204D92B
:205410004B4603F15804267836BB9DF81C0055190004A84298BF2D1A9DF81F00002808BFBE
:205430009DF8200016D09DF81C00B5FBF0F084B29DF833000EF07AFC9DF83120014620467B
:205450000EF00CFC044610F075FB024608A920460EF052FA4C460DE0814204D8BDF81200EE
:20547000401CADF812004C46BDF8120094F85B100CF0A2F93870244E84F8B5003068007DC2
:2054900005287FF41FAF2348007820B111F094F900283FF417AF387803A9ADF80C0042F2EA
:2054B0000C0003F0C9FDBDF80C00A4F8B00009E768460DF10E010AF05FF83068009A2B7839
:2054D00041F208144FF47A7101FB0202009259438A1A944210DCA1F5FA619142BCBF00F577
:2054F000FA6030604C4694F85B10208F0CF064F901460020397002E039784C46652084F8EB
:20551000B5100FB0BDE8F08F700D0020A0860100D02900205D0F0020BB2A0020F0B5044676
:205530000846ADF16C0D401E6BD0401E0DD0801E00F00381401E00F0E980401E00F0DB80B0
:20555000401E00F0A88000203CE142F2010007A90EF0A2F842F20B0008A90EF09DF842F254
:2055700006000DF165010EF097F842F207000DF166010EF091F842F2050019A90EF08CF880
:2055900004A809F061FE05460DF1670142F209000EF082F89DF86700002808BF002303D0B0
:2055B00002200FF0EBFF034607A8006808A920600988271D3C46B81C218005F007079DF8DB
:2055D00065609DF864109DF8662000F8011B9DF8674000F8016B03F0030600F8012B620795
:2055F00047EA926104AC41EA8611012700F8011B9DF8672000942946019707F05DF80A308C
:2056100099E042F206000DF165010EF045F842F207000DF166010EF03FF842F2040019A959
:205630000EF03AF804A809F00FFE05460DF1670142F208000EF030F89DF86700002808BF7A
:20565000002303D001200FF099FF03469DF864009DF8657004F8010B9DF8666004F8017B05
:205670009DF867209DF86770790704F8016B03F0030705F0070646EA916004AE40EA871017
:20569000294604F8010B002700962046019707F013F8001D4FE042F2150011A90DF0FCFF7F
:2056B00013AD42F2160029460DF0F6FF15AE42F2170031460DF0F0FF17AF42F2180039466D
:2056D0000DF0EAFF11A801682160406860606A6804F108035A6028681860306803F10801A0
:2056F000086074684C60386801F1080528607A686A60202066E042F214000DF122010DF0EB
:20571000CBFFBDF8221002200A1258E009A8002120220BF0E0FC42F2130009A90DF0BCFFB6
:2057300009A811F011FA024609A920460AF0A2F909A811F009FA80B244E042F20E0002A9AF
:205750000DF0AAFF0DF10A0142F20F000DF0A4FF0DF10B0142F20A000DF09EFF03A942F2E5
:2057700010000DF099FF0DF10D0142F211000DF093FF0DF10E0142F212000DF08DFFBDF803
:2057900008009DF80B209DF80C709DF80D609DF80E509DF80A1004F8010B02F0010200126D
:2057B00004F8010B07F0010042EA400206F0010042EA800205F0070042EA4012042004F82C
:2057D000011B22701BB0F0BD2DE9F04F06469E48001D0068ADF1340D80470B900AA98220F1
:2057F00004F0A6FE9DF8280018BB00248DF828404FF6FF75ADF804509DF82800ADF80650F6
:20581000FF2108228DF8000002A811F032FC8DF81840D420694602F0B1F99DF82800401C9B
:20583000C0B28DF828000328E4DB82200AA902F0A5F90020DFF808A2DFF808828DF82800BB
:2058500081469DF828008DF8019069468DF80000D02004F06DFE01274D46E8B99DF80B30EF
:20587000012B07D19DF80A0020B90DF1020011F027F888B9747B002C0CBF052209224F466E
:205890009C4209D10DF1020006F10E0110F014FC002818BF012507D1002F40F0BF801DB9B9
:2058B000707F002800F0BA804C469DF828008DF8214008A98DF82000D12004F039FE0028C8
:2058D00032D19DF82200FF282ED08DF800006946D42004F02DFE002833D102A8311D082244
:2058F00010F0EAFB00B330887788ADF80400ADF8067045B1307B9DF82810B7698DF818005A
:205910000DEB81010F61D420694602F037F975B1307F9DF82310884209D08DF8230008A92F
:20593000D12002F02BF902E0641C032CBDDB032C74D14F468DF80070D420694604F0F8FD9D
:2059500028B1DAF808100B988847192074E002AB184610F0B5FF4C4600B101242046341D97
:2059700030B918462146082210F0A6FB00284AD030887388327BADF804009DF82810ADF8E1
:205990000630002D8DF818200DEB810000F110000CBF4946B1690822016002A8214610F04D
:2059B0009BFF98F8380030B1D8F888201AB19DF80010204690474C469DF828008DF821403A
:2059D00008A98DF82000D12004F0B2FDE82807D09DF82200FF2803D0641C032CECDB10E0CF
:2059F0009DF800008DF82490337F8DF8220069468DF82330D42002F0C1F808A9D12002F0B6
:205A1000BDF8032C02DB7F1C032F93DB032F05D1DAF808100B9888471A200DE09DF8280032
:205A3000401CC0B202288DF82800FFF60AAFDAF808100B98884748460DB0BDE8F08FC04632
:205A5000B415002014150020B41500202DE9FE4F9B4692468946054611F0CAFB02908C48B9
:205A7000353801680CAFA94208BF416801A84A4653460090284603F09DFF834C061C13D1F6
:205A900094F8880140F0040084F888010298C4F87C5111F0A9FB9DF8040002280CBF6FF0F3
:205AB00002086FF00108ECE005F1780010F054FBB08CA4F85000B6F92480C6F808909AF878
:205AD0000400C6F804B086F82600A6F824806F48F56097E80C00202106F1100719401040CB
:205AF00087E80300002786F82770F06840680078022809D19AF80500012805D196F8270021
:205B100040F0100086F82700029811F06DFB94F88901042807D1D4F88001B4F9841194F858
:205B3000862111F02AFA11F063FB814694F8890130F004033ED104F13C000368D3B9314678
:205B50000FF076F938B3A5F8C08096F8270040F0800086F8270085F8C270E07920B1207884
:205B700010B101202072E771484611F03DFB484800781FE004F13C0031460FF059F950B181
:205B9000A5F8C08096F8270040F0800086F8270085F8C27048E0B4F9500000F6FF706FF373
:205BB0001F30A4F85000484611F01EFB6FF00100BDE8FE8F02280ED196F8270040F08000F2
:205BD00086F8270085F8C270484611F00DFBB6F92400BDE8FE8F012811D104F1C80010F0FD
:205BF000BBFA96F8270040F0800086F8270085F8C270206C0028E7D1484611F0F5FA206CB1
:205C100000282AD12078A76400BB6079012838D011F0EEFA8146A079A0B9B0680CF0FAFABF
:205C300058B9607A012803D1484611F0DDFA28E0484611F0D9FA04211FE004F1C80011F0BA
:205C5000CBFAF1E7134901200870EDE7012010F0A7FB192011F06EF813E0206CC06840681C
:205C7000007802280DD1F06840680078022808D19AF8050028B94FF4004104F1EC0010F03C
:205C90007FFE4046BDE8FE8FA00A0020FDEFFF9F290C00208B2D00202DE9FE4F0646307DE2
:205CB00001280AD196F916000CF038FD4FF6FF71814208BFE82000F00281F07B814A20B931
:205CD0001146491C0978022908DB012803D110460078022802DBF120BDE8FE8F346AB6F808
:205CF000289096F8347096F835B0B58B4FF000085FEA040A17D0744890F83830002B2ED09D
:205D1000016D00292BD004F0FF0088476E49096D04B20AF47F008847001900B2001D00B256
:205D3000C43084B200E0C4240DB12D1DADB267480078012809D147B16548C11991F8048044
:205D500010F80B002418641DA4B205EB090020184044801C80B210F011F8071C02D11A2051
:205D7000BDE8FE8F08EB09002B193881002D07EB030078600EBF0020E019801C00217422B5
:205D9000C7F8A00007F10C0011F073F94C442D1907F13C00FF211022A7F84C5011F069F929
:205DB00007F12C000F21102211F063F900243C707C707868716A328D09F05CFE07F18000EF
:205DD00006F12C010B2209F055FE07F18C00314610F0FEFB7089A7F89600307B87F8980032
:205DF000707B06F10E0587F899002A6869460A60AB888B80AA798A719DF80010204601294A
:205E100008BF01209DF80110012908BF40F004009DF80210012908BF40F008009DF8031047
:205E3000012908BF40F010009DF80410012908BF40F020009DF80510012908BF40F040002C
:205E50009DF80610012908BF40F08000A7F89A00707D87F89C00B07D87F89D00B28BA7F880
:205E7000A42022B1D7F8A000B16909F003FEB07F87F8A600306AC7F8A800B7F8A400C0B1DF
:205E9000D7F8A000A8B17868401E7860F82101707868401E78600470B7F8A410B7F8A460EA
:205EB0007868401A786039897018801C38817868B8650848007839460CF0F0FC2046BDE8EA
:205ED000FE8FC0469E0D0020141500206C0F0020440C00003C160020F0B500214422ADF1E4
:205EF000540D02A80BF0F7F8F22013A910F0C2FE834DBDF84C0013A9A5F86800F32010F06A
:205F1000B9FEBDF84C000DF10901A5F86A00E22010F0A0FE688CADF81200410806D305F147
:205F30000C01096805A80160BDF81200810805D3291D098806A80180BDF81200C10807D32D
:205F500005F1100109680DF11A000160BDF81200010908D30DF11E0005F14C01242209F0F6
:205F700089FDBDF81200400903D3A86A12906F6A11976448007800280CBF012100210120F5
:205F90000BF00CFEBDF8120041082CBF0F240B24810824BFA41CA4B2C10824BF241DA4B2CA
:205FB000010924BF2434A4B2400924BF0834A4B220460FF093FC071C00F09F8005260DF129
:205FD000090100F8016B0A68026049684160BDF81210083010F04AFFBDF8121084464808D4
:205FF0000BD3BDF81410604610F040FFBDF8161010F03CFFBDF812108446880807D3BDF81F
:206010001810604610F032FFBDF812108446C8080BD3BDF81A10604610F028FFBDF81C1095
:2060300010F024FF8446BDF81210374A9388080949D3BDF81E10604610F018FFBDF820103E
:2060500010F014FFBDF8221010F010FFBDF8241010F00CFFBDF8261010F008FFBDF8281054
:2060700010F004FFBDF82A1010F000FFBDF82C1010F0FCFEBDF82E1010F0F8FEBDF8301056
:2060900010F0F4FEBDF8321010F0F0FEBDF8341010F0ECFEBDF8361010F0E8FEBDF8381058
:2060B00010F0E4FEBDF83A1010F0E0FEBDF83C1010F0DCFE194610F0D9FE117810F0D6FEA3
:2060D000BDF812108446480906D3119960460EF01CFC12990EF019FC05F1140122463046D8
:2060F0003B4605F07FFB0820ADF80260074D01972968ADF800006846884715B0F0BDC0465A
:20611000B8130020DA180020D4110020D81500202DE9F047DFF80CA20746AAF13500DFF89A
:20613000F8810068800880F0E7800FF013FC814908310B6800261C17641C990D0AD2C0F17F
:206150003E0110F10A0F4FEAE101D8BF08218C42B8BF0C1CDFF8C4C1990E0FD2590E0DD363
:206170006246143A1168C1F304211629A8BF20391268C2F30462162A0EDB0CE0634AD2F8A7
:206190007C11C1F304611629A8BF20391268C2F30442162A00DB203A61189146162905DAF2
:2061B00011F10A0FB8BF6FF0090100E01521584C584D01F01F0242F4F85222802A6812F0AD
:2061D000030F18BF0126D20828BF46F002060FB146F00406424692F90740041B052C04DA18
:2061F0009479B44208BF918866D00F28A0F10F0827DB08EB0014A4F1F0084FEA282EBEF1C3
:20621000070F88BF4FF0070E7546062D88BF06255CF82570042404EB850465462C59E41BA5
:2062300004F0FF05F70824BFC4F307273D44B70824BFC4F307473D44770828BF05EB146517
:2062500001E00025AE465CF82EC0F7080CF0FF0424BFCCF307273C44B70824BFCCF30747F5
:206270003C44770828BF04EB1C64ADB2A9EB0101A8EB0E277D43002905F1800504EB152470
:20629000D8BF012103F0FF0334254D43A9B259434FF6FF73B1FBF4F18B4238BF191C802877
:2062B00089B2918005DA10F1800FB8BF6FF07F0000E07F20D0719671194800681F29106076
:2062D0004FF0000008D340F2FF128A4206D24908401C8A42FBD301E01F219180124F0F398B
:2062F000090940EAC10047EA0001CAF8FB1F0026CAF8FF6FBDE8F0870C490D4F42460820B0
:206310000F60921D1070BDE8F087C0463C1100506E62084024220840782D00209C130050A6
:20633000082009403500094000E7A48030100940FDFDA400AC3F00502DE9F04F0128ADF1D5
:20635000140D40F0EE80DFF814B2DBF8DC00012840F0E4800220CBF8DC0010F039FF0290DA
:2063700001200DF015FE5FEA000806D00120CBF8DC00029810F028FFD5E010F021FF6C49AA
:2063900003900020086001200FF024F9012818BF002003D100200CF091F90120654900909C
:2063B0000020654F08603868112010F053FD00280CBF00240124102010F04CFD08B144F0CE
:2063D00002040F2010F046FD08B144F004040B2010F040FD28B159480068594E016B30882B
:2063F00088470A2010F036FD002600B101264FF0805A0AF5DC75301C04D02868514E016B3F
:20641000308888475048012606602868816944F0200088474D48066010F016FD00F0010123
:206430000191400814D24A4810F0C1FC8146B9F1040FF8D0B9F1010F05D1DAF8D80142680C
:206450004348032190474349086820F0030008600020FFF75DFE2B683868986B8047019828
:2064700001280DD0B9F1010F05D1DAF8D80142683748314690473749086840F003000860C9
:206490002C48066028684169204688470B2010F0E1FC20B128682A4BC16A188888470A2001
:2064B00010F0D8FC20B12868264BC16A188888472548032206602549CBF8DC2000230B60D9
:2064D0002868416B204688470128F9D1386804200DF05EFD044616481F49066038680868A6
:2064F0008009FCD30098012802D130460CF0E6F810F098FC08200DF04BFD07460398CBF8A4
:20651000DC6010F059FE0CF027FA029810F05CFE57EA040018BF4FF0FF3804E06FF00408E6
:2065300001E06FF00108404605B0BDE8F08FC0460C400940000222432C200940B801001043
:20655000DE090000DA0900002820086080010443004003402422084014100940B80F002084
:20657000804A2DE9F04F13680546ADF13C0D0DF12A000360526842607B4C94F8B30005F15C
:20659000280105F12807002800F0E8806878002840F0E48010F010F9DFF8D091DFF8D48114
:2065B00000B3042046466A68A873301D12780068042A00F0958095F83000022812D14846B1
:2065D000007801280ED06A4905F1280002220E4620310FF0E5FB28B906F1160105A810F017
:2065F00024FD05AF686E002800F0B880012102AA09F0F4FE002840F0B1809DF80800A87396
:20661000E86C40B139460DF11E0208ABFCF774F9002840F0A38008A80090686E39460DF167
:206630001E0306F091FB002840F0988048460078012851D04FF400500DF122010DF02CF812
:206650000DF122000DF12A0108220FF0A9FB38B10DF12200394608220FF0A2FB00283BD192
:2066700094F85900002837D0A66CB4F8445042F2010004A90DF010F8049A4FF0004100207F
:20669000E2FB0610061C206D10F0A4FA86190498B04202D86D1C361AADB247467868804737
:2066B0005FFA80F8206CB04204D1208FA84208BF002608D026642587002084F835000FF042
:2066D0006BFC0126E064B968404688470EB10AF0A3FE012084F85800002084F859003DE001
:2066F0008B468047264C0D9095F8307022480A264FF00009804610F807A0207AB84206D1F4
:206710005246204659460FF0D7FC012804D0761E04F10C04F1D100E0A1465FEA09070FD1A2
:2067300098F80601164F461C810088F8066101EBC001F0B27F180A2804BF002088F8060101
:20675000384659460A2210F0C7F80C48094900788968B8720D9888470420A8730FB0BDE8D1
:20677000F08FC046640C0000D029002015150020340F0020B4150020CC100020C41900206C
:206790005A1100202DE9F043002B08BF002A10D10029BCBF00204FF0004106DB50EA0107B1
:2067B0001CBF6FF000006FF0004109F05EFEBDE8F0835FEA530898EA610803D50026404273
:2067D00066EB01015FF0000913F0004E03D00026524266EB03031C461546002C08BF8D424A
:2067F0009CBF2C1C0025070C47EA01470E0CB44208BFBD429EBF240444EA15442D04070A11
:2068100047EA01670E0AB44208BFBD429EBF240244EA15642D02470847EAC1774E08B4429E
:2068300008BFBD4200F29280870847EA81778E08B44208BFBD427BD8C70847EA4177CE0893
:20685000B44208BFBD4265D8070947EA01770E09B44208BFBD424FD8470947EAC1674E097C
:20687000B44208BFBD4239D8870947EA81678E09B44208BFBD4223D8C70947EA4167CE09C4
:20689000B44208BFBD420DD8E60146EA5566EF01B14208BFB84201D3C01BB14159EB0909DA
:2068B0004EEB0E0EA60146EA9566AF01B14208BFB84201D3C01BB14159EB09094EEB0E0EF1
:2068D000660146EAD5666F01B14208BFB84201D3C01BB14159EB09094EEB0E0E260146EA0F
:2068F00015762F01B14208BFB84201D3C01BB14159EB09094EEB0E0EE60046EA5576EF00FD
:20691000B14208BFB84201D3C01BB14159EB09094EEB0E0EA60046EA9576AF00B14208BF1D
:20693000B84201D3C01BB14159EB09094EEB0E0E660046EAD5766F00B14208BFB84201D329
:20695000C01BB14159EB09094EEB0E0EA14208BFA84201D3401BA14159EB09094EEB0E0E5F
:20697000A34208BFAA423EBF2D0A45EA0465240A8AD373464A465FEA080803D500264042F6
:2069900066EB01015FEA480803D50026524266EB03031E4617460B46024631463846BDE81E
:2069B000F0832DE9F043044694F830900F46984615468B20ADF1340D0DF10A0103F0B8FDAC
:2069D0008A20694603F0B4FD94F8250000283ED1B9F1000F19D1BDF80A104FF6FE708842D3
:2069F00005DCBDF80A1088422FD1694615E0B4F844009DF80A608DF80C0000128DF80D0045
:206A1000BDF80A008DF80E601BE0B9F1020F09D0B9F1030F19D104F1280103A810F005FBB6
:206A3000092612E0207CC00934BFB4F84200B4F844008DF80C0000128DF80D00208D8DF888
:206A50000E00001205268DF80F00002013E002280CBF05260926012818BF04F11C0104D1FE
:206A7000892006A903F064FD06A9324603A80FF033FF94F8260006EB0D01C8723A4603A841
:206A900031460AF08DFC002840F08E80B9F1000F19D1BDF80A104FF6FE70884205DCBDF801
:206AB0000A1088422FD1694615E0B4F844009DF80A608DF8200000128DF82100BDF80A0033
:206AD0008DF822601BE0B9F1020F09D0B9F1030F19D104F1280108A810F0A7FA082012E0E1
:206AF000207CC00934BFB4F84200B4F844008DF8200000128DF82100208D8DF8220000128D
:206B10008DF8230004203E6881460BA9822003F00FFD9DF82C10307B8142D8BF9DF82C0040
:206B3000002841D007460024722029460EF0FEFEB0689DF82C102018C8F800000078814284
:206B50002EDD2B68C10001EB0011D8F80000C91829604278012A1FD0807828BBB9F1040F23
:206B700006D0091D08A80FF025FD012816D017E008884B888DF82800042208A98DF82A306C
:206B900000128DF8290018128DF82B000AA80FF093FA012802D003E0807828B9002004E052
:206BB0007F1E04F10304BFD1F3200DB0BDE8F0832DE9F04F7C4C074660688946ADF11C0DEC
:206BD0008047A046714E724D6F4C8346012F68D00FF052FE00285FD06348007800285BD171
:206BF00062480078002857D161480078002853D16048007800284FD15F48007800284BD1DB
:206C10005E480078002847D15D480078002843D15C48007800283FD100200AF059FD0028C1
:206C30003AD127463878002836D1286A436CF068022104AA98479DF8100068B32C46B9F1C8
:206C5000010FBA4635461ED0524F226AE86897F9001011F1020F05D0926B97F90010904732
:206C7000E868226A4C4E96F9001011F1020F05D0926B96F900109047E868226A6FF0010157
:206C90003170397001E0E868226A01218AF80010D169884700206070D8F8081058468847DB
:206CB0005EE001200AF014FDD8F80810584688473A4800780F2842D12078012842D1384F66
:206CD00097F8C2000028FBD1286A436CF068022105AA98479DF8140068B197F8C20050B9F9
:206CF000207801282ED10020B9F1010F207029D00FF0CEFD26E0D8F8040080470222227040
:206D1000002302938DF80C20284F7B8181468DE80C00274BF0680837394602AAFEF796FE82
:206D3000002C01D50FF0BEFF224991F90000401C0870D8F80810EF604846884702E04846B8
:206D500006F0D0FE2078174D022803D1287808B10FF0A8FF2878012802D020780228FCD03D
:206D700007B0BDE8F08FC046902D0020922D0020942D0020912D0020932D0020961B0020F6
:206D9000971B0020981B0020A31B0020C419002000170020941B0020951B0020410F00201D
:206DB00040280020A21B0020B4150020D8120020A13101009E1B00202DE9FE437B4E8046D9
:206DD0000F46B8F1450F06D1304634220FF084FDC6F89C60E7E00FF01CFA3B2808BFF4205A
:206DF00000F0E280724C04EB8004A07810B9E178002938D0E178814208BFFB2000F0D48053
:206E1000B8F1580F25D0B8F1600F1BD0B8F1E00F0FD0B8F1E80F05D03A78904220DC91421B
:206E30001EDB20E006F1E7003978007881421AD1B9E097F900000BF071FC4FF6FF7181428B
:206E50000ED010E038880A280ADBB0F5804F07DA09E038888F2803DB46F2B041814202DA22
:206E7000E820BDE8FE83544D686880478146207862783946801994300FF02EFDA9684846BE
:206E900088474046503800F08C80801E73D0401E00F084808D387CD0401E63D0401E75D091
:206EB000801F1BD00D387ED10E2096F815718DF8000017B11B208DF8000096F9D6109DF94A
:206ED0000000884203D0E0206946FFF775FF0FF0F3FA96F81501002841D164E0032096F82D
:206EF000E7108DF8010081294FF005008DF8020006DB842904DA8DF8010008208DF80200EF
:206F10009DF8010096F8B910884204D04F200DF10101FFF751FF9DF8020096F8C51088425D
:206F300004D057200DF10201FFF746FF214C94F83800A0B10FF040FC88B1E26E7AB1022027
:206F500000278DF803000DF103018DF8047042F21B009047E26E42F21C0001A990470BF035
:206F70003BFE20E096F8D7000CF0D2FA01281AD01A20BDE8FE8396F8BD0018B902200DF0ED
:206F9000F3FB10E002200FF0BDFE0CE00FF044FC09E096F9D6000FF0AFFD04E00FF048FCDC
:206FB00001E00FF09FFD0020BDE8FE83A00E00209C02000014150020B41500202DE9FF4705
:206FD00007467878002840F0E78097F8961002291CBF0329E82097F88B108029C8BFE820D4
:206FF00097F88C10092901DB0A2900DDE82097F88D1009B1042905DB8029C0F2CC808629E7
:2070100080F2C980002840F0C780684C04F1E7000078884204D007F18D01E820FFF7CCFE12
:2070300007F18C01E720FFF7C7FE07F18B01E120FFF7C2FE07F198015020FFF7BDFE97F87D
:20705000960002280CD04FF6FE70A4F8B40007F18E0104F1AA000FF0E8FF07F18E0504E006
:2070700007F18E052888A4F8B400514807F180010B220FF031FC4FF001080220A7F816806B
:207090002946387501A80FF0A3FA97F89A60B7F89890786807F19A01002EA0F10100786014
:2070B0000CBF002040464E780EB140F002008E780EB140F00400CE780EB140F008000E79DB
:2070D0000EB140F040004E790EB140F0800079684A1E7A60374B08703E7D7968481C386284
:2070F000701E0026087038893E65801C38811878BE65002840D04FF0040A87F86960F88A99
:2071100087F86BA0C00934BF94F8B90094F8E20087F86A00296807F16C0001602B890381EF
:207130006C6844600FF048FB30BB07F16C0007F18E010FF07AFF204C206810F47F0F0CD0D5
:2071500087F82CA0206807F12C01424600F47F003863384602F06CFB206810F0FF0F0BD049
:207170002A2087F83C00206807F13C0100F0FF003864384606F01EFF00963846832101AABE
:207190004B46FCF7F1F9061C02D1384607F03CF8301C01D106E0E820787018203870384681
:2071B0000BF0CAFD0090BDE8FF87C046A00E0020C82B00204C150020AC0800002DE9F047D9
:2071D000064637680C465FEA0208ADF1180D14BF00214FF0FF3107F1480081460FF0E8FFFC
:2071F000002808BF0B2000F0DF80002565707148FC60B8F1010F057004D065700220FC60B2
:207210000EF03EF82078012840F29080801E012857D9801E01282CD9801E012800F2B88073
:207230000FF0E6FF8246A078009021782846062908BF0120019001200290A068228A636809
:20725000E16806F01FFD074650460FF0CDFF002F40F0A080B8F1000F02D00FF0A1FA02E090
:2072700030460EF08DFC002800F087800FF0F1FE21E00FF0BDFF012782460097A168A2788E
:20729000606824782B46042C08BF3B1C08F02EF8074650460FF0A8FF002F7BD1B8F1000FE1
:2072B00002D00FF07DFA02E030460EF069FC002863D00DF085FF3E49C1F8B0510D600746E4
:2072D00068E00FF095FF8246E08A0090E0680190208B0290A0780390207D04900121059157
:2072F00022782846022A08BF081CA368E178626802F0E0FC074650460FF076FF002F49D1C3
:20731000B8F1000F02D00FF04BFA02E030460EF037FC002831D00DF083FF071C3AD1E078D8
:20733000A168E28A236909F09DFDC8E70FF060FF8246E08A0090E0680190208B0290A078AC
:207350000390207D049001200590277807B90546E1786268A368284602F06AFD0746504621
:207370000FF042FFB7B9B8F1000F02D00FF018FA02E030460EF004FC08B9142014E00DF076
:2073900037FF071C06D1E07821690CF021F896E74FF0FF37B8F1010F02D002200DF02EFDEF
:2073B00048460FF01DFF384606B0BDE8F087C046504502408E2D00202DE9FE4F794C074697
:2073D00094F83D00002800F0DA80DFF8DC81B7F84210B8F8BA00884240F0D18007F1280058
:2073F0000EF044FB002800F0CA80002598F8BD0084F83D5010B102200EF03EFE6148007825
:2074100010B101200EF038FE387C400905D310200EF032FE80200FF07DFC20200DF0A4F921
:20743000594E06F120000CF09BF87A6851781078334600EB0120C0F30321C0F3003684F8FB
:20745000391000F00F0184F83A60C0F3031684F83E1098F8E30088F8C0600F2804D088423F
:2074700002DDD67806B9014688F8A11098F8A1A083F84050BAF10F0F09D194F83B00022828
:207490007DD10DF03DFD07F0FBF8BDE8FE8F3F480078012803D001202946FFF789FB4348AB
:2074B0004068804700900EF057FC3948DFF80091DFF8E0B0066898F8A12099F80030D9F8CB
:2074D0000400311A980091FBF0F05BF822100CF085FFC9F804605BF82A0001912E4EB06084
:2074F000F0600CF097F9019831680DF03DFD09F0E5F92E4900988968884794F83B000228A0
:207510000DD127480CF02CF898F8A12034F812004FF470719140091A21480EF0CFFA98F887
:20753000C030388929460BF009FE20630F2B14D098F8A11094F83900994208D0401C6FF004
:207550000F0598408101A1EB80016D1805E0401C98408501A5EB8005A03D6563022004F1AB
:20757000200584F8380028460BF0FAFF0B48A062616B28460EF0A2FA10200FF0CBFBBDE8FD
:20759000FE8FC046D32B0020782C0020A21B002040170020840A0000801B00206D0B010050
:2075B000882C00201C190020A00E0020B4150020241B00202DE9FE4F0CAF89469A46044665
:2075D0007D680292294603F0B5FE061C00F0D9803888F082DFF8CC81347598F8380018B112
:2075F000012C04BF1520307506F1800029460B220FF072F9012C04D00D2C1CBF7068401CEB
:2076100000D170683062002598F8380035650028B5654CD0052C18BF012C43D14FF0040BA3
:2076300086F86BB0F08A86F86950C00932BF57485D4816300078029986F86A000A6806F148
:207650006C073A604B687B60088938810FF0B4F840BB06F16C000FF0E8FC4D4F07EB840730
:20767000386810F47F0F0CD086F82CB0386806F12C01012200F47F003063304602F0D8F86D
:20769000386810F0FF0F4FF003090BD02A2086F83C00386806F13C0100F0FF003064304635
:2076B00006F088FC98F8380008B10D2C13D00095029A534630464946FBF756FF071C61D138
:2076D000E41F012C03D8707E40F020007076304606F09AFD56E00FF06FF8294600B101218A
:2076F0002B48343009B94FF00309052186F86B10016811F0F70F12D02A2186F83C1098F880
:207710000120006806F13C01012A00F0FF0030641CBF20F008003064304606F04BFC00951F
:20773000029A534630464946FBF71EFF071C29D1184806603489756801A964200CF06EF9E2
:20775000154E6D1E231DA01C99B2A6F87800C1F3022040F0080005F801090A1F297091B2B4
:20777000AA1CC6F88450104609F074F99DF8040000280CBF09480A48C6F8C000C6F88000FA
:2077900000E01A27F8B2BDE8FE8FC046590F0020A4080000F8190020D81200204E905555DF
:2077B0000E7A5555141500206C0F00202DE9F0411C4615468C4208BF854282BF00230022BD
:2077D000E5E0002C08BF002D0AD100290EBF00286FF000006FF0000100F0E1F8BDE8F0811D
:2077F0005FF000085FF0000E002C08BF8D429CBF2C1C0025070C47EA01470E0CB44208BFD8
:20781000BD429EBF5FEA044444EA15445FEA0545070A47EA01670E0AB44208BFBD429EBF76
:207830005FEA042444EA15645FEA0525470847EAC1774E08B44208BFBD4200F2938087084F
:2078500047EA81778E08B44208BFBD427CD8C70847EA4177CE08B44208BFBD4266D80709B1
:2078700047EA01770E09B44208BFBD4250D8470947EAC1674E09B44208BFBD423AD88709F6
:2078900047EA81678E09B44208BFBD4224D8C70947EA4167CE09B44208BFBD420DD8E60168
:2078B00046EA5566EF01B14208BFB84201D3C01BB14158EB08085EEB0E0EA60146EA9566FE
:2078D0004FEA8517B14208BFB84201D3C01BB14158EB08084EEB0E0E660146EAD5666F0184
:2078F000B14208BFB84201D3C01BB14158EB08084EEB0E0E260146EA15762F01B14208BFAF
:20791000B84201D3C01BB14158EB08085EEB0E0EE60046EA5576EF00B14208BFB84201D3AC
:20793000C01BB14158EB08084EEB0E0EA60046EA9576AF00B14208BFB84201D3C01BB141DD
:2079500058EB08084EEB0E0E660046EAD5766F00B14208BFB84201D3C01BB14158EB080877
:207970005EEB0E0EA14208BFA84201D3401BA14158EB08085EEB0E0EA34208BFAA423EBFA0
:207990002D0A45EA0465240A89D3734642461E4617460B46024631463846BDE8F081704721
:2079B000F0B542F20400ADF11C0D0DF115010BF073FE42F2050005A90BF06EFE664C6748E4
:2079D0009DF81510A0666420414321666449C4F884109DF814104843E0676248C4F8A000BA
:2079F0006148007880B942F2020069460BF054FE68460EF041FA04F15C000BF0A3FA04F126
:207A100034000BF0BDFC27E042F2030069460BF043FE0EF08FF80546684629460BF0B0F8B5
:207A30002D1A04F1780084F85B500BF08BFA04F134000BF031FA012742F20200694684F803
:207A500054700BF029FE68460EF016FA04F15C000BF078FA84F85870E8200DF116010BF05A
:207A7000DDFF9DF81600032804BF012084F8B40094F8B80000286DD13C4D0021302205F194
:207A90000C0009F028FB20460021332209F023FB37482862374FAF6105F114000BF052FACB
:207AB00042F21B000DF117010BF0F6FD9DF817000DF1170185F8300042F21C000BF0ECFDC0
:207AD0009DF817109DF8170085F8311095F83010012641B148010EF005F8686308B90FF0BB
:207AF000AEFA95F8310040B100EB800080B20DF0F9FFA86308B90FF0A2FA1F4905F13C008C
:207B10000A270A684B6802607F1E436000F10800F7D1002195F8307085F88C1047B1686B6A
:207B3000FF220346C2777F1E997703F12000F8D195F8317047B1A86BFF22034602717F1E55
:207B5000D97003F10500F8D1281D062209F0C3FA84F8B86007B0F0BDD0290020113601008E
:207B7000E9F40000D56F010015150020CC100020A5B50000002A7515740C00002DE9F041B8
:207B9000704B714ADFF8B8810C46D128014610DCD12878D0713800F0B080401E00F0A98050
:207BB000401E00F0A280113810D04C3800F0868007E0D23853D0401E40D0401E33D0401E61
:207BD00028D008460FF02AF80B2802D1F420BDE8F0815A4D05EB8005A97809B9E87850B19E
:207BF000E878884208BFFB2000F0A6802278914269DC904267DB554E7068804729786A78C8
:207C100007464046401821460EF066FEB1683846884790E02178022955DA1846641C042293
:207C300000EB810084E0207803284CDA1746C100241D182201EB0011781879E026783046E8
:207C5000022840DA2C2505FB0680611C102239300EF042FE616905FB0680C1646BE0227849
:207C70006178022A2FDA02292DDA40462C2301EB42064F1C03FB0205022285F8387000EB07
:207C90004600A23018E022786178022A1BDA032919DA2C23404603FB020595F8303099426F
:207CB000A4BF4B1C85F8303002EB4202891801EB4101032240189030A41C39E02078677880
:207CD000022800DA17B1E820BDE8F08141462C22C5197E1C02FB00136A0083F8286002EBF3
:207CF000C50288180A227C30E6E724B3184608221EE004B3104648221AE0B4B9404600F1B6
:207D10007C04A0F1080200F1900300F1A201022042F82C4F9360401E116104F10A0403F18F
:207D3000090301F10401F3D105E040465822243021460EF0D1FD0020BDE8F081F8040000CE
:207D50004427002038280020F0270020B41500202DE9F843644C0746207808B10EF0A2FFAA
:207D7000A0460120614988F800000978012902D00021FEF71DFF5F4D60495F485C4C012F3F
:207D90002A68D1F800900078A77035D9BF1E52D07F1E13D07F1E02D0781E47D043E092F803
:207DB0006900607192F86A0020710020A07103F0F1F82A68002A64D1BDE8F883002860D07E
:207DD000564ED6F8981021B1032088472A6896F83800002855D0776D002F52D0D06D20B1CD
:207DF00002210023B8472A68776D106E002848D008210023B84743E000206071D18A4048B8
:207E1000C90934BF90F8B91090F8E2102171A77837B990F897701FB10229C4BF0220207161
:207E300003F0B8F82CE00EF03DFF29E0002060710FF027F924E0334F38788600D9F83C0067
:207E5000804779683C22401AB0FBF6F0B0FBF2F151436278401A9101A1EB8201091AD9F836
:207E70003C003C318FB28047274906FB0700086791F8740000F0F00040F0020081F874005E
:207E90002A682248007878B912B90EF00BFF2A685168087800F02000E0708878E07108785E
:207EB000800901D20FF000F8A078042819D0184D68688047A17802290CD016490F7817B960
:207ED00015490F7837B1022188F80010A9688847BDE8F883832188F80010A96888470EF000
:207EF0004BF9BDE8F883C046942D0020A21B0020241A0020700D00204C1500202017002077
:207F1000A00E0020241B0020D81200208C2D0020B4150020902D0020922D00201415002053
:207F30002DE9BC4305466D4800880021820804D2B5F89A20D20828BFE82110F0600F04D19E
:207F5000B5F89A00800828BFE8212889B0F5006FA8BFE82195F8980030B995F894000028C6
:207F700008BFF52100F0B580002940F0B280DFF87091D5F8A800DFF8708199F8381010B9AD
:207F9000012903D02BE0002900F0A2800EF014FC68B9D5F8A8104046BD3041F002010078BB
:207FB000C5F8A81018B141F00801C5F8A810D5F8A81011F0FF0F05D02A2085F83C0001F067
:207FD000FF072F6411F47F0F07D00420D5F8A87085F82C0007F47F00286399F838100020DE
:207FF00069B3404995F894700B6804226FB925232B750968C98AC90934BF98F8B91098F820
:20801000E21085F86A10891C08E015212975D98AC90934BF98F8B91098F8E21085F86A100C
:2080300085F86B2005F18C0785F869003B6805F16C010B607C684C603B890B8101E0012165
:20805000297595F89C70EF760446AC65B5F89A102C6595F89D30E9826A682B7795F82C70CF
:208070002A620F2F09D00246B5F8A40005F12C0100B90122284601F0DBFB28BB95F83C10C4
:20809000FF2901D1AF6D27B105F13C01284605F091FFC8B9009495F89810B5F8963005F109
:2080B0008C022846FBF760FA071C0CD12889B0F5006F03DA284606F0A7F804E0E520687002
:2080D00028460AF03DF93846011C02D1BDE8BC831821284608F016F8BDE8BC834816002091
:2080F00014150020700D0020A00E00202DE9F043894614460546ADF12C0D69460CF0C6FDBA
:208110005FEA000800F0C480AD1C0226284602A90BF0E5F8071C00F0BB809DF80900814536
:2081300009D0F6197D1908F10200B61CAD1CB6B2B042EBDCACE0401E05F1020500F08B8018
:20815000401E52D0801E38D0401E2BD0401E24D0401E18BF622040F0AB80202F40F0988095
:2081700028686F6805F10801206004F10806676001F108050A684B68326004F110077360AA
:208190002A6868683A6005F108067860306804F11801086073684B6089E0022F78D12888D0
:2081B000208084E0202F73DC20460021202208F092FF3A462046294677E0042F68D12888F3
:2081D000AD1C208015F8010BA070287800F00100E0702878C0F3400020712878C0F3800025
:2081F000607128784011A07161E00A2F50DD0DF112000021162208F06EFF28682D1D2060CD
:208210002988271D42F20B00398004A90BF044FABDF81000A18888423ADCA81C10F8011BC5
:20823000A17110F8011BE17110F8011B217210F8011B0123C1F3C202A2720DF1120200F019
:20825000F9F928B39DF82700A0819DF81670E78104F1100026E0042F1ADD0DF1120000217B
:20827000162208F038FF15F8010B207015F8010B607015F8010BA07015F8011B0DF1120291
:208290000023C1F3C2002071284600F0D3F908B967200DE09DF82700E0809DF81670278166
:2082B00004F10A000DF11601112207F0E3FB00200BB0BDE8F083FEE72DE9F04F684C206829
:2082D000ADF12C0D002840F0C78004F124063068002800F0C18063480078022800F0BC808F
:2082F000624D281D006880470A90606AB046074678B35D4E4FF0000A4FF01D093B7D082040
:20831000711E11F8012F9A421ED0401EF9D14046394652460CF082FA787E30F07F0005D113
:2083300094F82F00401E84F82F0004E094F82E00401E84F82E0087F8019057F80CBC38461E
:2083500009F0FEFF5F4602E0BA4657F80C7C002FD4D1352007F076FC454EA968002849D141
:20837000452007F06FFCA96800283DD1D8F8000038B1017D252904D050F80C0C0028F8D135
:2083900010E078B196F8580050B3684601A907F0F3F8384800990078001F884213D801200B
:2083B00086F85500152007F04DFCA96848B10A98884720680DF106016C3000F0C7FB58B106
:2083D0000FE00A9847E0252007F03CFCA9680A988847002086F855000420FFF7B9FC3BE002
:2083F000192001F08FF837E00A98884708200BF0F1FA31E00A98884796F8B400B8B10DF0FC
:208410009BFD317800290EBF0921491EC9B201EB81017118D1F802100EF013FE42F2107173
:20843000814292BF00206431081AC0B200E000206968002808BF0620D9D0C6F8980088471B
:208450000446D6F8A010D6F8980006F1A8020CF06DFCA968204688470BB0BDE8F08FC046AD
:20847000700D0020B3170020840C0000B4150020D0290020BB2A00202DE9F843664C0026A5
:2084900005466676687D0628A4BFE8216176A97D0E2903DD03281CBFE8216176032805D12B
:2084B0005E48008840083CBFE820607695F8280008B1E8206076E87D092801DB0A2801DD8F
:2084D000E8206076287E08B1042805DB802801DB862801DBE820607604F118072946384656
:2084F0000CF0DCFD291D112207F12C0007F0C2FA95F8280004F11809002804BF84F8606055
:20851000A87D04D095F8290084F86000688DA4F85600687E84F85800A87EDFF8048184F821
:208530005900E87E822784F85A00287F98F8D76084F85B0098F8E63084F85C70394F84F8B6
:208550005D6005F11D01E763042684F8406098F8E72084F85E3009F1490084F85F200B229E
:208570000EF0BAF9607E00284ED1687800284BD1287EA77E8DF800000FB1EA20607605F10B
:208590001701E720FEF718FC94F8600028B1287E022808BF01208DF8000098F8E7009DF895
:2085B0000010884203D0E8206946FEF705FCA77E1E4C601C007808B10EF074FBB8F8BA003E
:2085D00019490880C7B1032F12D0052F05D0012F03D0022F01D00EF065FB022060700BF0BC
:2085F00093FC4FF6FF70A8F8BA001149088005E00BF08AFC032000E00120607027202870B3
:2086100030460DF039FD01E02A20287028460AF093FBBDE8F883C0460C2C002048160020EC
:20863000A00E0020256D0100CE190020E42C0020521700202DE9F04F154601F00708C1F3A5
:20865000C2074FEAA119044683460C22ADF1240D0021684608F03FFD6248B8F1000F36D0D3
:20867000B8F1010F7ED1228801A9A6780A80E41C8E7014F8011B01F00F018DF80810228878
:208690000DF10A031A80BDF80A30A41C4FF0000C6B75019ECDF818C04168B14207D1017A20
:2086B0009DF80820914202D14189994208D006990C30491C06290691EED96046614601E0CF
:2086D000017840788DF800108DF8010022E014F8013B14F8016B8DF8003000228DF80160BF
:2086F0000C38079210F80C1F994202D14178B14207D00799491C06290791F3D910460146F4
:2087100003E04168027A4089687501918DF80820ADF80A0003A806F097FD9DF800109DF83E
:208730000100B8F1000F11D0B8F1010F1AD1019904989DF808209DF81460484086EA0201F4
:208750000918BDF80A20BDF8160004E09DF80C2051409DF80D205040401803D1EF701FB15B
:20877000022F05D0002039E02188281DA41C0180B9F1010F27D0B9F1020F2CD1BDF80A1043
:20879000281DC91DCA10214607F074F9BDF80A00C11D04EBE104F0B1401E811000EB51714B
:2087B000C910C9B26D182B798710012600EB577121F00701401AC0B2401C06FA00F0FF305B
:2087D0001840287107E0291D20460AF05FFD207804EB8004641CA4EB0B04A0B209B0BDE8D6
:2087F000F08FC046581700202DE9F04FADF1840D209002F06BFC0DF071FD0026012804D139
:208810000DF062FF022808BF01265B490868C0F38150012806D151F80C0C0127010E07FAA1
:2088300001F00643554800780DF006FA544D2C46286038B1FF2204F1400107467F1E01F81E
:20885000012BFBD1209909684FF0000901F0FF02FE2A1DD0DDF880C001F0FF074A460123D7
:20887000FF2F0ED0B84203D903FA07F73E4201D002207EE001F0FF0147EA0909611881F814
:2088900040205CF8041F521C01F0FF07FE2FE7D1092006F023F92098002124220823606062
:2088B00017A80EF081FC4FF0010804F1240017AA8DF8748041460EF073FC236843B3002737
:2088D00094354FF0040BBA4608FA07F0064219D119EA000F04BF07F0FF0141F4C04105D06F
:2088F000E019209B90F8401053F82110254804F0F1FBF8B24FF0FF310DF01AFD2368C5F89E
:2089100000A001E0C5F800B07F1C2D1D9F42DBD301A80021302208230EF03EFC1A4E307856
:208930000025102101AB0990184A009504F108000EF02EFC0DA82822082329460EF024FCB9
:208950000DAA7068124914952B46139004F160000EF016FC0F4951F80D0C474620F4F85058
:2089700040F4005041F80D0C0B4EC1F8FF7F2846376021B0BDE8F08FB43F00508D2D00206A
:2089900034260020007FC7678C0C00005D630100813D01000D300940080009402DE9FE4F4E
:2089B000544E0746301D00688047534C00258346A01C05701FB10CF0A7FE09F00FFF94F87A
:2089D0003800B04610B1E06B00B1804709F080FDDFF8749109F11C0090F900000EF08CF862
:2089F0000CF0A8FE0EF07EF80DF022FF0DF014FFDFF808A107270AF1240656F8040B00B142
:208A100080477F1EF9D13E480560456005614FF470018160C1600AF1040007680FB10BF043
:208A30009DFC38484E4600688AF80E50BA3EC0B112E048460CF0BAF8029002A80BF08EFCD9
:208A500021E048460CF0B2F8019001A80BF086FC14E068460BF082FC07F074FF00280090DD
:208A7000F7D129480078012803D028460146FEF79FF82648264F057007F12409786A002871
:208A9000DFD109F10409B86A0028D2D17D62BD622048A06187F82E501F4BE36187F82F5012
:208AB0001E4A22621E4961621E4B87F830501E4AA362204BE2621D4963601F4A21631C4F8B
:208AD000A260204B65701D4967631D4FE16058462761D8F808106361884706F1BD0152209F
:208AF000FEF76AF996F8D7000AF012FD2846BDE8FE8FC046B4150020141500203C16002056
:208B1000801B0020842D0020A21B00208F2D0020700D0020AFED00001D700100915C01004B
:208B3000317F000005D6000049600100056D01003DBA00007BE90000DDAB0000F930010070
:208B500009F80000192401005A0F00202DE9F04F0546824660480E460178ADF1140D0DF0A4
:208B70002BFE5F4C00283FD0DFF8808108F104000068012914D0287A022835D15749504687
:208B900002220F4620310DF00BF938B903208DF8080007F1160168460EF047FAEA4623E02A
:208BB00095F8089014F809A080470A274FF0640B8E340390207A484506D152462046294665
:208BD0000DF07AFA012804D07F1E04F10C04F1D104E00027F772A07ABB463073D8F8081099
:208BF000039888475F4672E021464FF0000864278B468D6B91F8310086F81E804446D94683
:208C10000AE099F800106D1C2034ADB234E099F83100641C6D1DA4B2A04217DDE8780028E9
:208C3000F5D028790BF082F8514608220DF0B8F80028ECD1E878B07728880004706028794A
:208C500086F80B80F077A87847463073DBF83440002F08BFBB46C5D086F81E8042F2190008
:208C70000DF10A010AF018FD0DF086F983461D480178642745468146A94228DDA07F002895
:208C9000BFD0E07F0BF052F8514608220DF088F80028B6D1E07A022803D0E07A58B1612762
:208CB00010E0616858460EF0CCF9BDF80A200E495143814201D9474604E0A07F6C2740F0D0
:208CD0000800A07730462146202206F0D3FE384605B0BDE8F08FC04615150020340F002075
:208CF000CC100020FC100020808D5B00B41500202DE9F041071CADF1200D00F0C180F86B22
:208D1000002800F0BD80B7F84020002A00F0B880007817F130014FF0000603D097F83810ED
:208D3000052902D0002E00F0AB80584C401E2BD0801E18D0C01E40F0A380012A40F0A080AB
:208D5000514C0725E0788DF81C5000280CBF0121311C3046E17008F021FFE07802228DF8AF
:208D70001D0028460BE0012A40F08A80B4F854000122401CA4F8540004208DF81C00394655
:208D900007AB02F02FFD7BE0684631460C2208F0A2F9B7F840000B284CD1FD6B15F8010BF2
:208DB00084F820002B786878AD1C03EB002328460DF014FE8046281D0DF010FE0546387A1A
:208DD0002077022806D0396804F1140001607A68426001E03888A08203F00100190928BF9D
:208DF00040F00800590928BF40F010006084834218BF0226B8F57A7FADF8020008D3244866
:208E1000404505D3C4F8248040460CF069FA00E00226606AB5F57A7F019007D342F210700C
:208E3000A84203D3A5620DF0F9FD00E00226A06A029000E0012602258DF8016068468DF87D
:208E500000500AF075FC0DF10D009DF801108DF80C500EF00BF8BDF802100EF007F8019956
:208E70000BF053FD02990BF050FD39460D2203AB284602F0B7FCB4F85A00401CA4F85A00ED
:208E900008B0BDE8F081C046D4110020B8130020407E05002DE9F04F0746880FADF1140D43
:208EB000C0F0BC80002009F01BFF62485D4E4FF0000900F11408C8F80090012048F81C6CA0
:208ED0000DF09AF858480DF09BFF584DBC68CB4640F60A0605F1140095F820102A7995F8A5
:208EF0002130A5F816908246C5F818B001F0F0010680012A85F8201003F0F000A4F8029030
:208F100040F0010085F8210001D17B7CC3B1B8680088A6F10801814208D0B0F5C15F05D0B8
:208F3000218B4FF60F400840208304E0218A4FF60F4008402082B86887F8119004F0EEFACD
:208F5000B868694604F02CFC68460DF0BBFE3346D91F4A1C00E03446666836B1308883424F
:208F700003D0814218BF8242F5D1C4F804A0607B00F0F000607305F13C000EF06CF8806880
:208F9000008881421FD082421DD03E8D06B397F8340097F83560C7F82CB000F0F00087F871
:208FB000340006F0F00040F0010087F8350007F12803AB619AF80D00A7F82A9000F0F0009B
:208FD0008AF80D0004E0DA4605F1580080E80006B9680A8A4FF6FF3010400882D8F800005F
:208FF0000028FBD0A87AC8F8009070B901200CF0F1FA01280FD0607B00F0F00040F00100D7
:2090100060730B480DF0FCFE05E00BF053FB0028FBD00BF06DFBB86848F81C0C05B0BDE8BD
:20903000F08FC04601010E044D2D0000A00A0020ED1E0100081004402DE9F84F8846054665
:209050000DF022F901464FF6FF70884210D042F21C0BAB4509D0ABF10100A84205D01A3871
:20907000A84202D0001DA84205D10DF0A5FB10B16820BDE8F88F534C480000EBC100241866
:20909000D4F8027017B9D4F8066016B3D4F80610B94208BF692000F093806078401E12D06F
:2090B000401E09D0801E14D1D8F80000874200F2818081427ED30CE0B8F80000874279D890
:2090D000814277D305E098F80000874272D8814270D33D4F78688047ABF11A0A2B463B4EF8
:2090F0000090A3EB0A03012B25D90A3B012B14D9DB1F3DD1207862780021301807F0EBFFE9
:20911000637840460DF020FD834298BF181C02D940460DF019FD02462BE00CF00BFDBF6882
:20913000B8F80010884243DD207862784146301806F0A0FC23E00CF0FDFC814640464946CE
:2091500009F01EFDBF68A9EB00005FFA80F9B9F1000F2DD0207862784146301806F08AFCEB
:209170001B485146A94218BF401C80F8009006E0627820784146301806F07CFCBF680AF108
:209190001900A84204BF002086F887005846A84213D196F8870096F886104218322A01DC9C
:2091B00008430AD1022086F88600302586F887500098B8476A20BDE8F88F0098B8470020A5
:2091D000BDE8F88FC4000000B41500208C2A00202A2A00202DE9F843634C5C4D5C4EDFF832
:2091F0007881604F94F8E4100846401E0B2864D8DFE800F07E2C43062343062343067967BA
:20921000042907D001220A2945F8212C14BF0220032004E0202045F8210C0120024684F8CF
:20923000E200002045F8390C0827C5F8FF7FC5F8F37F45F8392CBDE8F883052914BF092015
:209250000620002784F8E400376078E094F8E170383D0120002FC5F81B0004BF06200021DE
:2092700002D00021F160032084F8E400032045F8010C31603068800861D294F8E4103548C9
:20929000012703290ED00068456800216022052300914046A84794F8E400062814BF0A200B
:2092B0000720CFE700684568002160220523022000904046A8470420C4E70DF05DFFBDE8ED
:2092D000F8832648264F0026012506600E203D6005F01AF902200BF091FD84F8E45084F8C4
:2092F000E360BDE8F883002038600C25786024E04FF08059D9F8A0010168202088472C3DCB
:209310000F2045F8010C41F61D56C5F80360D9F8A401466800214FF4C07207230225404669
:209330000095B047D9F8A401C66800214FF4C07207234046B0470120386084F8E45004F152
:2093500078000DF049FFBDE8F883C04639400C4038600C40A401001000A00C402C500C4008
:2093700004800C4034600C40B80F00202DE9F04304466668A7680D46ADF1340D0DF038FF70
:209390003178012903D10DF02FFF0020A9E04FF0010886F800800DF027FF28787070687879
:2093B000B07068687060A868B060E868F06028693061287D3075687D7075A87DB075A8698C
:2093D000B061287F3077687F7077A87FB0774FF00009C6F82090C6F830904D46756275638C
:2093F000B562B56386F82C50102386F83C3086F82D5086F83D50786805F070FB204605F076
:20941000E1F8204606F0B6FC70B937480068C16838688847786805F077F80DF0E9FE3570E0
:209430000DF0E2FE2C465BE001A82946302208230DF0B2FE0694387BCDF800902B4A0990A0
:20945000B96801AB06F180000DF0A2FE01A82946282208230DF098FE05942549386901AAA8
:209470002B46079006F19C000DF08AFE01A82946242208230DF098FE8DF81C80B07838B966
:2094900006F1D000294601AA0DF08AFE19483061707838B906F1EC00294601AA0DF080FE13
:2094B0001548F06001A82946242208230DF060FE0695ADF814501149079406F584700A2257
:2094D00001AB0DF051FEB969FA6906F140000DF09CFB0B4A06F16C00042123460CF062FA96
:2094F00020460DB0BDE8F083D0010010BDC10000A54A0100B36F0100AB6F0100A9010100E9
:20951000556D01002DE9F8435E4D804695F83800002798B12A6F8AB1D5F8900070B142F2FB
:209530001A0069469047D5F89000804730B19DF8000018B1B8F1E10F08BF0127524A02F101
:20955000E70000780BF02CFF407B02280CBF05260126514C2068002800F09280B8F1000F6D
:20957000914675D0B8F11B0F02D1017D05296FD1B8F1E90F2CD05FBBB8F1E10F16D10DF0F9
:2095900057FA90B12068C18AC9080FD299F8C810817699F8B6104A1C89F8B6204068817097
:2095B0003046FEF7D5FBBDE8F8832068B8F11C0F1DD1216A002950D0884734490020097835
:2095D000206001295CD00146FDF7F2FABDE8F883F1200DF00AF82768B87E50B90DF028FA61
:2095F00020B12068C18AC90801D2CFE7206847462FE07868398907F02DFA78680088000908
:2096100005D395F8380010B10BF0EAF82768F88AC00811D3387E00F07F003876387D03288F
:2096300003D1787E40F004007876F0200CF0DDFFE168206888470FE015490126B87E0E707E
:20965000401EB876F0200CF0D0FF12480078A8E70027477008F074FE2068C08A000A0AD331
:2096700095F8380018B999F8D70009F051FF99F9D6000DF041FA0020206010200DF04AFBE1
:20969000BDE8F88314150020A00E0020A21B00208C2D0020261A0020700D00202DE9FE4379
:2096B000604C614D0E46B00959D35D4800F1280980464DE00178D0290EDBD02909D1817826
:2096D0003970C17879700179B97085687D60C168B9600DF0ACFA47E004F10805286009F0B3
:2096F0002BFB28460AF03AFE3EE0884798F83010491E88F83010A9688847009801788DF83A
:209710000410A0604778CFB1DC2F0DD0DD2F0BD0E42F09D0F32F07D0DE2F05D0DF2F03D06F
:20973000E82F18BFDB2F0BD103F064FF9DF80400162805D168460AF011FE01E009F0FCFABB
:209750009DF80400162803D004F108000AF006FE48460BF02BFA002869680090C5D1F00B8C
:20977000A846C00305D0314F07F0ECF800280090A0D1700905D32E208DF8040001A809F005
:20979000DBFA700805D325208DF8040001A809F0D3FAB00805D326208DF8040001A809F056
:2097B000CBFAF00805D327208DF8040001A809F0C3FA300905D329208DF8040001A809F050
:2097D000BBFAF00908D300208DF805002D278DF8047001A809F0B0FA300A08D300208DF8F3
:2097F000050030278DF8047001A809F0A5FA6068D8F8041080B18847616800270091D8F8C6
:20981000081067608847009804F10806306009F093FA30460AF0A2FD0020BDE8FE83C0467E
:20983000700D00203C160020B4150020A41B00202DE9FE4F07461046002F00910CBF4FF071
:20985000E80B4FF0000B002900F0AB80BBF1000F40F0A98060B17868401E7860F8210170B2
:209870007868401E7860002606703889801C3881009C4FF000094FF0020ADFF83081CDF894
:209890000490083C14F8080F00F00F010F2900F08580012820D004287AD1454D95F83800A9
:2098B000002875D0296D60688847061C26D03889B7F84C103018801C81421FDB78686D6DBF
:2098D0006168019B3A46801BA847B8B178683D89801B786076195AE00098019E042309EB6C
:2098F0000001C91C11F8010FFF2841D021283DD13889B7F84C200B30824202DA1A20BDE834
:20991000FE8F7868B8F8D020401E7860121202707868401E786098F8D02002707868401E18
:209930007860019D057098F8D2007A68107098F8CE2078681201401E786042F00F0202700C
:2099500098F8C0C098F8A1207868401E786042EA0C1202707868401E786021250570786813
:20997000F61DB6B2401E7860052505705B1EB9D17868C6F30121401E786041F08801017068
:209990007868401E7860067038893618B61C3E81BAF1010A09F108097FF474AF7868B86537
:2099B00001E04FF0E80B5846BDE8FE8FA00E0020141500202DE9F04F5D4C054600208A4664
:2099D000ADF12C0D80461746B4F952100A93DDF850B084F88901B4F950008BF80080401A9C
:2099F00040F6F87101400829A8BF012080F29280B4F95000401CC0F30B030CF02FF90646B0
:209A1000D4F87C01B384854207D194F88801410824BF00F0FE0084F888010A98006800B920
:209A300040463062387B00F00F00022814BF4046B868BAF1000FF06175D00AF19C000DF0C5
:209A50001EFB002865D128460BF008F8051C1AD1E36BC3B109F0A0FA236C08902BB1216C25
:209A7000E26B304605F0D8FD38B9236C5BB9E26B3046694605F0D0FD28B1012384F889314E
:209A9000E06B3060E66394F88991B9F1000F4AD10DB9E56B95B12A683046294605F0BCFD97
:209AB00018B92D68002DF6D108E00223286884F889312246306092F889912E60B9F1000F86
:209AD00031D10A980179504604F042F90146012926D094F88901002825D1012923D0E16B8F
:209AF00009B10868D0B9387B00F00F02022A1AD1C01118D141B9206CA8B1216C30464246B4
:209B100005F08AFD28B10EE03046424605F084FD48B902208BF80000464604E00968E0E730
:209B3000042084F8890130460BB0BDE8F08FC046A00A00202DE9F04F504E7068ADF11C0D34
:209B500080474F4A934611784E4D04919BF80020B168012A0BD001248BF8004088472878DA
:209B7000012805D020460021FDF722F800E08847464C454FDFF81891E06807F1B001814239
:209B900006D1494691F90000002818BF002761D170688047404B0590002003F13801A7F8C2
:209BB000B2000F78002F07BF4FF48601021C39492022804639489A460378CDF808809B0928
:209BD00004D20078000938BF012000D302208DF80C008DE8060036493148324B006802AA7C
:209BF000FBF734FFB7680028A08030D4494691F900009AF801302C4A401C08702C49002BFF
:209C100092F90000E16000F1010010700CBF40468020B4F84410254B4FF67F720A401043C2
:209C30000143A4F84410B3F8BA00B3F8BE10A4F852000822A4F8501003F1D80104F14703E2
:209C500018460CF049FE0598B847012702E00598B847474670688047B16817B9049A8BF8DB
:209C7000002088472878012803D000200146FCF79FFF384607B0BDE8F08FC046B415002009
:209C9000961B0020A21B0020D8120020001700209F1B002000004F8C14150020912D0020E9
:209CB000D0190020F11400009E1B0020A00E0020881300202DE9F04F8A4609AF4FF0805137
:209CD000ADF11C0D90463D69059001F5D8700490D1F8B001D7F808B0416906932720884770
:209CF000524C4FF00309143CC4F884970126C4F87C67C4F880970220C4F8FC06F868C4F8AF
:209D1000080430460DF070F9D4F808040008F8D2D4F88C07800F28BFB14655D2681E4146A1
:209D30000C238DF800000DF1010011F8012B5B1E00F8012BF9D1022D19BF0020011C98F8F0
:209D50000C1000208DF80D108DF80E008DF80F000099C4F83C15019BC4F84035029AC4F823
:209D70004425039BC4F848353968BAF1020F4FEAC542A1EB0A08A2F5002106D34FEA4A52F2
:209D9000A2F580026FF315021143264A0A43C4F84C258246C4F85085BBF1000FC4F854A51A
:209DB000214DC4F858B511D02E6078682060C4F808B030460DF018F9D4F88C078008F8D3E3
:209DD000D4F88C07000801D3CA4627E0C4F88497D4F88C0710F0030FFAD1D4F8800720F0AB
:209DF0000200C4F880073F7D47B1049F3868016A272088473868016927208847C4F87C67D7
:209E10000598C4F8806748B12E6006982060C4F80880C5F800642062C4F82880504607B0B5
:209E3000BDE8F08FC801042000004842184002402DE9F04F894609AF4FF08051ADF1240D22
:209E50009246059038683D69079001F5D8700490D1F8B001D7F808B041690693272088477C
:209E7000504C4FF00308143CC4F884870126C4F87C67C4F880870220C4F8FC06F868C4F850
:209E9000080430460DF0B0F8D4F808040008F8D2D4F88C07800F28BFB04653D2681E5146D4
:209EB0000C238DF800000DF1010011F8012B5B1E00F8012BF9D1022D19BF0020011C9AF86D
:209ED0000C1000208DF80D10019B8DF80E0000998DF80F00029AC4F83C15B9F1020FC4F818
:209EF0004035039BC4F844254FEAC542C4F84835A2F5002106D34FEA4952A2F580026FF3C1
:209F100015021143254A079D0A43C4F84C258146C4F85055BBF1000FC4F85495204DC4F888
:209F300058B511D02E6078682060C4F808B030460DF05AF8D4F88C078008F8D3D4F88C07EB
:209F5000000801D3C14624E0C4F88487D4F88C0710F0030FFAD1D4F8800720F00200C4F8E6
:209F700080073F7D47B1049F3868016A2720884738680169272088470598C4F8806740B181
:209F90002E6006982060C5F800642062079FA760A762484609B0BDE8F08FC046CC0104204A
:209FB00000004842184002402DE9FE4F524D286808B90CF077FE554C04F13800DFF83C9137
:209FD000DFF840A1DFF8408107789FB94D46686880474B490F7847B95246A96817782FB9E5
:209FF00083234246137088476DE0A96802234246137075E0D4F8981009B104208847676DF9
:20A010002A685FB1D06D20B102210023B8472A68676D106E10B108210023B8473C4E306A27
:20A030003C4F016CF86888474D46834668688047029033480578002D48D1504600780028F0
:20A0500044D1D4F8841000208847F42001A909F0E5FC9DF90400304D58451ADCAB79C3B9AA
:20A07000D9F8081002988847A878042801D00CF019FE04214046AF790170D4F88410781C16
:20A09000A87109B1032088470320688100F0FAFA27E083214046346A0170636CF8686A46DC
:20A0B00000219847B6F90600BDF90010884214BF0020012009F08AFDD9F808100298884765
:20A0D0000835287838700CF057F80AE0022140460170D9F8081002988847D4F884100420C6
:20A0F00088470E480078012803D000200146FCF75FFDBDE8FE8FC046700D0020B415002043
:20A11000902D0020922D0020942D00201415002000170020C4190020241A0020A21B0020DA
:20A130002DE9F8434E4E84460120002430704D484F4D04704C48DFF83481047005F14E00F6
:20A150000088B14614EA03074FF0020606EA020608BF002E13D120464FF0E04710401F40D5
:20A1700008BF002803D11D2006F030FC54E0454695F90000401E28700CF096FB4CE0424629
:20A1900092F900303C4E5B1E137043F20842824207D06F8E931C834203D0BA4218BFBB4240
:20A1B00017D1304608300068826C60469047008843F6030181420BD0204601F071FF98F96B
:20A1D000000000283FD098F90000002838DD42E06F8EB5F86A1043F60400884205D0B8424E
:20A1F00003D0B5F84E20904203D12248007803281AD1B1F5505F05D0080B0BD31D2006F075
:20A21000E5FB07E01D480168304601F5C071016004F0BCF80CF024FB98F9000098B198F96D
:20A23000000000280CDD16E0022811D0204601F037FF98F9000030B198F9000000280ADC5E
:20A250000CF030FD07E020460146FCF7B1FC02E0204606F0BBFB89F80040BDE8F883C046B6
:20A27000A21B0020981B0020971B00209E1B0020D8120020261A0020181700200C0100218C
:20A290002DE9F84F994692468B4606460CF0B0FF4E4C0090B4F95210B4F950000AAF401A89
:20A2B00040F6F871014008297CDAB4F95000401C6FF31F30A4F85000B4F950800BF0CEFCEF
:20A2D000054606F178000BF047FFC5F808B085F826A0C5F80490A5F824803D48EE6097E8D7
:20A2F0000C00202100271940104005F1100383E8030004F13C0085F827700368002B43D1CB
:20A3100029460AF095FD002844D0A6F8C08095F8270040F0800085F8270086F8C270E07907
:20A3300020B1207810B1E7710120207200980CF05BFF206C002845D12078F0B960790128DD
:20A3500040D00CF055FF0646A07988B9A86807F061FF40B930460CF047FF04F1EC000421C9
:20A370000CF00EFB2EE004F1C8000CF035FF02E0184901200870304622E001200CF010F854
:20A3900019200CF0D7FC1DE004F13C0029460AF04FFD50B9B4F9500000F6FF706FF31F30A6
:20A3B000A4F850006FF0010809E0A6F8C08095F8270040F0800085F8270086F8C270009822
:20A3D0000CF012FF4046BDE8F88FC046A00A0020FDEFFF9F8B2D00202DE9F0434D4CDFF8C3
:20A3F000388194F83F600027ADF1140D002E57D198F89660002E53D0C768007A454600F032
:20A410000701C0F3021900E0BF1C0E46701EC1B24EB17A783878B5F8BE6000EB0220B042DB
:20A43000F2D1022710E005F19406443600E008374846411E5FFA81F9A0B3304639460CF003
:20A45000B9F80028F3D0032794F83F0040F0040084F83F0002A80BF01DFB01200BF00CFE89
:20A4700004F13401872000F063F804F13C01852000F05EF804F13D01862000F059F804F184
:20A490003E01882000F054F80120009004F134060196B5F8BA30394602AA0520FDF78AF8B5
:20A4B000002F33D198F8A1100F292FD0404690F8C0208A422AD090F8BD0038BB174800781E
:20A4D00020BB17480078012803D001200021FCF76FFB144C606880472146134C94F83B2083
:20A4F000022A11D194F83820FF2A0DD00F4A176857B9576A47B98968884704F1200009F0DD
:20A510002FF806F02BFB01E08968884705B0BDE8F083C046942B0020A00E00204A16002047
:20A53000A21B0020B41500201C190020700D00202DE9F0410C4601467138022840F2978057
:20A55000133825D04D4F4C387BD0401E62D0401E4AD0401E38D04A4D401E2AD0401E1AD09B
:20A5700008460CF05BFB06460B2E11D0414D6868804741498046B000425CBF184018427819
:20A59000394620460CF0A8F9A968404688470DE0F420BDE8F0812278022A68DA2946601CB9
:20A5B000483101EB820104220CF096F90020BDE8F0812278032A5ADAD3002946201D03EB54
:20A5D00002131822C918EFE72678022E4FDA2C25601C05FB0671102239310CF07DF905FB1C
:20A5F0000670C06C6061E1E7207802283FDA2C2101FB0070667890F83800B04237DD23784D
:20A610006278394602EB430201EB42010222A231A01CC9E72078022829DA2C2101FB00708F
:20A63000667890F83000B04221DD20786278394600EB4000121802EB420289180322903186
:20A65000E6E72078022812DA2C2101FB0070667890F82800B0420ADD6278207839468018C6
:20A67000420002EBC00289180A227C31D0E7E820BDE8F081B4150020F8040000442700201A
:20A69000F02700202DE9FC414948484C494F4A490278A37865893878042B71D101F13C06F8
:20A6B000337803F0F003337000268E630DB901256581884641490832554300FB05F291F8C8
:20A6D00038500092002D50D00D46AA6F002A4CD0EB6F002B49D004F1080168469047844666
:20A6F0003B4B2179DFF8E0E060791A68BCF1650F31D0BCF1000F28D1107D052811D130484D
:20A71000017871B9186890F82C00042809D119686D6D906D096B3346A847002808BF1A20EF
:20A7300016D02C4D6868804726490E68002E08BFA96807D0A96804F10C02964213D03668E4
:20A75000002EFAD1884738780FE0704606706046FEF7D8FE22E082F8690082F86A10704656
:20A77000E96F06701C20884718E01849009E04F10C076161B6FBF0F138460BF0D5FE0DE064
:20A7900091F83C30083280005543884603F0F0036843886343F0030381F83C3098F87400F6
:20A7B00000F0F00088F87400BDE8FC81241A0020C5190020241B0020D81200201415002085
:20A7D0005D0F0020801B0020942D0020B99F0000700D0020B4150020F8B5071C00F0A18082
:20A7F000B86840F6030120264A1C02E04068761EF6B260B15EB10388994218BF9A42F5D17E
:20A81000F9681CC828311CC149C881E849007868BA690026BE6168B3F968486800780228D4
:20A8300018BF42F0020297F82700002300F00700401E09D0401E04D0801E08D14FF0805339
:20A8500004E04FF0804301E04FF00053324697F82700000908D397F8270010F0070F03D0DE
:20A870004FF0807032430343B7F92440084621467C68A0470CF0BCFC2A4C0546B4F95200D6
:20A89000401C6FF31F30A4F8520004F14C00016881F827600CF097F828460CF0A5FCB4F9C0
:20A8B0005000B4F9521088423BD1F86890F8C20000280CBF0520072004F01EFC04F5AA7445
:20A8D0002568F868854208BF656890F8C240002C0CBF0468341C80F8C2604DB195F8C230CC
:20A8F00023B92868A04228BF041C01E085F8C260A4B10D480068B4F1FF3F12D0B4FBF0F10C
:20A9100001298CBFB4FBF0F10121F86878300CF027FCF86878300CF05FFCF8BD012009F0AB
:20A9300049FAF8BDA00A0020B00C00002DE9FE4F514C814604F13C0A50460CF08CFB904698
:20A950008B46074608F0010000900CF051FC0325BBF1FF3F019015D1266C2EB1206CC06849
:20A97000814508BF206C0BD00CF042FCDAF8006074E0F168894570D10CF036FC301C71D0F0
:20A99000B0F924B058460AF0A9FE00286AD0216C814248D0B84217D104F1C8000BF0DCFBB0
:20A9B000E06B0068E06397F82700394640F0040087F827000AF110000AF03AFA5FEA980068
:20A9D00022D3E76B01221BE017B9832D20D01CE03968884225D104F1C8000BF0BDFB396824
:20A9F0000868386091F8270040F0040081F827000AF110000AF01CFA5FEA980004D30022C6
:20AA10004846394607F036FA832501980CF0ECFB6079012829D004F1EC0002210BF0B0FF25
:20AA300023E03F68D0E7009F90F82720012505FA07F13E1C41EA020180F8271014BF0C48BC
:20AA50000C480AF09BFF5FEA980004D3E16B48462A4607F00FFA832504E03668002E88D14B
:20AA70000CF0C2FB01980CF0BFFB2846BDE8FE8F0100020401000104A00A00202DE9FF41F1
:20AA90000646080BC0F092804A49C8680025012788460D70C3694F722BB1016AC90802D350
:20AAB00004212A469847444908F170002A460CF0BFFA42480CF0A4F9D8F80C004168414CC2
:20AAD000886808B9C86820B1A4F11C00C5613C490160384608F004F925603B4844F81C0C18
:20AAF000B1684D80B068028840F60200904208D0B2F5C15F05D00B8B4FF60F421A400A832D
:20AB100004E00B8A4FF60F421A400A8200F1080C7774ACF10702531C00E039464F6837B12D
:20AB30003888844503D0824218BF8342F5D12F464F60487B00F0F00040F00100487308F1D7
:20AB50003C000CF088FA8068008882421BD0834219D0308DC8B196F83400758596F8353079
:20AB7000F76200F0F00086F8340003F0F00040F0010086F8350006F128024A60487B00F095
:20AB9000F000487301E0C8F86050B068694602F007FE68460CF096F8B06802F0BFFC206866
:20ABB0000028FCD02560B06844F81C0C0090BDE8FF81C046A00A0020756401004D2D0000B7
:20ABD000510007061C10044001010E042DE9F04106467478ADF1180D002C40F0898049484B
:20ABF000B6F896100088884218BFE82406F18C0101A80D460BF0ECFC01A80AF037FF424BF3
:20AC100040B996F8990040B1A3F13800007820B9E8246DE0002086F89900002C68D196F873
:20AC3000990000280CBF01200520042737752946F0820DF10E000BF0CBFC706896F898406E
:20AC5000401E7060411E7160B6F896800470327D71680024481C3062501E08703089346574
:20AC70001A78B465801C3081A2B386F86B70296806F16C0001606B6843602A8902810BF022
:20AC90009BFD06F16C0228BB06F18C0110460CF0CCF91E4D286810F47F0F0CD086F82C70A6
:20ACB000286806F12C01012200F47F0030633046FEF7BEFD286810F0FF0F0BD02A2086F840
:20ACD0003C00286806F13C0100F0FF003064304603F070F90094304603210DF10E0243464A
:20ACF000F8F742FC041C02D1304603F08DFA2CB174701A203070304608F01EF806B0BDE8BA
:20AD1000F081C0465A0F00204C150020B40800002DE9F04706464FF00108ADF1600D0922CF
:20AD3000B07D8DF84C8006F117018DF84D000DF14E000BF0D1FD464D68688047814616A9DF
:20AD50008120FFF7F5FB707D002854D09DF85800022817DA042000238DF80300347D8DF816
:20AD700002809DF858708DF8013069468DF80040781C8DF85800D220FCF700FF812016A905
:20AD9000FCF7FCFE00274FF0FF0A3C46307D8DF8217008A980F001008DF82000D120FFF754
:20ADB000C7FBC0B99DF82200FF2814D08DF800006946D420FFF7BCFB20B1A9684846884772
:20ADD000192042E0307D69460DEB80000461D420FCF7D4FE01E08DF822A08DF82440307D58
:20ADF0008DF8234008A98DF82000D120FCF7C6FE7F1C032FCADB307D00279DF84D208DF890
:20AE100040000DF14E018DF841700DF142000BF063FD8DF84B80D02010A9FCF7AFFE071C08
:20AE30000FD1307D314610228DF828000DF129000BF052FD30690AA90F90D320FCF79EFE41
:20AE50000746A96848468847F8B218B0BDE8F087B41500202DE9F04FFF25ADF1140D8DF8F3
:20AE700000504FF6FF79ADF80290ADF804900AF013F8DFF81CB104900BF10200008800275B
:20AE9000001F84B2082C64DB4E46B046C246201F02A9082280B20AF063F9BDF80800814529
:20AEB00008D1BDF80A10894506D1BDF80C20924502D107E0BDF80A1051EA000317D1BDF819
:20AED0000C30A3B9BDF80E1008466FF30E0060B908460830844206DA0BF0E4FE04980BF080
:20AEF000B3FA00204FE008462EE0241F2EE0C20BD30327D1BDF80C20854203D18E4208BFEB
:20AF100090451FD0C5B28DF800500E46ADF802609046ADF804809DE80600384607F0ACF912
:20AF300080B9BDF80E20A01A07F18851001F083280B292B20AF014F9BDF80E003F1808372B
:20AF5000BFB201E0BDF80E00241A083CA4B2082C9DDA09F0A3F93FB10C484FF088513A46D8
:20AF70000BF0D2FF0BF00EFE04980BF06DFA5A46507800281CBF0020011C03D1C7F58054E4
:20AF9000391DA0B2518005B0BDE8F08F04E00100281C00202DE9F8430020444C8DF8000080
:20AFB0000BF0D5FF2279484E424DDFF81091012191404FF6FF725218024096F8380062817C
:20AFD00020B3326F12B342F21A0069469047384867790378A3B19FB99DF8003083B1D6F806
:20AFF000940068B180474946491C2A78097830B1678908314A43B0FBF2F0C01960816779F8
:20B010009DF80010608907FB01006081A078002847D1294F386AC06B80474E468046648903
:20B03000297870783B6A08304443D86B8F0080476968234D2A787578224E3C23401AB0FBD6
:20B05000F7F103FA02F0B1FBF0F205F108034243891AB1FBF3F25A43891A05F10803691AFD
:20B07000641896F8581096F83C5098B2083401F0F00107FB048341F0020107FB0032736503
:20B0900096F8744086F8581005F0F000B26340F0020086F83C0004F0F00086F87400BDE817
:20B0B000F883FFF7EFFABDE8F883C046241A00208C2D0020241B002000170020C419002036
:20B0D000600F0020D8120020141500202DE9F0434A4D95F8E700ADF12C0D00287AD13F4F52
:20B0F000387B01240021242285F8E7407E6885F8E6000823C5F8106101A80CF039F80026BF
:20B1100005F10C00069601ABADF814603449079632460CF029F8334905F1300001AB324647
:20B130000CF022F8304905F1540001AB32460CF01BF8B96820468847DFF8BC802B4808F11E
:20B1500004037A7B00781868C0F3815922B1B9F1030F04D185F8E140B9F1030F1ED0B9F108
:20B17000020F1BD0B9F1010F2DD14FF08059D9F8A4011F4F456831464FF040521C230320B8
:20B1900000903846A847D9F8A40131464FF400720923456800943846A84714E002200AF016
:20B1B0006FF8B9F1030F0CBF4FF47A7142F21071104800685435B1FBF0F128460BF0D0FFA0
:20B1D00028460CF009F840460068C00802D230460AF056F80BB00020BDE8F083240C000089
:20B1F000C7C20000750C0100BD0701008D2D002000A00C40B00C0000B03F0050B80F0020C7
:20B210002DE9F84F064630798028D4BF0020E82071790027092901DB0A2900DDE820B17908
:20B2300009B1042903DB802975DB862973DA002871D1DFF8F88098F8A1000F286BD0B8F838
:20B25000BA104FF6FF70884265D0B8F8B410884261D0F079314C01280BD040B1FF285AD1C5
:20B2700094F83B00002856D101252F4602E0012500E00225DFF8A8A00AF12000834608F003
:20B290006FF90AF1100008F06BF904F1200008F067F9DFF89C9009F1040000688047214BC6
:20B2B00084F83B500246FF21002060631D6884F83810002D0CBF0121011C012F84F83D10B3
:20B2D000554684F83C7008BF032085F840004846816810468847B11DE820FBF76DFD711D98
:20B2F000E720FBF769FD311DE120FBF765FD94F83D00012802D120200BF004FD0A4898F859
:20B31000A1104FF47077A86207FA01F000F2636158460BF009F9BDE8F88FC0461C1900206E
:20B33000782C0020700D002025200100A00E0020B41500202DE9F84F05464448DFF81091F3
:20B3500083462E18093699F8380034788846B0B1D9F8501099B10BEB8507786B00F0FF001C
:20B3700088478246D9F85010786B00F47F008847504480B218B131784018001DC4B2354830
:20B39000007801280CD198F808704FB1324898F80930C1190E79C05C0019401DC4B200E08B
:20B3B00000260D2D09D106EB0408B8F1F80FD8BF2A4F1CDD0BF076FC05E030198046801C90
:20B3D0000AF0DCFC074697B902200AF0D7FC011C0AD00BEB050090F825001A270870204E39
:20B3F0004F70307807F05AFA0020BDE8F88F08F10202384600210BF03CFE07F10C00002149
:20B4100074220BF036FE07F13C00FF2110220BF030FE07F12C000F2110220BF02AFEE01906
:20B430007860022D3E810BDB0B2D09DA7868401E78606D1E05703889641EE4B2401C388131
:20B45000A7F84C403846BDE8F88FC04670080000141500206C0F0020440C0000A40D002084
:20B470003C16002070B5ADF1380DFFF72FFE3E4908682822082340F00200086001A800214F
:20B490000BF082FE394D3A4E3A49A878002301AA079006F1EC000BF073FE0021302208231E
:20B4B00001A80BF079FE287800241921ADF81C40314A099001AB009406F170000BF068FE46
:20B4D0002822082301A821460BF05EFEE8782B4901AA2346079006F590700BF051FE01A813
:20B4F0002146302208230BF057FE01206A78ADF81C001A2101AB099206F18C00204A009441
:20B510000BF046FE1F49224606F1C80013460BF02BFE1D480BF074FC1C4A2346042106F115
:20B5300028000AF03FFA25464FF6FF70A6F8C400052386F8683006F1580181E830004FF4B5
:20B55000FA70C6F85C01C6F860012B4686F8C73033717371B371F37133727372B372F3722D
:20B570000B4A13700EB070BD00200940A20C0000A00A0020496901001DFE000021FB00002D
:20B590005130010051530100CDB60000F53601008A2D00202DE9FE4F0AF0EEFC434C04F123
:20B5B0000C020290116820614FF40050491C1160694608F071F8DFF8FCA0DFF8FC9094F806
:20B5D000330000285FD0A66B94F8310000254FF0FF0BA0462F4654E0B07F800821D3F07FEC
:20B5F00008F0A4FB0146082268460AF0D9FBC0B1716802980BF025FD2D49814211D8F07F25
:20B61000B77709F095FD86F81FB0DAF80000804794F8323013B15B1E84F83230D9F8081089
:20B63000884798F830006D1C2036ADB236E0F078800822D3307908F079FB014608226846FE
:20B650000AF0AEFBC8B13088010402980BF0F9FC1749814211D83079F77009F069FD86F87E
:20B6700004B0DAF80000804794F8333013B15B1E84F83330D9F80810884798F831006D1C60
:20B69000ADB2A842D3DC94F8320048B1A046666B98F8300000254FF0FF0B2F46A8429BDC30
:20B6B00004F1140007F04EFCBDE8FE8FCC10002000A493D6B8150020B4150020F8B5424CE4
:20B6D0000D46A8085DD2E8087CD301260420E67209F0D6FD0BF0B6F904F1580282E8030014
:20B6F00004F13C000BF0B7FC0746E06877B1FD6850B1854208D0EB6933B1286AC00803D331
:20B7100028460421002298472846E06041682F4A09781160416812680978914207D0876985
:20B730002FB16FF0FF0100224FF00073B847022009F0A6FD112003F0D1F96671E168087C97
:20B7500010B12079012803D00E2003F0C7F9E16849681F488F680FB9CF681FB10021C16138
:20B770001C4F07601C4A40F2FF711160002787611A4941611A480BF043FB19200BF0ECFCA3
:20B79000F8BD04F14C0630460BF065FCFFF724F830460BF060FC25F0020504F13C0158B98D
:20B7B000E80803D208460BF056FC58B104F1C8000AF0D2FC042101E045F0020104F1EC006C
:20B7D0000BF0DEF8F8BDC046A00A0020D02108400010044051000706000004600A0000406A
:20B7F000A58E00002DE9F04F0C4692468046994600213822ADF13C0D684605F06CFC2068ED
:20B810006D4628606068686020892881207A032804D0022003268DF80C0002E003268DF8F6
:20B830000C60374C207818B104F12C000BF01AFAA08DADF80A0060781F28B4BF411C00218C
:20B850000027B8F1050F617040F080000BD0B8F1040F05D0B8F1020F08BF40F0600004E012
:20B8700040F0200001E040F040008DF80D00ADF828A04FF0010BCDF8249022498DF80EB0A6
:20B890000A680BA80260496841608DF8356005238DF83660B8F1050F8DF8343012D0B4F82E
:20B8B0005600B8F1040F08D0B8F1020F0FD1B4F85C00401CA4F85C0009E0401C80B2A4F885
:20B8D000560004E0B4F85000401CA4F850000E4918206A4613F07CFCC0B258B1B8F1050FE8
:20B8F00009D1606A09F0FCFCB4F85000401CA4F8500000E05F4638460FB0BDE8F08FC04673
:20B91000B8130020F5070000A95C00002DE9F041414C0746206800287BD0DFF80081002F88
:20B9300018BFE92F17D10AF0F7FA4546297801EB81016918C1F8020095F8B560287800EB32
:20B95000800029184E702878401C2870C0B20A28A4BF00202870324D68681C2F32D0314EEA
:20B970004FB1F079032806D1E12F04D0002088F8B200072000E0052008F02CF82468F079D9
:20B9900003280ED06CB1002084F86900E18A2648C90938BF2938007884F86A003846FDF799
:20B9B000B1FD98F85700012833D168688047044606F028F9A96820468847002088F8570080
:20B9D000BDE8F08180470646A96894F82F0002281ADA216804F124000AF07EFB94F82F0074
:20B9F000A968401C84F82F00304688472068007D252819BF012088F85600012088F85500C3
:20BA100000202060BDE8F08130468847F120FDF779FDBDE8F081C046700D0020D0290020CE
:20BA3000B4150020AC170020820F00204549B0B5044601F13800007800287FD094F88B000C
:20BA5000002871D13520207504F18D01112204F16C000AF041FF04F13C00FF2110220BF0B3
:20BA700008FB04F12C000F2110220BF002FB94F88C0004F13C0500283ED0401E29D0401EFF
:20BA900014D0401E58D12A20287002272764042305F8103C4FF410222263032184F86B1010
:20BAB000204606F079FD071C3BD137E02A200A272870042327644FF44C1205F8103C02218C
:20BAD0002263204684F86B1006F066FD071C28D124E02A2002272870042327644FF41022C9
:20BAF00005F8103C01212263204684F86B1006F053FD071C15D111E02A2002272870042377
:20BB100027644FF4502205F8103C00212263204684F86B1006F040FD071C02D1204602F008
:20BB300073FB381C0BD1B0BD01280AD1886C8047002808BF002002D0192000E018200AF0FF
:20BB5000EFFFB0BD141500202DE9FC410746BE6833687D68986B20F4FA609863AC6B44B173
:20BB70003168886B40F4FA6088634FF0FF30BDE8FC81AA6329630024EC776C630CE09DF8B0
:20BB90000000296B08706B6B286BAA6B401C2863581C6863501EA863A86B90B93168886B84
:20BBB00040F4FA6088636A6B6878296B0128A1EB0201296303D1EB68384698476A6B1446BC
:20BBD00046E005F14000694608F028FC0028D6D50BF00EFB204F8046387820B9022009F07E
:20BBF0004FFB0120387040460BF0FEFA1B49086840F4007008603168886B40F4FA608863C4
:20BC10006878D8B9696805F1EC000BF0D1FA90B9AC630BF0EDFA0646387818B1022009F010
:20BC3000EDF83C7030460BF0DFFA1027696B286BEF77401A2863686BBDE8FC8195F82D0081
:20BC500030B1686B20B1AC6305F19C000BF080FA2046BDE8FC81C046882D00203010004056
:20BC70002DE9F04F09AF9A4616460D46ADF1440D3C89D7F80480109000203F888DF83C00C9
:20BC9000BC4201DAC24501D30BF00CF8002E69D0364810F80690042EA4EB09044FF0000051
:20BCB000A4B2B8BF01205FEA000B0EBF3F1BA04400242F49082307A8A7EB0907BFB211F895
:20BCD00001295B1E00F8012BF9D1290E00F8011B2B0C00F8013B2A0A00F8012B9DF83C10D4
:20BCF00000F8015B234D06702868109A4369686898470646B6F1FF3F24D001208DF8010099
:20BD10009DF83C608DF802600BAA04928DF800B08DF80390CDF80880CDF80CA002218DF8FD
:20BD30001410ADF8164007ABADF818702E686868326A019369469047064628688269686842
:20BD50000FA99047002E18BFE4200CD1B9F1000F08D0444448460BA911F8012B401E04F874
:20BD7000012BF9D1002011B0BDE8F08F480C00007F0F0020702D002070B5424C0646683C56
:20BD9000607800287DD0B4F95200B4F95010884213D0304608F062FE38B9216C21B1216CE2
:20BDB000C9688E4208BF206C38B1B0F9241002224FF0E043304604F059FB0BF019FAA178EE
:20BDD000002943D0491EC9B20029A1703ED10BF00BFA002565702078E66058B1012007F0F3
:20BDF000E9FF022007F0E6FF06F140004FF0FF310BF0DEF906F140000BF0A6F906F1780095
:20BE10000BF09EF906F19C000BF09AF904F1EC000BF092F904F170000BF08AF904F590701C
:20BE30000BF08AF904F18C000BF082F904F1C8000BF086F9E56004F128000AF0EDF8307C59
:20BE5000012817D10E2002F05FFB13E00BF0CCF9E068864204BF0020E06006F140000BF02F
:20BE700073F906F178000BF06BF906F19C000BF067F9002504F5AA742068B04214BF65603C
:20BE9000256070BD080B00202DE9F043404C054660781F4690460E46ADF1440D012803D03B
:20BEB000FFF7E0FA01206070AEB13648337801684FF0010909FA03F001420CD0B8F1000FAA
:20BED0006E6008D0C5F808800BF092F9A178022903DB0BF089F9002051E004EB8102491C1A
:20BEF000C2F85451C9B2A1700BF07EF94C461FB909A80AF0BBFD09AF386828607868E86000
:20BF1000387C2874B86868617869E861B8696C742862788A6882F86800B1A8610021A0223A
:20BF300005F1280005F0D7F868460021242208230BF03AF98DF8184005F1400000216A46BD
:20BF50000BF02EF968460021242208230BF010F90D49069505F1780000226B460BF004F941
:20BF700068460021242208230BF002F90749069505F19C0000226B460BF0F6F8284611B013
:20BF9000BDE8F083D42108403D64010011700100A00A00202DE9F8430AF0AEFB3E4E054683
:20BFB00015F00A0F4ED0376C002F4BD03869B9693A4A34464FF0000840F00A002840084353
:20BFD000B8613B69C4F84080A2F1100000F108021168994307F11003116093E806000168BF
:20BFF000121C91430160394604F14C00814608F01FFF022104F1EC000AF0C2FCA06C08B3AE
:20C01000F8684068007802281CD197F8270040080CD297F8270080083CBFA06C20640FD3F2
:20C03000A06C2730017841F0020104E0A06C2730017841F001010170A16C484608F0F8FEF3
:20C05000C4F84880326C05F0020005F00807074316D102F1100003C8002301EA0307284034
:20C07000002F08BF00280BD010699769054072644FF4804106F1EC003D4395610AF080FC50
:20C09000306C30B906F13C000AF0E5FF08B103F07FF9BDE8F883C046A00A00201C10044076
:20C0B0002DE9F0473E4C8246A07830F0010708D0042806D0032804D0052802D00AF0F2FDD0
:20C0D000A078384E677904210528DFF8CC90DFF8CC80317007F10101CDB265711DD1022D1D
:20C0F00055DC48460768BAF1010F50D07868398904F0B0FC78680088000905D34146087895
:20C1100010B108F06DFB657928460AF0BAFF8320307009F0D5F9BDE8F087234FE73F97F8A2
:20C13000B810A94233DB032831D007F04DFBA078042809D14146383991F8380020B1D1F852
:20C15000841009B102208847207997F8C510421C9142C4BF401CC1B22171484605686868B3
:20C17000298904F077FC68680088000904D34146087808B108F034FBFEF70CFFA078042833
:20C1900008D08320307007F045FDBDE8F087E12004F01CFCBDE8F087700D00204C150020D8
:20C1B000241A0020942D0020870F00202DE9F8438146D9F808703868066CD9F80450466438
:20C1D0006A6CAB6CA86B16F4F06F0146A2EB03082AD1F00911D270095DD301B395F83C40CA
:20C1F000641EA14298BF0C1C4846214608F0FAFCA86B001BA8630DD04DE081B1484608F06D
:20C21000F1FC95F82D10A86311B9002843D101E00020A86305F19C000AF09AFF3BE048466C
:20C23000414609F0EDF836E0F20A19D24FF00008444602E0A86B401EA86340B348460121BA
:20C2500008F0D0FC3868446814F00F04C0F80480F0D0286B401E2863686B401E686316E03D
:20C27000386844680022202904F00F044260CCBF20270F1C4846394608F0B4FCC7F12007BD
:20C29000B845C8BFB8464846414609F0B9F8EC77484605F087FDB0090BD3A96A49B10F46EA
:20C2B000484608F0D7FCA86218B94846391D07F07FF9BDE8F88370472DE9F04105463E48F8
:20C2D00004780F46002DADF1280D42D03B48466A002F3ED08046D6B17069C0B10123ADF89B
:20C2F000223006208DF8200029460C2200236846ADF8243003F0BEFB03A839460E2203F0B1
:20C31000B9FB766908A803C81A226B46B047787B012668B9002C14BF0FA013A0698810225C
:20C3300007F034FB397B13A00A2207F02FFB08E0002C14BF12A017A00AF042FC19A00AF0D8
:20C350003FFC88F802600020314605F027FC88F803600AB0BDE8F081526573746172746504
:20C37000643A20307800C046537461727465643A203078004368616E6E656C3A2000C0464F
:20C390004465766963652052657374617274656400C046C04465766963652053746172742B
:20C3B000656400C04672657175656E637920486F7070696E6700C046B8130020D411002047
:20C3D00070B53F4C0646A07EADF1200DF0B994F85C0082281AD0394B40F2016046F25C0593
:20C3F000ADF8080034491868ADF80A50426A086802A99047812814BF6FF07F009DF90C00EA
:20C4100009F0D1FB94F85C10226B505494F85C00822814BF401C002004F1180584F85C0053
:20C4300094F85C0005EBE00292F82C00411082F82C10400807D294F85C00401C84F85C0038
:20C45000C0B28128ECDB94F85C0081282CDA05F14401E120FAF7B0FC02204FF6FF738DF81C
:20C470001800A17EADF8103031F0020018D0012919BF0720832108208021002249350092BD
:20C4900004AA0195FBF796F8DB2807D0E52805D0F32803D0DF2818BFE8280AD1607603E09C
:20C4B000304604F0C9FE04E02A203070304606F043FC08B070BDC046D01900202017002077
:20C4D0000C2C00202DE9F04707467D68D7F8089090460E460AF08CFE8246A86A002864D129
:20C4F00005F5847009F038FE0024EC772E6250466C620AF079FE0AF07BFE2F4E33788246C0
:20C5100023B9022008F0BCFE0120307050460AF06BFE2A49086840F480700860384641462D
:20C5300008F098FBA862C0B93846414607F040F8A878D0B9A96805F1D0000AF039FEE8B957
:20C55000AC621020E8774946284604F0EDFE0AF04FFE8246307840B323E0D9F80010886BD1
:20C5700040F020008863A87810B12046BDE8F087A96805F1D0000AF01BFE10B1686ABDE8EB
:20C59000F0873846414607F013F81020AC624946E877284604F0C8FE0AF02AFE8246307827
:20C5B00018B1022008F02AFC347050460AF01CFE4FF0FF30BDE8F087892D00203010004034
:20C5D0002DE9F043DFF8E0808946054617464FF0FF31ADF13C0D40460AF0EAFD334C04EB29
:20C5F000C504666825680AF003FE2168096800290BD42968002905DCB9F1000F09D04FF09E
:20C61000FF3108E0B9F1000F03D00AF0EDFD002442E02968491C29600AF0E6FD2868022826
:20C630003ADA1FB90DA80AF09CFC0DAF38686860B76800213022082301A80AF0ADFD4FF04A
:20C650000009069401AB307B194A09903946CDF8009005F12C000AF09BFD01A82422082332
:20C6700049460AF0A1FD012705F1640001AA8DF81C7049460AF094FD05F1480001AA3946C3
:20C690000AF08EFD706802F029FA0A4A05F118002346042109F086F940460AF0A1FD20462C
:20C6B0000FB0BDE8F083C046282D0020140C0000DD5B0100A36F01002DE9F04106AF3D79FA
:20C6D0003E68984604460B1CADF1180D074611D0012B15D130797379641C3870B17904F86F
:20C6F000013B337A04F8011BB17A04F8013B7389181201E03178707804F8011B04F8010B0E
:20C710008AB9002D0CBF42F20C0042F20D00694606F0C2FF9DF80000BDF8003004F8010B65
:20C73000181204F8010BB8F1010F34D0B8F1020F39D1002D0CBF42F2020042F203000DF1D3
:20C75000020106F0A9FF7589CDB1681E01468B100DF1020201EB5371C910CBB2811000EBC0
:20C77000517121F00701401AC0B20121401C01FA00F0D15CFF3080F0FF000843D054E81D5A
:20C790000DF10201C210204603F074F97089C01D04EBE00407E0002D14BF022101212046B5
:20C7B00002F000FC0419E41B06B0A0B2BDE8F0812DE9F04390460A68D8F80040167881464B
:20C7D00000271D463846ADF1140D531C242E0B6053D112F8016F5B1C4C2E0B600ED1AA686B
:20C7F000E41C24F00304241D54F8040C494606F099F92968EF600127091A2960462E1AD147
:20C81000E41C24F00304241D54F8040CE41C029024F00304241D54F8040C002749460390BD
:20C83000AA68ADF8047001A803F086F82968EF600127091A2960532E1FD1E41C24F0030463
:20C85000241D54F8040CE861C8F80040288B0090A968EA69D9F800004346F7F7FDFED9F827
:20C870000040002714B10119C9F80010D8F800402968EF60091A01272960662E0AD12B8BA8
:20C8900023B9E41D24F00704083403E0E41C24F00304241D1FB9E9690E700127EF60C8F832
:20C8B000004005B0BDE8F0832C4870B50568B5F1FF3F08BF002509F011FD01284DD107F040
:20C8D0004DFC142849DB26482649002601230660254A0B60254C136020680028FCD1264A67
:20C8F000131D2349186820F00300014321480068C0080CD2106810F0030F0AD041F00300A6
:20C910001860106800F003000328FAD101E041F001011A481960006820B1194800682846CF
:20C93000F5F76AFD174818490660184D0A686FF35B4245EA0200086015490868C0F301304D
:20C95000012806D10A681348104040F400320A60086020680028FCD170BDFEE71C13005064
:20C97000840460425C600C40082204430C00684204000020B03F005000400340800128437C
:20C99000000120438C210840482003400000390104000940FFFFFCFC2DE9F04F09AF3C8934
:20C9B0007D6816464FF0000A0246002EADF1440DA04610933C888DF83CA05CD0304810F81E
:20C9D0000690042E03DAA8EB0900C8462D18F868A4EB080407AB0827A4B2C01D10F801C9D2
:20C9F0007F1E03F801CBF9D1080E264F03F8010B080C03F8010B080A03F8010B386803F898
:20CA1000011B9DF83C101E704369786898478346BBF1FF3F2AD0042E04DA03208DF80000AB
:20CA3000022002E002208DF800008DF8140002959DF83C608DF8026001218DF8011038689B
:20CA50008DF8039007ABADF816800BADADF81840026A0193109E04956946786803969047C6
:20CA700083463868826978680FA99047BBF1000F18BFE42000D1504611B0BDE8F08FC046FB
:20CA9000480C0000702D0020394833492DE9F047012500240570DFF8C480DFF8C8900C70A6
:20CAB0002F4901F16A06378882460220104014EA030608BF00280FD120464FF0E0471040A1
:20CAD0001F4008BF002832D0424692F90000401E107009F0E9FE2AE0424692F90000401EAA
:20CAF0001070BFB94A8E43F2084320464646934204D191F84010090938BF281CFFF7D0FA54
:20CB10004846047096F90000F0B196F90000002817DD1DE0B7F5505F07D1144812490068D9
:20CB300000F5C070086001F031FC09F099FE48464246047092F9000030B192F90000002801
:20CB500006DC0AF0AFF803E020460146FAF730F88AF80040BDE8F087981B00209E1B00200F
:20CB7000D8120020971B0020181700200C010021A21B00202DE9FE4F83460020304E009015
:20CB90007068019180472F4C0290E06804216A4604F0CEFF2C4DDFF8B4A0DFF8B490DFF8D3
:20CBB000B8802C4E2BF0010725F00105BD4213D0504620F00100B8421CD1494691F90000EC
:20CBD00010F1020F18D03068826B91F90010E068904781280ED10FE0414691F9000010F184
:20CBF000020F09D03068826B91F90010E0689047812801D00AF056F83068C66A1749019A78
:20CC1000E0685B46B047061C01D50AF04BF8BD4207D0504620F00100B84204BF49460E70A8
:20CC300001E041460E7001200090E06804216A4604F07EFF0249029889688847BDE8FE8FE8
:20CC5000B4150020C4190020F9DE0000E9F90000951B002020170020941B0020D812002025
:20CC70002DE9F84F07463248DFF8C89000EB4706183699F83800348890468B46B8B1D9F865
:20CC90005010A1B12C4D05EB8705686B00F0FF0088478246D9F85010686B00F47F0088473E
:20CCB000504480B218B131884018001D84B225481230007801280CD198F808604EB11F48E6
:20CCD00098F8093081190D79C05C2418641DA4B200E00025281980B209F050F806461848C7
:20CCF00090F80090D6B13046002122460AF0C1F94FF00008A41937700D4986F8018006F1DB
:20CD100080007460CA5D3581594609F0E5FD4846314605F0C3FD4046BDE8F88F8DF80070F7
:20CD300068461A2103F0EEF91A20BDE8F88FC046880300001415002070080000440C000018
:20CD50003C1600205A0F00202DE9F04F364E0025ADF1340D07464FF0010AA846A9460C93D8
:20CD7000DDF858B00B914AE017F8020FAD1CADB2401E1BD0401E09D0401E04D0401E36D1A1
:20CD9000022C34D138E0032C31D135E0072C2ED1B9787878FB1C40EA0120A6F844001868DB
:20CDB00006F14802106086F859A025E0052C1ED1CDF80890B91C0A8802A802808978817034
:20CDD0000B9803A9FBF7C2FE9DF82A00A0B1029B40F0020000F0F7008DF82A0006F1500284
:20CDF00003931068049003A805F0B0F904E008EB0400801C1FFA80F8E7196419A5B23846DE
:20CE1000694608F019F9041CAED1022D03DC4D466720A84600E048460C990D800DB0ABF894
:20CE30000080BDE8F08FC046D02900202DE9F84F0D46064628684FEA900A3248504502D3DC
:20CE5000287A022802D00320BDE8F88F0AF0D0F9DFF8B4800090D8F8580108F5AA79B0423C
:20CE700014BF00240124A00080F0040059F8007006F19C0083460AF002F968B957B107F13F
:20CE90009C000AF0FCF838B93846022100F060FF074602E0022700E000271C4800686FB9C4
:20CEB00098F8880140F0020088F888010098C8F87C610AF099F90020BDE8F88F2A68A100CE
:20CED00001EBC40149440A612E7A0E76BAFBF0F1012998BF012158460AF042F958460AF0C9
:20CEF0007BF900980AF080F9012F07D1D8F88001B8F9841198F886210AF03FF88320BDE854
:20CF1000F88FC04640420F00A00A0020B00C00007CB5354C054694F8A1000F285ED0334853
:20CF3000697E0078890959D2297E002841F00201297639D069684A1C1078801010F0030FB9
:20CF500032D000F0030002280ED1B4F8B4304FF6FE70984208DD56791179002001EB062135
:20CF7000994208BF012004E004F1AA00491D09F021FBC8B9687E696840F0010068764A78D7
:20CF9000C2F38102022A2DD1491D4A7809784FF6FF7601EB02218E4224D1297E00F0EF0062
:20CFB00041F0200129761CE0687E114E40F0030068763078B0B994F8D7008DF80000FF2303
:20CFD0008DF8033094F8E6608DF8016094F8E7508DF80250684609F0CCFF7CBD687E40F076
:20CFF000010068767CBDC046A00E0020141500205719002070B50546344C2878ADF1200D01
:20D0100000284FD1208F04F148066B88ADF800003146ADF81030E22009F01CFE0DF11200AD
:20D03000314609F08AFF6988532009F005FB208F04F13E063146ADF80E004A2009F00AFE0D
:20D0500001A8314609F079FF00268DF80D60A08FADF8020094F83A308DF80C30304608F01C
:20D0700057F95220314609F0DBFA94F850000F281CBF01206070E06828B102681AB10DF166
:20D090000E0069469047032007F0BCFF94F85200032818BF042813D104F10800102109F000
:20D0B000B7F90DE00020607009F076FD41F2883008F02EF90649B1F84E00401CA1F84E00D4
:20D0D000216E09B12846884708B070BD70140020B81300202DE9F0470D4606465FFA85FA82
:20D0F000280824BF2E4845402E494FEA8A03C85885EA00023240C2F300672B4A06EA050448
:20D11000B043224006F4E0240243B4F5E02F01D1500E14D306F4E020074310D002F4E02777
:20D13000B7F5A02707D0B7F5803704BF22F4003242F4A02203E022F4803242F4C022DFF895
:20D150006C80CA5008F1D00739680122002002FA0AF40C4218BF101C5FEA000906D1F00D94
:20D1700004D34146C5F3805001F80A00300E0BD30AF03EF8290E34BF0021211C3A68A2435B
:20D19000114339600AF030F8B9F1000F06D0F00D04D34046C5F3805100F80A10BDE8F087D0
:20D1B000006000A000100840007F077F002002402DE9F04117460D460AF01AF8324C804659
:20D1D000207883266DB16D1E04D06D1E55D0681E11D00EE0B4F8C4004FF6FF71814202D0C2
:20D1F00005E0206C08B9802648E0206C808C388044E0032642E0386800215022054603F0EF
:20D210006AFF022704F5AA7C04F5B272A5F110015CF8040B41F8100F137A0B735068486063
:20D2300052F80C3B7F1E18448860F1D1206C002808BF02200ED0206CC068276C286297F8CF
:20D250002600236C85F82C00D869226C6862106AA8620320E76B8FB105280FDAFA68010114
:20D270006A5097F826204C192273FA6962603A6AA2603F68401C40B2EDE73870404609F05A
:20D29000B3FF3046BDE8F081A00A00202DE9BE410546DFF8CC802978B8F86000E1292FD039
:20D2B000B8F86200E92926D0B8F86400D9B92D4C2869676A02903FB37F692FB3A16A193120
:20D2D000814221D806208DF800000422ADF802200023ADF804309DE8030002ABB84708B9F9
:20D2F0000298A06210E0401C80B2A8F8640019A009F07DFE08E0401C80B2A8F8620003E078
:20D31000401C80B2A8F86000687830F07F071ED000F06001402906D12F7827B9B8F85210D1
:20D33000491CA8F8521000F06001202906D1287820B9B8F85800401CA8F85800602906D1D0
:20D35000287820B9B8F85E00401CA8F85E00BDE8BE81C04664617461436E663A2000C046E1
:20D37000B8130020D4110020F0B52A4A2A491778ADF1140D002F44D02C48077837F07F07F0
:20D390003FD1488C2A4F254D2A4B401C0024488407F16806012097F87410287001F0F001D9
:20D3B00087F8741019783C67012902D02146F9F7FFFB09F034FE1C4D281D00688047074684
:20D3D000029402201C4A164B8DF80C0021468DE803001068314602AAF8F738FB1749002809
:20D3F000A1F12001088008D40E49154C91F90000401C0870A4F114000660A9683846884783
:20D4100006E0888C401C88840020107009F062F805B0F0BD922D0020241A0020971B002036
:20D430006D0F01009E1B0020B4150020942D0020D8120020A21B0020D0190020141A00207E
:20D45000201700202DE9FC47314CA11D0888401C088008F091FD0026B0463546814628460B
:20D47000694604F013F88246BAF1FF0F4CD09DF80030606B23B900EB4A104068010402E011
:20D4900000EB4A104168484609F0DBFD864203D29DF800700646D0466D1C0A2DDFDB1E4D46
:20D4B000281D0068804794F833106FB9A26B08EB88030026FF27491ED218D670137917716F
:20D4D000C9B284F833100CE0616B0022FF2701EB48118A77CB7FCF7794F83210491E84F87B
:20D4F00032100C4A643BD9B2136804EBC1013C310B6052684A6094F88C10491E84F88C104B
:20D51000A9688847BDE8FC8709F099FDBDE8FC87CC100020740C0000B4150020E0B50188B9
:20D530000025A1F6020159B143F20402891A04D0491E57D190F8246000E00226C76901E0AC
:20D55000C67B4769002F4DD03F1F052044F2380357F8041F0A04120C934203D0401EF7D11E
:20D570003F1D01E0C1F30345002D3BD01F4B3046401F18D01C4A401E10D0001F0CD0801EC6
:20D590000DD0C01E06D00F3819BF1A1C6032184A443204E0121D02E0121F00E0083A10686B
:20D5B000C0F3834003E01A461068C0F303200F2806D0A84216D921F4702141EA004110E06C
:20D5D000761F0AD0761F08D0761F06D00F3E1CBF21F4702141F4802103D121F4002141F411
:20D5F000E0213960E0BDC0460011005020130050C4100050F0B5064600210B22ADF1240DC8
:20D610000DF1190009F035FD2E4F2F4C3078C01E14D0801E04D0143810D0801F01282DD8EB
:20D6300001208DF8180006F18B0103A809F0FDFC032538788DF8145068B112E000208DF88B
:20D65000180006F18B0103A809F0EFFC032538788DF8145028B9B4F8BE000225ADF80200B6
:20D6700005E00DF1020004F1D80109F0DEFC8DF80A50B4F8BA00ADF8160017E002208DF876
:20D69000180006F1320103A809F072FA0DF1020006F1280109F06CFABA34208806F11C01FF
:20D6B000ADF816000DF1190009F0BCFC0B208DF8000077788DF80170684600F0DBF809B018
:20D6D000F0BDC0464C150020A00E00202DE9F84F8A463149044601F1B400007828B92046E2
:20D6F0005146F7F7C3FDBDE8F88F0A25884642F2107B20465146F7F7B9FD98F8B4100028D0
:20D7100048D19AF80060D4F80090002937D023480168C88AC20832D280094FF0000702D3CA
:20D73000087D15282BD008F007FC98F800308446002B0EBF09235B1EDBB20A2003EB8302D0
:20D7500008EB0201491C0A78964207D0002B0EBF09235B1EDBB2401EF0D110E0D1F801101A
:20D77000604609F06EFC642101FB09018B4505D942F242706426401AB0FBF6F717B9002005
:20D79000BDE8F88F20686D1E07442760B1D109F056FC6120BDE8F88FD0290020700D002038
:20D7B00080B50288A2F602073FB143F20502BF1A14BF002090F8240000E0C07B2C4AD2F8FA
:20D7D0008832401F0B6048D0401E3CD0001F30D0801E24D0C01E18D00F380CD0D2F890023D
:20D7F0004860D2F894028860D2F8BC0220F0784040F080503AE050694860D06A8860506C80
:20D8100020F0784040F0704030E010694860906A8860106C20F0784040F0F04026E0D0685B
:20D830004860506A8860D06B20F0784040F0C0401CE090684860106A8860906B20F078409A
:20D8500040F0A04012E050684860D0698860506B20F0784040F0405008E0106848609069F1
:20D870008860106B20F0784040F02050C86080BDC410005070B50646304930780D5C401FEA
:20D890001CD0083851D0401F4FD0284608F076FA041C0DD130780C2808D1706830B1301D1E
:20D8B00006F05CFD284608F069FA0446002C43D02A462046314609F00FF837E0B07810BB60
:20D8D000327A307C51005410401901F00E01091804F0380040182430C0B208F04FFA041C06
:20D8F0002AD03146182208F0F7FF04F1180060607168242208F0F0FF6068243060617169F5
:20D91000327C0E46D6E7012816D12435E8B208F035FA041C10D03146182208F0DDFF04F194
:20D930001800606071682422EBE7344624B104480078214604F0B2FF70BDC046EC0B0000C5
:20D95000A41B0020F8B509F067FA04F0C3F909F07BFA044604F00C000C284BD0E0081ED242
:20D9700007F040FF264E376805460120014608F041FC31686943884211D2224C8220B0FBB9
:20D99000F7F0291A204609F0EBFB204609F024FC0120F8F7D1FC204608F0DEFB2CE0200940
:20D9B00028D2194809F003FA0428FAD0174A610905D220B11168104621F0010103E0104682
:20D9D000016841F001010160983210684FF0805540F003001060D5F8B801816920208847C2
:20D9F0000B4CD5F8B8712068B86B804701202060206801E009F01FFB09F014FAF8BDC04679
:20DA1000B00C0000C40F0020004003408C2108402C200940F8B5324D6868804706462E4CB1
:20DA3000A9682068002853D160698047676A40F01000002F4BD00022797E0140884205D00D
:20DA50003A4657F80C7C002FF6D140E004F12400394606F0E3FE002F39D02760787E30F005
:20DA70007F0005D194F82F00401E84F82F0004E094F82E00401E84F82E00A9683046884781
:20DA900023681889D98A05F059FBA0851348007807F086FC0546D88A000A08D3D87E05F050
:20DAB00037FD206890F91C0009F026F82368687B012803D002280DD1052005E0187E40107C
:20DAD00080F0010000F00100FAF742F9F8BDA96830468847F8BDC046700D0020870F00208F
:20DAF000B41500202DE9F047294E04463078ADF1280D012849D1DFF8B09009F120000068C8
:20DB1000244F436CF868022108AA98479DF82000002831D1DFF8948008F1040000688047C9
:20DB30000024022582461C48059404A90490F8688DF81850FFF77AF93570029417498DF8AE
:20DB50000C50174B4C8126468DE86000F86802AA0831F7F77BFF002801D509F0A3F8114950
:20DB700091F90000124E45464F46401C0870A968FE605046884708E03078012805D1002034
:20DB9000012C307001D008F083FE0AB0BDE8F087A31B0020C419002000093D00D81200205D
:20DBB000A13101009E1B002000170020B4150020E01200202DE9FF412E482D4F00683E7811
:20DBD000C06B80477968401AB100B0FBF1F4B868FF680025A8464146BC4271EB080101DA68
:20DBF000B84206D82946424684428A413CDA074600E0294638463246F317001BA94108F006
:20DC10008FFE272704464FF47A7200230D46ADF802700820ADF800002046F8F7B3FD0190B0
:20DC30001548016868468847029843464FF0000100F6FC02A41A9D416042A94111DA0F48D0
:20DC5000026829462046F8F79DFD0D4604464FF000016042A94104DA204606F05FFA0020D0
:20DC700000E00120064908700090BDE8FF81C046241B002020170020D8150020B019002065
:20DC9000932D00202DE9F84F2E4C012683461D4690468946C4F87C670320C4F880670AAFA7
:20DCB000C4F88407D4F88C0710F0030FFAD1387A58B14FF0805ADAF8B001016A27208847F9
:20DCD000DAF8B0010169272088470220C4F8FC063868C4F80804304609F086F9D4F8080423
:20DCF0000008F8D2D4F88C07800F28BF301C26D22868C4F83C056868C4F84005A868C4F8FF
:20DD10004405E8681049C4F848053879002814BF081D081CC4F84C05C4F850850020C4F889
:20DD30005405C4F8580509490E60C4F800B0C4F80880C1F80064C4F82090C4F82880BDE85F
:20DD5000F88FC046044002402800002000004842314A2DE9F0410446106C002301261F4697
:20DD700087420CD0106CC068844208D1106C90F8260008F041FF3E46031C18BF176CD56B0C
:20DD9000DDB1D56B17E0C868844205D191F8270040F0080081F82700096826E0E8688442CD
:20DDB00008D195F8260008F027FF002608B10BB92F4603462D68002DF0D1002E18BF02209E
:20DDD00027D1002B14BF002F002022D0106CC0683946844209D1106C884206D1106C273049
:20DDF000017841F008010170D16B0029CBD1C2F87C4192F8880140F0010082F88801BE8CE6
:20DE1000C2F8804103F00103A2F88461012082F88631BDE8F081C046A00A0020F0B50646D8
:20DE30000F4600251446ADF1240D8B200DF10E010095FCF77DFB8A2001A9FCF779FB707AD2
:20DE500000282ED1387AA0B9BDF80E104FF6FE70884205DCBDF80E10884220D101A90DE02A
:20DE700020489DF80E700488BDF80E008DF812700CE0022807D0032811D1394604A809F0A3
:20DE9000D4F809240BE038888DF812008DF81040211200128DF8111005248DF81300284648
:20DEB00011E002280CBF05240924012818BF311C04D1892007A9FCF73BFB07A9224604A8AE
:20DED00008F00AFDB07A04EB0D01C8736A4604A8214603F065FA002814BF281C009809B02C
:20DEF000F0BDC0465A0F00202DE9F041294D012001462870F8F75CFE27496FF00100087088
:20DF10002B480068C06B8047244C074621786068A2688B003E1AB6FBF3F05843361A880012
:20DF30001F4902FB03F8B1FBF0F0904201D208F0B9FEB91B1B4861604144FEF71BFE1A4CA0
:20DF5000A06867682168404207F00EF8002F08BFA16808D0A16878688142DCBF401A786082
:20DF70003F68002FF7D1E068884202D0A06005F051FC02F0A3FC0D4C606880470646FFF712
:20DF900019FEA1683046884708F0C0FA00202870BDE8F081A21B0020941B0020241B002081
:20DFB000FFF6C2FFF9DE0000801B0020B4150020201700202DE9F84F07460E1C14BF4FF0E3
:20DFD00000094FF0E809002F4FD0B9F1000F4ED17868401E78603F210170BD6D002D0CBFC9
:20DFF000802000207968DFF890A00224083E491E7960DFF880B008703889A7F85440801CAE
:20E01000388116F8080FFF282CD02A2828D1706830B35546296D8847804678689BF8002090
:20E03000A0EB08007860716829B96D6D3A460023A84748B10BE06D6D786871688DF8002022
:20E050006B463A46A84710B9EB20BDE8F88F3889B7F854504044388108EB0500A7F8540054
:20E07000641ECED17868386501E04FF0E8094846BDE8F88FE42C002014150020F0B52F4C8E
:20E090000546A07EADF13C0D022806D0012804D005281CBFE820607649D194F8600000280F
:20E0B0004AD1002109A81822617608F0E2FFCDF828D009A8294600F0B5FC94F82E0094F8B5
:20E0D0005810814220DD266B70B10746BDF80A007189884204D13046694607F06DFB98B9DC
:20E0F0007F1E06F12406F1D194F82E00276B8100242201EB40117818694608F0EDFB94F895
:20E110002E00401C84F82E000D48007828B19DF8340010B994F8580028B909A8FFF7AAFB72
:20E1300094F8580040B194F82E10884204D12A202870284604F000FE0FB0F0BD0C2C00208B
:20E15000360F00202DE9B841804607F0F3FCC01DC51098F82300002849D198F87E4007F0A3
:20E17000E9FCA04243DD264A1368E010191891F86C1004F007042141CFB207E0401CC0B200
:20E190001918C40091F86C7088F87E4047B9691E8142F3DC1068002188F87E10417029E05D
:20E1B00098F97E10C0000830884226DD401A79080BD298F87E10401E4FEA670701F101019C
:20E1D00088F87E10F3D1BDE8B88198F87E000D49087098F87E0088F8810098F87E00401C2A
:20E1F00088F87E000320F9F7B3FDBDE8B881002088F87E00072005F0EDFBBDE8B881C0466A
:20E21000700D0020C41900202DE9F041054608F055FC287E000904D2287D012808BF022736
:20E2300000D00527DFF89C80464670688047264C04F124010B68002B08BF0D600CD07F1EDD
:20E250000026FFB202E07F1E1346FFB253F80C2C22B92FB143F80C5C012601E0002FF2D173
:20E27000D8F8081088471EB3216928468847E88AA168C00818D2D8F80400804794F82F10AC
:20E29000491C84F82F10D8F8081088470C4991F8380028B10846C06C10B18047BDE8F08190
:20E2B000FFF7B8FBBDE8F08128468847BDE8F081F1206870284604F043F8BDE8F081C0469A
:20E2D00014150020B4150020700D00201A481B4901641B4941641B4981641B49C1641B49F5
:20E2F0000165022280F8202019494165194981651949C165194901661949416619498166D9
:20E310001949C16619490167194941671949016019494160194981601949C1601949016140
:20E33000002180F83C1080F83F101749C161C162012180F830107047942B0020CD6F0000D0
:20E35000A5300100953B010031340100ED220100154B0100B55C0100D53E0100A12D01003A
:20E370002D43010011680100E90A01005D3F010001650100F56C0100696001004DFF000032
:20E39000B523010077700100256D0100F8B5264C236813B908F086FC236824480068044680
:20E3B00008F096FBD860204608F078F8264C18826068804706461E48A1680278832A30D140
:20E3D0001C4DEF782FB386210170082007F054FEE88C1B4F1949401CE88417483A788162F6
:20E3F0001849812A09DB0978842A07DA40F6485292FBF1F101F6B83106E0097840F64852B7
:20E4100092FBF1F101F2A321203008F08DF8A16807E08522027030468847002002F0D6FAC9
:20E43000F8BD30468847F8BD700D002018170020942D0020241A0020F4190020713801001B
:20E45000870F0020241B0020B415002003B42DE9F0472C4C4FF0000908AF84F80190396885
:20E47000ADF1100D02A80160B988818002A803C89A46164602F0DEF9A046051C14D04C468D
:20E4900086B128466946012206F06AFE1AF804009DF80010884205D1641C6D1CE4B2ADB23E
:20E4B000A642EEDCA64227D0B8F80200F61C4FF6FC7440F6F87134402018814203DA08F05F
:20E4D00031FCFCF7C7FC396802A8BE88016002AD868095E803002246534601F0DDF998F8CA
:20E4F0000100B8F80210002818BF814604D10919083188B2A8F80200484604B0BDE8F04759
:20E5100002B07047281C00202DE9B043044608F06FFE81462748021992F8EE10491ECFB2A5
:20E53000002F82F8EE703FD1254901EB84014A880C78904634F07F0718D1E1090FD24FF00C
:20E55000805000F5DC75D0F8B8018169104688472868416B404688470228F9D11EE000EB97
:20E570008800D0F804110020884717E04FF08055D5F8B801016A10468847D5F8B801816AA5
:20E5900040468847D5F8B801016B404688470A4901200860094908688008FCD304F03F00A7
:20E5B0003F2801D0FFF7B0FF484608F01DFE0020BDE8B083B80F00202820086028200840AE
:20E5D000B0090000F0B52B4D05F12C0158C9ADF11C0D02AA58C20AC94FF0805682E80A0028
:20E5F00047688468D6F8D001C16820688847216821488A6B10408863206840F2F27141646D
:20E6100097F83C0097F83D10C0100DEB80008068084321684863684608F086FDD6F8D001CC
:20E63000397F466805EB8101BA698B68797F206855F821101943BB7F05EB8305AB690B436E
:20E650000199B0470D490A1F106840F010001060086840F001000860A07D0027FF2802D02C
:20E67000E07DFF2800D11FB1086840F44040086007B0F0BD440A00000DF8FFFF30100040A4
:20E6900029482DE9B0410025DFF8A080294C0570ADF1140D88F83B50012088F83800201D0C
:20E6B000006888F83D508047234924310F686FB1797E8A0806D341F001017976397E01F08A
:20E6D000FD01397657F80C7C002FF1D1A1688847102008F01FFB082008F01CFB98F83C0098
:20E6F000E0B90920124C8DF80000B4F8BA108DF80F50E027ADF8021094F8D7308DF80170C4
:20E7100094F8E6208DF8043094F8E7108DF8052068468DF80610FFF7ADF801E088F83C50A0
:20E7300005B0BDE8B081C046141500201C190020A00E0020B4150020700D002070B50546D6
:20E750002B4C2878ADF1200DEB2829D040B3E92806D0E12843D14FF4FA7006F0A9FD3EE05D
:20E7700004F156010878401C087094F85200032818BF042803D14FF4FA7006F099FD94F844
:20E790005600032809D094F85200022827D104F10800102107F03CFE21E007F03FF91EE082
:20E7B00094F85200022817D104AE6946304605F0F5FD5220002107F033FFE06820B102685C
:20E7D00012B1304669469047042006F01BFC04F10800102107F01CFE002084F856000548BB
:20E7F0002A30016809B12846884708B070BDC04670140020C614002030B50446ADF12C0DC0
:20E8100008F084F9002818BFFC2050D168462146112201F02FF9A57C617D8DF81250607C14
:20E830008DF81510E37C8DF81100227D8DF81330A57D8DF81420002105B10121257E8DF8C6
:20E85000161094F825208DF81850E07D8DF8252094F824308DF81700E58C8DF8243004F1E2
:20E8700019010B220DF11900ADF8265008F034F8607C1A2550B9812007F034F904460A941A
:20E89000A4B1FF21812208F0F4FB09E09DF81510880000EB411080B207F024F904460A94D4
:20E8B00024B10720694603F081FB002528460BB030BD10B5401EADF1380D28D0401E09D0BE
:20E8D000801E4FD0401E43D0401E3FD0401E3BD0002048E001A800F0B7FC04460CA942F25D
:20E8F000090004F0D9FE9DF83000002808BF002203D0022006F042FE024601209DF83010F5
:20E91000009001AB204605F0CCF90A3028E001A800F09AFC04460CA942F2080004F0BCFE31
:20E930009DF83000002808BF002203D0012006F025FE024600209DF83010009001AB204605
:20E9500005F0AFF9001D0BE020200CE002200AE042F2130004A904F09FFE04A808F0F4F8B5
:20E9700080B200E004200EB010BD704770B5204E002086F85400032186F85500E82007F094
:20E9900067FE5220012107F04BFE1A4D482205F1700406F15C00214601F06CF816486867B7
:20E9B000343CF4601548E8671548C5F8A0001548C5F894001448A8671448174CC5F8800008
:20E9D00013481649C5F88800124847F23052C5F8900004F1980005F08DF84EF660221049A0
:20E9F000A06104F1BC0005F085F8E06170BDC04670140020B813002005D00000DD4A0100E3
:20EA1000A91801004DE70000815301005D030100790D0100E90F0100D4110020716501005E
:20EA300009610100F8B505460E460520287096F849006968E870F06B4861686806F128015E
:20EA500008F096F8B6F842006968488196F84600696848746868002404761F486968007817
:20EA7000C873686806F11C01193008F0DBFA307C69688873706810F8011B6A68918110F8F1
:20EA9000013B6A68918941EA0321918107786A68F91117F007071174214607EB470218BF6F
:20EAB000012189184018401C10F8011B297201F00702E860491001F0380101EB42014018C4
:20EAD0007268318968618B18834239BF2C72211C801A091A2974F8BD860F0020F8B50646D1
:20EAF00008F086FB264D0746A91991F8EE00421C002881F8EE203ED1224C04EB86042678F3
:20EB100006F03F003F2801D0FFF7E8FF648836F07F0018D1F0090FD24FF0805000F5DC75F2
:20EB3000D0F8B8014169204688472868416B204688470128F9D11EE005EB8405D5F80411A8
:20EB50000120884717E04FF08055D5F8B801C16920468847D5F8B801416A20468847D5F892
:20EB7000B801C16A20468847074901200860074908688008FCD3384608F036FB0020F8BD00
:20EB9000B80F0020B009000028200860282008402DE9F84F294C8A468346211D08880A251D
:20EBB0004FF0FF09002604F13C084746401C088038465946082207F0F3F830B16D1E07F1A1
:20EBD000080706F10106F3D100E0B146B9F1FF0F05D1207A401C2072FF20BDE8F88F48468E
:20EBF000694602F053FC0546FF2DF5D09DF80000012806D0A06B05EB8501401880F804A050
:20EC100004E0606B00EB451080F81FA009490A6808EBC900026049684160074E7068804796
:20EC300094F88C10491E84F88C10B16888472846BDE8F88F740C0000B4150020CC10002036
:20EC50002DE9FF47DFF8888001270446214E88F800703078012803D038460021F7F7A8FFC0
:20EC7000204605F09FFD214D68688047002482468DF80C701849029418484C8302238DE8DB
:20EC90001800174B006802AA18318946F6F7DEFE1449AA680028C8800AD4134B93F900004E
:20ECB000C1F80C90401C1870504690473C460AE040460470504690473078012803D02046C1
:20ECD0000146F7F775FF20460090BDE8FF87C046981B0020A21B0020D8120020D019002091
:20ECF000D1340100001700209E1B0020B415002010F47C1F70B51CD110F00F0F1CD0014603
:20ED10000024012202EA010091435200401E0BD0401E07D0801E03D0001F07D1093404E092
:20ED3000241D02E0E41D00E0641DA4B20029E9D133E010F00F0F01D0002070BD0646022444
:20ED50004FF4803505EA0600AE436D00B0F5803018D0B0F5803013D0B0F500300ED0B0F58B
:20ED7000802009D0B0F5002004D0B0F580100FD1072008E0062006E0052004E0042002E032
:20ED9000022000E00120FFF794FD2418A41CA4B2002ED7D1022CD8BF0024204670BD70475E
:20EDB0002DE9F0470020DFF89080224E234D88F83D0096F8A19095F84000401CC0B20428CC
:20EDD00085F8400030D0202005F0CEFC96F8E3100F2917D098F83E7096F8A100B84211DD72
:20EDF000194C8946606886F8A170804782461448144950F827008860C86004F00BFDA168AC
:20EE10005046884795F8401096F8A13038F819404FF4707205F11000491C9A4001FB14211D
:20EE300006F04CFEBDE8F08706F06AF8FFF728FCBDE8F087A00E00201C190020782C0020F1
:20EE5000840A0000801B0020B415002070B52348214D286522484FF08056E864D6F8D80173
:20EE7000204C036801210A46ADF1400D20469847D6F8D80142680121204690471A480126D0
:20EE900006601A48F9F7B0FC05F0C8F9284607F057FC05F118044FF4E1302946206000201B
:20EEB00005F0DCF912493C22082308600021684608F036F9F0344FF46170002307940D49EA
:20EED00008906A46069605F1580008F025F908F01FF910B070BDC046080200202970010013
:20EEF0006D4401000040034004011CE2C40A0000980600208131000090B50446002140227A
:20EF1000ADF1440D684602F0E6F8A0788DF80000E0788DF801009DF8000000BB616811B11E
:20EF300001A805F079F8217A01F007028DF82820E0689DF82870C1F302118DF8301027B177
:20EF50009DF828100B9000EB41009DF8307007B10D90207C8DF8380067690F9719E06168F2
:20EF700011B101A805F058F8677A8DF82970A37A8DF82A30207A8DF82800E27A8DF82B2063
:20EF9000217B8DF82C10677B8DF82D70E389ADF82E300348006801696846884711B090BDE9
:20EFB000741B0020F0B5012904460546ADF1140D04D0022941D142F2030001E042F2020010
:20EFD000694604F069FB04B16D1C06F0B3FDC01DC010C0B2002830D000230646ADF1010CD5
:20EFF0001F4618461CF801EF00224EFA02F101F00101884211D028B97F1CBFB25CB102EB58
:20F01000C30103E03CB102EBC301491E05F8011B091205F8011B80F00100521C082AE4DB17
:20F03000761E03F10103DDD130B12CB1D800401E05F8010B001228700FB9002005E004B15D
:20F050002770012000EB870080B205B0F0BD70472DE9F843254C804660688047814669469E
:20F07000722006F063FC3225FF27002600994046091D07F09FFA012808D000986D1E06F106
:20F09000010600F118000090F0D100E03746A16848468847FF2F18BF381C22D1144DD4F8C3
:20F0B00004900A2700263C3512492846082206F077FE30B17F1E05F1080506F10106F3D143
:20F0D0000DE040460168296040686860C847064A92F88C10491C82F88C10A16888476436D9
:20F0F000F0B2BDE8F883C046CC100020B4150020CC100020740C00002DE9B841044608F086
:20F1100077F8DFF89880054608F5C4710878A04308F5AA7408702068002808BF002706D09A
:20F1300020689C3007F0ABFF002700B10127606838B19C3007F0A3FF0024384318BF012419
:20F15000274698F8880120BB012F22D0D8F87C0110B3C76917B1016A890811D24069D8B103
:20F170000746284608F040F8D8F87C0100214FF400030A46B8470020C8F87C01BDE8B88156
:20F19000284608F031F8D8F87C0102210022B847F1E7284608F028F8BDE8B881A00A002039
:20F1B00038B504F011FB02F0CDFE204D05F13800007820B11F4808380168012088471E484B
:20F1D000007810B91D48007808B107F06BFD1C4C606880471B4AA1681378022B1CD1144C7F
:20F1F000A31C1B78042B1CBF832313708847A17831F0010008D0042906D0052907D100206F
:20F21000607107F03EFF01E0FBF7C4FEA178042903D006F0B1FF00E0884795F8380020B140
:20F23000E86C10B1102007F075FD38BD14150020241A002018170020902D0020922D002069
:20F25000B4150020942D002070B50446E820ADF1280D09A904F0E2FB9DF82400694606F0A9
:20F27000ABFF00280CBF00981E480DF125016060E82004F0D3FB9DF8250004A906F09CFF3D
:20F2900058B90599C8200322B1FBF0F0401EB0FBF2F15143401AC0B200E00020207206F042
:20F2B00049FC00216081656821700F4B61700A4608925968A9420CD1197A267AB14208D1FC
:20F2D0005989814205D1187820705E786670104606E008990C33491C06290891E9D90120AB
:20F2F0000AB070BD38C40D00581700202DE9F047254C01258246984691460E46C4F87C573B
:20F310000320C4F8805708AFC4F88407D4F88C0710F0030FFAD1387858B14FF08057D7F84F
:20F33000B001016A27208847D7F8B0010169272088470220C4F8FC06C4F80894284607F0EE
:20F3500053FED4F808040008F8D2D4F88C07800F28BF281C15D2B8F1010F14BF08200C20C2
:20F37000C4F84C051021C4F850150020C4F85405064A1560C4F800A0A160C2F80054266231
:20F39000A162BDE8F087C0460440024000004842B0B50546264CE968E06888423FD1A86883
:20F3B00002F038FFA0B1E9684968A06C0978022900D168B9012004F0FDFC832835D1E06810
:20F3D000783006F0C9FE04F1C80007F005FFB0BD16492869A1F10802136805F11007184324
:20F3F000106097E80C0051F8102C181C104341F8100C00270F60A86841F81C0C0F68002FF4
:20F41000FCD004F13C0007F0DEFA2564206CC06840680078022808D14FF4004101E04FF408
:20F43000806104F1EC0007F0ABFAB0BD1C100440A00A00202DE9F041DFF8948006460C46E7
:20F4500036F07F0015D1002E3ED1224D243D686880471E49096831F81620144321F8164070
:20F47000A968884741461431086806F0A5FDBDE8F081042006F082FC071C25D04FF6FF704E
:20F4900038807C8007F01CFD41468C78A7F10C05FF2802D0C96A40184478FF2C06D13846A4
:20F4B00007F0C5FB06F0FEFEBDE8F081304607F049F801463A46FF20A872204605F01CFC5C
:20F4D00010B1384607F0B3FBBDE8F081842D002094190020D815002025483EB50078002877
:20F4F00043D042F20100694604F0D6F842F2050002A904F0D1F81D4D95F8540010B39DF8FF
:20F51000080000249DF80810009B2864642285F85440581A02FB00F1E96705F1780003F033
:20F5300011FD01A804F0D6FF124801992E300078B1FBF0F2451E4243891A01918D4214D90A
:20F55000204610E09DF8081064204843E86705F1780003F0F7FC288F401C288700242C6470
:20F57000012085F8540004F035FA3EBDD02900205D0F00208C2A00202DE9F041224C0646EF
:20F5900004F1580005780F46002D04BF0020011C1CD0204D1D49281D0B780068D3B91C4830
:20F5B0000568E06C07F016FB228FB0FBF5F1B0FBF5F3891889B203FB05F2236C3980801AF2
:20F5D000C018306085421CD8401B491C30603980BDE8F08180475FFA80F804F1780007F0DD
:20F5F000D1FB226C4FF47A73410001EBC001B1FBF3F0238F3060A9683B8080183060404638
:20F610008847BDE8F081C046D02900205D0F0020942A0020B4150020F8B50F46002302B9A3
:20F630000123DFF890C00021EFB13D6ADDB1C669CEB1FC68C768A74207D0DCF854110CF53E
:20F65000AA77A14214BFF968B968B4086FF05047A4EB9504641AA74225DDB4F1704F01DBBE
:20F67000002C20DD01210AB3D769FFB1066AEEB1D268C068824208D0DCF854310CF5AA7001
:20F69000934214BFC068806800E00020C0EB97006FF05042A0EB9600824204DDB0F1704F49
:20F6B00003DB002801DC0020F8BD012301EA0300F8BDC046A00A00202DE9F043254C0746E4
:20F6D000243C606AADF1240D00283ED0002F3CD0387A002839D004F0D3FB5FEA000834D0B6
:20F6F000062000250323A1468DF808002E46ADF80A30B5F5FA7F28DAD9F82400ADF80C50A7
:20F7100004AB02AA0469009392E803000A230022A047B0B9387A9DF81810814210D1022825
:20F7300004D1BDF810103A88914207D0032807D104A93846082206F033FB08B9284606E012
:20F75000761CB04505F10105D3DC4FF0FF3009B0BDE8F083F8110020F0B520480127F84290
:20F7700001D004F0A3F8204D204F214EBD4206D203CD0478A4003459401CA047F6E71D48F5
:20F79000002800D08047164D164FBD4202D210CDA047FAE7F0BD03251BE0416808300A1C83
:20F7B0002A400BD11A1C2A40AB4305D0046804300C600431043BF9D1131C05D00478013095
:20F7D0000C700131013BF9D1021C2A4001D0A84304300368002BE0D17047C046FFFFFFFFED
:20F7F000000000000000000088800100E88001004480010055C5011070B504466068254EED
:20F810004078ADF1480DC00921D3B4F842003546E63DB5F8BA10884219D11D480078A0B983
:20F8300095F8C40098B104F1280006F01FF970B9012000901C340194B5F8BA3005F1AA02FB
:20F8500003210620F7F7B6FE1FE006F019FE0BA80021182201F03FFC02A821460C900BA806
:20F87000FFF7E0F82C208DF82C000BA803F064FA3546503D287810B19DF83C0028B1052071
:20F890008DF82C000BA8FDF7F5FF12B070BDC04615150020860F002003B426482DE9F041AC
:20F8B000058806AF1446ADF1080D98464FF6FF70ADF800000222ADF802006946ADF804008F
:20F8D00044F40040ADF80600601986B2304602F053F8BDF80600022269466FF3DF30ADF8ED
:20F8F0000600304602F048F8A1102846CAB2414602F042F8387840F40040ADF80000788833
:20F91000ADF80200B88802226946ADF80400304602F032F8BDF80000022269466FF3DF30E9
:20F93000ADF80000304602F027F802B0BDE8F04102B070472A1C00202DE9F843002A8946EA
:20F9500007464CBF47F6FF75151C002F08BF002033D03888002808BF002403D02A4600F03E
:20F9700085FB0446281B002826DD388828B1291B484613A204F02EFB0419B868E0B1D7F865
:20F9900004802E1BB8F1000F0DD0404607F0DCF8401DB04207DC291B48460AA2434604F077
:20F9B00019FB04192E1B122E06DBBB68291B484606A204F00FFB04192046BDE8F883C04658
:20F9D0003A2000C0222573222C2000C06C696E652025643A20007047F8B5234D012001462E
:20F9F0002870F7F7E5F86FF00100204C1D4927690870381C28D0A1684268914203DA07F0B4
:20FA100051F927693846C8B105F0B4F87968884224BF2769381C11D200F050FF14E026694D
:20FA30007068002802D507F03DF92669304603F097FDB168307B88472769384620B105F0BF
:20FA500099F879688842EAD2094C606880470646FEF7B0F8A1683046884706F057FD002019
:20FA70002870F8BD951B0020A21B0020801B0020B4150020002A4AD05FEA000C8B071CD1C0
:20FA9000830722D1102A08D370B4103A78C978C0103AFBD270BC103238D0042A2CD3082AF1
:20FAB00005D30C2A24BF08C908C008C908C008C908C092072AD0920F22E00B780370491CE9
:20FAD000401C521E22D08B07F7D1C30714D18307D8D0121F12D308C903801B0C4380001DAC
:20FAF000121FF8D20AE008C903701B0A43701B0A83701B0AC370001D121FF4D2121D05D06D
:20FB10000B780370491C401C521EF9D160467047F8B507F06DFB234C0746D4F8C00010F42F
:20FB3000602F33D0D4F8C000400CC6B2700807D2B00803D2F00828BF022602E0012600E005
:20FB50000026751D002168B202F090FFD4F8C03006F111010120884023EA00013846C4F82B
:20FB7000C01007F041FBB00004F1A8010A18D7682FB1085800224FF000632946B8470A48FF
:20FB9000006830B9022004F015F902E0384607F02BFBD4F8C00020B104F59070002106F0F6
:20FBB000EFFEF8BDA00A00200C1004401CB51F4C04F1780005F07EFE04F15C0005F07AFE91
:20FBD00004F1940005F076FE0021882204F1340007F04FFA06F018FF05F0ACFF84F85A006C
:20FBF000134984F85B001348086001200DF1010184F8B30042F2040003F04EFD42F2050000
:20FC1000694603F049FD0C489DF80110A0666420414321660949C4F884109DF8001048438B
:20FC3000E0670748C4F8A0001CBDC046D0290020101700201151010011360100E9F40000FB
:20FC5000D56F0100D0B5244C04F124010F68002F3FD0002215280AD13B7D0126022B08D06D
:20FC7000032B06D0052B04D0042B02D000E03B7D0026984200D016B17B7E5B0905D23A4688
:20FC900057F80C7C002FE5D123E00846394604F0C5FDF88A2760000A03D397F91C0006F087
:20FCB0002BFF387D022818BF052802D1012006F0E3F92068407E30F07F0005D194F82F00EB
:20FCD000401E84F82F0004E094F82E00401E84F82E003846D0BDC046700D00202DE9F84366
:20FCF000234D884606464FF0FF3105F12400814607F05EFA00200CE0FF2909D02A688A4260
:20FD100004D905EB8101D1F894700FB1002627E0401CB8F1000F03D018F82010FE29EBD1C0
:20FD30000024346074600127B46011E0FF280ED005EB80000B787268C0F8946007FA03F088
:20FD5000104370600A680949304605F03DF8641CB8F1000F04D008EB84010878FE28E5D12C
:20FD7000484607F03DFA3046BDE8F883007FC76734260020B0B5456884682349607DA27D94
:20FD9000ADF1180D40F000400090207D0027FF2A41EA000001904FF0020002D0E27DFF2A4C
:20FDB00000D13FB1E37DA07D1943039140F0004002900420FE214DF8201005F1580069464E
:20FDD000FFF78CFF6866002808BF381C1AD0617D0F2205F02BFC686E217D102205F026FCAF
:20FDF000A17D3846FF2902D0E27DFF2A00D140B1686E112205F01AFC686EE17D122205F0A2
:20FE100015FC012006B0B0BD0000C0A03EB506F073FC0446204D2149286981422FD12049E7
:20FE300005F17000002207F003F90120287006F0B7FA00204FF6FF71B5F8C43068719942AD
:20FE500009D10220ADF80000684605F097FDBDF80800A5F8C400286C60B905F13C0007F0C6
:20FE7000FAF8031C06D003F021FE40B91846FFF78FFA04E005F1EC00022106F081FD04F052
:20FE9000804104F00200084305D005F1EC004FF0005106F075FD3EBDA00A00204D2D000062
:20FEB000A5BF000098B5244C0746A8B1401E0BD0401E2CD1204690F8402042F0080202F05B
:20FED000EF0280F8402022E094F84020204602F0E70242F01002F4E7214601F174021078A4
:20FEF00091F83C3000F0F000107003F0F000002281F83C0091F840308A6343F0080000F0D2
:20FF1000EF0081F84000F420413103F087FD002F08BF44F620600CD007F01EF84FF4FA67EF
:20FF30000A2244F6206390FBF2F15143401A07FB0030A06498BDC046D812002038B5054699
:20FF500095F83000032839D195F83A00032835D105F128044A202146F6F72EFF8A20214689
:20FF7000F7F70CFE6C686178207800EB0120ADF8000069465020F6F71FFFA41C6178207828
:20FF900000EB0120ADF8000069464B20F6F714FF8B206946F7F7F2FDA41CE1202146F6F73A
:20FFB0000BFF641C6178207800EB0120ADF8000069465320F6F700FF002000E0E820044922
:20FFD0002A24087028462C7002F0B6FE38BDC046252C00202DE9F8432020EFF3118780F3B1
:10FFF0001188214CA068012107F08EF84FF001090B
:020000040001F9
:200000004FF0000865692168A4F81C906A1A2168A4F81E80461B401A904227D387F3118819
:2000200040464519361A4846294607F071F8B042F7D92021EFF3118781F31188E18B01290F
:2000400003D14046294607F063F8B0F1FF3F06D0A169801B814238BF081C411901E0A06909
:20006000291807F051F8A4F820902560A4F81C8087F31188BDE8F883780100207FB50346AD
:200080001F480D4601881F480088144614A6984205DB32462146284603F0A4FF1DE09942A5
:2000A00006DB184606F080F80028F2D04268F1E715480088002808BF0CA2EBD00095002C29
:2000C00048BF47F6FF74114E0020114901946A46346802901846A047029800907FBDC0466C
:2000E0007B6D6F64756C652325647D007B6D6F64756C652D726F70653A25787D00C046C0D8
:20010000120C0000A60C00008E140000C40C00000155010090B50C46214A0178575CADF17A
:200120001C0D0B2F8DF8007035D0002F36D00C2F04D0112F29D106F082FD26E01A2C22D031
:2001400090F899100190C7688DF80210038A0297C28AADF80C30510905D21249827EC8313F
:200160000978891A00E000218DF80E10877F8DF8107090F91F308DF81130826A0592417FCB
:200180008DF80F1001E0002001908DF801406846FDF778FB02E04470FDF734FA07B090BD92
:2001A00094030000A00E00202DE9F04107467868BE68044600F5847005F0D6FF30681C4946
:2001C00080690968C0F3C00008BB07F019F8194D8046287820B1022004F018FE0020287006
:2001E000404607F009F83168134D886B20F020008863286820F480702860606A216A091AE6
:2002000021622369626A38469847BDE8F0814FF4FA70B0FBF1F1012998BF012104F58474C2
:20022000204606F0A5FF204606F0DEFFBDE8F081B00C0000892D0020301000402DE9F04116
:2002400080461E4800680D46416927208847012404FA05F61A4DC5F80064C5F87C470327A7
:20026000C5F8807717480460C5F88477D5F80404012818BFC5F80444C5F8FC63124804609B
:20028000C5F800801023AB60204606F0B5FED5F88C074008F8D3D5F88C17204611F0404FFB
:2002A00009D1C5F884770021C5F8FC16D5F80024164218BF081CBDE8F081C046B00100109B
:2002C0000440024000E04842000048422248F8B50C460178012904D0417A012918BF0120E7
:2002E00034D190F8C710CA080AD390F8C620A24206D101F0FB0180F8C710002780F8C670B1
:2003000006F07EFF074606F063FF06460121204602F0B4FB0E48210201F47F41084305F0E2
:2003200035FB0C4A1168054604F10C030120984081433046116006F047FF384606F05CFFC0
:2003400005F0FF05012D0CBF81200220F8BDC0460100080408100440A00A002070B505468A
:20036000204C2878002836D16078012833D0281DFFF7AAF9B0F1FF3F2DD1298AC8132AD0FB
:2003800001F00F010F2926D12046018F4FF6FF728A4204BFE9890187A97C80F83A10AE88DB
:2003A0008687298A01F00F020F2A05D080F85020C1F3031180F8511090F850100F290AD1E9
:2003C000012141700848064606F08CFC012802D1304606F04CFE6C34216809B1284688475E
:2003E00070BDC04670140020901200207CB515460E46044600E004192046694604F024FE12
:2004000000282ED014F8021F8E42F4D1491E04F1010420D0491E12D0491E08D0491E18BFDD
:20042000622029D102281CD12078287023E0032817D114F8010B2870207868701BE0072899
:200440000FD161782078A41C40EA0120288020682E1D30600FE0052803D1207806282870E7
:2004600001DD67207CBD2D1D0020641C2860A678AE702088288000207CBD70472DE9F04189
:200480001E4615460F46044606F0A2FE8046384605F02CF9071C04D097F8270030F07F00BE
:2004A00003D1404606F090FE28E097F8270010F00F0F1BD113487968884202D07968A166D6
:2004C000786004F1600080E86000404606F07CFE04F140004FF0FF3106F072FE04F17007BB
:2004E0000020A06697E80300BDE8F081404606F06BFE97F8270010F00F0FFAD10220002177
:20050000BDE8F081F520010070B506467468B568606E05F068FE29681C488A6B10408863F7
:20052000304600F037F8304601F044FC2968C86A20F01000C862296815480A6B1040086354
:200540006868FDF7E9FF04F1800006F0F9FD04F19C0006F0F9FDA07818B904F1D00006F06D
:20056000FBFD607818B904F1EC0006F0F5FD04F5847006F0EDFD06F043FE0021217006F065
:200580003BFE04F16C0005F04FFD70BD0DF8FFFFFEFCFFFF2DE9F04106467568B46806F0D6
:2005A0002FFEA96A39B921688969090903D206F023FEBDE8F0810027AF6206F01DFEA17D13
:2005C0003846FF2902D0E17DFF2900D118B12846214600F0B1FE2168886B20F02000886378
:2005E0000D49086820F48070086006F009FE0B4C8046207818B1022004F008FC2770404617
:2006000006F0FAFD686A296A091A29622B696A6A30469847BDE8F08130100040892D0020B1
:2006200038B50C4644220546002100F05CFD04F12801284606F0B0F804F1320105F10A000E
:2006400006F0AAF8E06B6861B4F840002883B4F842006883B4F84400A88394F84600A87772
:2006600094F84700E87794F9480085F8200094F8490085F82100B4F850006884E06C686265
:20068000A07B85F8280094F8520085F82900606D0B2204F11C01E86205F13000FFF7F2F9B9
:2006A0002089A5F840006068E86338BD70B51E4DAC68064606F004F84FF47A71001B4843F6
:2006C000030C05F04FF92969401A48BF404240F6B8319B19994210D306280EDAE9688C4293
:2006E0000BD8286848B1114A091B51438A0C02EB1141884288BF011C08E00D494868400842
:200700000ED208687D2100F0FF004143C82905D3B1F57A6F88BF4FF47A6103E0C82101E00E
:200720004FF4FA61084670BD442D002040420F00AC3F00502DE9F8431F4C00264FF0010819
:200740004FF002093746A51E15F8020F03280FD0022824D168786368022820D0304606F097
:20076000F9FB0146384606F08FFB85F8019011E0304606F0EFFB014663686878012805D0FB
:20078000384606F081FB85F8018003E0404606F07BFB6F700246C9B2184604F04BF9761CCC
:2007A000022ED1DB05F02EF918B104F1200006F05CFCBDE8F883C046D81800207CB504208A
:2007C00004F010FF022818D0032816D019480068C0F38150032814BF41F288324FF47A728C
:2007E0001649174C09684C342046B2FBF1F106F0BFFC204606F0F8FC7CBD4FF08056D6F834
:20080000A4010D4D446800214FF040521C23032000902846A047D6F8A40100214FF40072AB
:2008200009230126446800962846A047022004F0EDFA7CBDB43F005000A00C40B00C0000AD
:20084000C00F002003B42048F0B505AF3E787D880088BF88ADF10C0D001F84B2082C2CDB60
:20086000201F6946082280B204F082FCBDF8000086420FD1BDF8020085420BD1BDF804004C
:20088000874207D1BDF806006FF3DF30241A241FA0B213E0BDF80600C10BCB0309D100F1A5
:2008A00008018C4202DA06F005FA06E0241A083C00E0241FA4B2082CD2DA002003B0BDE857
:2008C000F04002B07047C0462A1C0020F8B51E4C002528462268A168256190420CD05268E8
:2008E000914209DD04F04EF90146206842689142C8BF41602061A168676837B118B14268DC
:200900007B689A4201DD38462061C8B14068814216DD0F4D044605F108000068A04201D89D
:2009200006F0C8F9094E706880470746EC60204600F062FEFDF746F9B16838468847F8BD6D
:2009400005F012FA2561F8BD801B0020B4150020241B00202DE9F8431C481F4D07786868E8
:20096000804781461A4883680026344680469C4212D013F8020C874208D134B163B1384644
:200980004FF40041FEF75EFD13E01C4604B91E4653F80C3C002BECD15FB9686880470D498D
:2009A000096831F817206FF3DF3221F81720A96888472CB108F108002146324603F036FFDE
:2009C000A968484688472046BDE8F8833C16002094190020842D0020B41500202DE9F041E3
:2009E000804600271A481D4D07701A481A4E077096F83800D8B1F36F2C68C3B1207D3528D3
:200A000009D16068218900F02DF860680088000901D303F0EDFEF16F4046884710480078E5
:200A200001280BD038460146F6F7CAF806E002F0D3FE01F08FFA4046F8F76CFD286810B1EC
:200A4000007D352801D005F013FFBDE8F081C0468C2D0020942D002014150020700D002028
:200A6000A21B00200829C8B50BDA00293BD00278491E92FAA2F24FEA226200F8012BF6D129
:200A8000C8BD464206F00306891B37188AB2361802F00301864209D9361A0378761E93FA41
:200AA000A3F34FEA236300F8013BF6D122F00302D71987420AD93A1AD21C96100268761E4D
:200AC00092FAA2F212BA40F8042BF7D1CF19874209D93F1A01787F1E91FAA1F14FEA216121
:200AE00000F8011BF6D1C8BDF8B50546012003F043FE1D4C04F1140002F03AFD04F1240095
:200B000002F036FD69684A78087800EB0220ADF800008F7804F114066FB953206946F6F79E
:200B200053F905F128014A20F6F74EF905F128018A20F7F72BF806F1200005F11C010B227B
:200B400005F0D2FEBDF80010384604F0C7F994F83F00800803D36878002105F04DFE00204F
:200B600084F83F00F8BDC046942B00201C491B4898B5FF220F7890F83B301A4980F838203D
:200B8000012B15D091F8A10091F8C010884224D015480024047006F04AFA01F06FFC13481D
:200BA0000078012819D020460146F6F709F898BD002380F83B3087B18DF8032091F8D70075
:200BC0008DF8000091F8E6708DF8017091F8E7408DF80240684606F0D4F998BD1C19002029
:200BE0009F0D0020A00E0020912D0020A21B002070B50025ADF1200D07A8ADF81C5006F0D5
:200C000039F81B4CBDF81C10208F884227D194F85300032811D004280DD0022810D104AE39
:200C20006946304603F0C2FBE06820B1026812B1304669469047042000E0032004F0EAF99F
:200C4000A06D04F03DFB5220294605F0F1FC4FF47A7004F04DFB284604F062FB05E0032068
:200C600005F0A2FF052004F0D5F908B070BDC046701400202DE9B84106F0C2FA1C4C1B4DD7
:200C8000804604F1E000007848B92C46A168022088470746102003F083F90FB31DE001F038
:200CA0008FFA70B9134800683221B1FBF0F101B901213034204606F05BFA204606F094FA04
:200CC0000EE0002084F8E0002C46A168022088470746102003F064F917B1A16803208847AE
:200CE000404606F089FABDE8B881C046240C0000B80F0020B00C00001D491E482DE9F0412B
:200D0000352751F8048B51F804EB51F804CB51F8046B51F8045B40F8048B51F8044B40F858
:200D200004EB51F8043B40F804CB51F8042B40F8046B40F8045B40F8044B40F8043B7F1EE4
:200D400040F8042BDDD151F8045B51F8044B40F8045B51F8043B40F8044B51F8042B40F8E8
:200D6000043B40F8042B09680160BDE8F081C046B874010000C0002138B505461B491D4CCC
:200D80002878E0B96878012815D0022809D0032826D10846002181704021083005F040FBDE
:200DA0001EE004F13A000078FF280CBF0120022005F0FAFE14E004F108002021EEE76A7883
:200DC000032A08BFEA2804D0012A09D141F2883000E0074891F8542081F8552004F0A0FAA1
:200DE0007434216809B12846884738BD70140020E09304007014002070B51B4C054610220E
:200E0000ADF1200D04F171016846FEF73BFE0026049509208DF8146004F10D018DF8160045
:200E200001258DF815500A680DF1170002604A684260097A01720D496A4618200EF0D0F96A
:200E40000B4918208922631D0EF0CAF97120314605F028FFD520214605F024FF5D20294696
:200E600005F0E6FB08B070BDE807000021AD00008D7B00002DE9F0431C4E044600271D466B
:200E80008846A2EB0409ADF1140DC6F8B071012006F0B2F83068C00FF9D3306A0090706A54
:200EA0000190B06A0290F06A039044B128462346694611F8012B5B1E00F8012BF9D10320CE
:200EC000C6F838026CB108EB09016D1E491E11F8010F15F8012F904218BF042002D1641E96
:200EE000F5D1384605B0BDE8F083C046504502401849B0B50546164C0F7820781FBB164A38
:200F00008100B2FBF1F1A94202D205F0D3FE20786168154F800005FB0014A7F10C000068D7
:200F2000C06B8047211AA1F54871090806D30B4A011B891A090828BF00F5487408482146D7
:200F4000FBF720FEB0BD074901200870B0BDC046241B0020A31B0020FFF6C2FF00093D007F
:200F6000F9DE0000932D00202C170020F8B51A4E1A4D0120002414EA030730704FF00200AD
:200F800000EA020008BF00280CD14FF0E04004EA0201184008BF002904D11249888D401C60
:200FA000888503E095F90000401E287005F09AFA05F05EFC0A48047095F9000030B195F922
:200FC0000000002806DC05F075FE03E020460146F5F7F6FD3470F8BDA21B00209E1B002021
:200FE000971B0020241A00202DE918410446DFF870802078E02828D1404642788178012A44
:201000000AD049B990F85220012A05D190F8540001281AD001200CE0104BB3F86620521C03
:20102000A3F8662041B9491CC9B2817000234370022005F0B9FD08E0002004F041F90320C8
:2010400005F0B2FD052003F0E5FF40467C30016809B120468847BDE81881C046B813002037
:2010600070140020F8B500680E4617464FF0FF310446483006F0A4F84FF0FF35092E08D0C1
:20108000217A0120B040084211D108433546207210E0227A0721012303FA01F0104202D036
:2010A000491EF9D503E0227A0D4610432072B5F1FF3F0ED06FB129463846FFF7BFF840B1D7
:2010C000217A0120A8404FF0FF3580F0FF000840207204F1480006F08BF82846F8BD0022B5
:2010E00013460A46194671B510F0030F0BD0002A82BF00F8011BB2F1010210F0030FF6D1D7
:20110000002A08BF71BD11F0FF0141EA0121042A18D341EA0141082A0FD30E46102A08D35F
:201120000C460D46B2F10F0312F00F0272C0103BFCD812F0080F18BF42C012F0040F18BF13
:2011400040F8041B12F0020F18BF20F8021B12F0010F18BF017071BDF8B5054606F050F85B
:201160001A4C0126074605F19C00E67004F0FCFF2078012811D094F8880170B1B4F95000E9
:20118000B4F95210884208D1384606F035F80720FDF7BAFF06F034F80746B4F95200B4F90D
:2011A0005010884218BF85F8C2600AD105F1780004F0DAFF304602F005FEE17920780843D1
:2011C000E071384606F018F8F8BDC046A00A002038B51B4D95F8A1000F2824D0194C3B3C2B
:2011E00094F83810FF291ED094F83A0068B102290BD103F0C7FC216B0F4C95F89820401AE3
:201200002178083101FB12010BE003F0BBFC616B0A4B95F8C020081A1988401A34F812105F
:20122000411A002901D5002038BD4FF6FF708842C8BF88B238BDC046C51900209C0D00203E
:20124000A00E0020571900201C4938B591F85C3001EBE304657F012203F0070302FA03F300
:2012600083F0FF032B4063778B7E01F11800032B18D091F86030012B10D0022B08D0B1F8B8
:2012800056108A409102A1EB821101F570710EE0B1F856209101A1EB820108E0B1F85610F0
:2012A0008A4001E004490A789102A1EB82111C3005F042F938BDC046690F00200C2C00209B
:2012C00000B500212022ADF1240D6846FFF70BFF1848018FADF8181090F83A108DF80B104A
:2012E000808FADF80E0002218DF8161009208DF80C0001218DF81F1003208DF80D000020F9
:201300008DF808008DF81B006A468DF81A0007498DF81D0018200DF063FF0549B1F84C0085
:20132000401CA1F84C0009B000BDC0462D6F0100B81300207014002038B50C4621680546B1
:20134000886B20F020008863686E217D012202F091FB686E217D012203F06CFB686E217D05
:20136000002204F06BF9686EA17D002204F066F9A878012806D005F1D0004FF0FF3105F041
:201380001FFF03E0216888690009FCD2686E217D102204F053F9A17D0020FF2902D0E27D7E
:2013A000FF2A00D118B1686E112204F047F938BD2DE9F84F8346894617467120114604F00A
:2013C000BDFA81206946F9F7BBF84FF0F308002507E0B8F1000F23D038686D1CEDB22C304E
:2013E00038609DF80000A8421ADD3868066890F804A0002402E0641C0A36E4B2A245E8DD9D
:20140000737A002B0CBF052009208145F3D14A463046594604F058FE0128ECD14FF00008F5
:201420004046BDE8F88FFEE71A487CB5007880B342F2050001A902F037F942F201006946EE
:2014400002F032F9144C9DF80400216C88420BD80098884203D805F0FAFD01250DE00022DE
:20146000012584F8542004E001259DF8040084F85450401A64214143E16704F1340606F1C2
:20148000440004F01FFA06F1440001F063FD84F858507CBD5D0F0020D0290020F8B50B466F
:2014A0001A4991F831708D6B4C7A6430C2B25FB100206D1F6D1DEE7816B12E79B24207D0F4
:2014C0007F1E00F10100F5D1641CE0B2487204E0FF281CBF0021197016D10120187091F842
:2014E00030704C6B4B7A5FB10020203C2034A67F16B1E57FAA4207D07F1E00F10100F5D188
:201500005B1CD8B24872FF20F8BDC046CC10002038B5054601201A4C68712879B0B90EF09A
:2015200034FA2178002904BF6FF00704051C15D0491EC9B2217039B90EF051FA606803F01F
:20154000F7FF0020687118E0054613E00EF01DFA05462078FF2805D16FF0060428460EF09C
:201560003EFA0BE0401CC0B20128207002D1606803F0F5FF28460EF032FA0024204638BD28
:20158000B81B002070B51B4C06460E220D4604F12C00FEF777FA687B20B9022020776B880E
:2015A000A38208E003202B1D20771A6804F114010A6058684860606A03F09AFE3046294684
:2015C000FAF782FE207801280BD0687B48B9288869882A1D01F09AF9011C02D001A005F029
:2015E0000EFD70BD41757468204572726F723A20307800C0B8130020154998B50F7817BB46
:20160000144A1178144F52688B00890000FB0324B7FBF1F1814201D205F04CFB1148006869
:20162000C06B8047211AA1F54871090806D30B4A011B891A090828BF00F548740A482146CE
:20164000FBF7A0FA98BD06490120087098BDC046A31B0020241B0020FFF6C2FF00093D002D
:20166000932D002020170020E9F9000038B517481749007818B90846007828B906E0084681
:20168000007830F07F0001D005F014FB114D68688047114C0C3C2178A278914207D10F4A0D
:2016A000A9681278D20803D28847012038BDA968884705F0BCFCA078FDF7CAFA012804BFB2
:2016C000A078207005F0D4F838BDC0464C150020942D0020B4150020D0190020912D002074
:2016E0002DE9F84380461848077817B9174D287810B90120BDE8F883154E7068804781464D
:2017000068880124B8F1000F0ED1214603464FF6FF72B9404A40104068807BB170B9002087
:2017200004F0F8F8044609E018B9204604F0F2F868882146B940084380B26880B168484621
:2017400088472046BDE8F8833C1600209C0A0020B41500202DE9F8438146EFF31188202040
:2017600080F31188174D154C134F012605F11C000660A4F114000660F86A016A14208847B8
:20178000D9F81000810C14BF000C04202060386802682321002090470948066054F8180CEC
:2017A00020F4C02040F4803044F8180C2E6088F31188BDE8F883C046840100101820094013
:2017C000800224430000244330B504460D4642F20900ADF12C0D09A901F066FF9DF8240062
:2017E00008B342F20B000DF10E0101F05DFF00230094BDF80E00029300040190684602F051
:2018000035FC044604A942F2030001F04DFF04F099F9024604A9B4FBF5F06843241AE0B2A2
:2018200002F072F806E042F20D0003A901F03CFF9DF80C000BB030BD2DE9F843194D064601
:2018400028780C469846012805D0687A012818BF6FF0010024D162600A20208001F0F8FA14
:20186000071C1CD4A77005F0CBFC8146204604F08DF80446484605F0BFFC04F0FF04012C30
:2018800006D03846012101F0F9F86FF0010706E005EB8705A83545F8088C45F8146C38463E
:2018A000BDE8F883A00A0020F0B50546194C2878ADF11C0DE9281CD028BB002694F852009E
:2018C00084F8566002281ED104AF6946384602F06DFD5220314604F0ABFE2046C06820B19C
:2018E000026812B1384669469047042003F092FB09E094F85600401C84F85600C0B203287D
:2019000001D104F093F88C34216809B12846884707B0F0BD701400202DE9F041074617483B
:20192000174CC01F06786068804780461549A268087886281CD1104D05F12A021088401C9C
:2019400010808720087005F0B7FAA16840468847082004F0F7F9E879B04207D127B900209D
:20196000FFF73CF8BDE8F0811B20F9E7E920F7E740469047BDE8F081241A0020F02C002018
:20198000B4150020942D00202DE9FC4716460C46054604F089FA164F81467868804780461B
:2019A00003F082FA8246B2002146484605F0B4FA504604F051FD02E02D1D241DADB230468C
:2019C000411ECEB278B128466946042203F0D0FB68462146042204F0EBF90028ECD00549B9
:2019E000012048700870B96840468847BDE8FC87B4150020281C00202DE9F8430024002B0B
:201A000016460F468046254606D5002FC3F1000302D57F42761E2D2599463846494602F0C7
:201A2000E5FC0CA0405CB7FBF9F7002F04F1010408F8010DF1D1A64205DD3021301B401E1E
:201A400008F8011DFBD10DB108F8015D4046BDE8F883C04630313233343536373839616204
:201A6000636465660000704730B5401E4FF00004ADF12C0D0AD0401E04D0401E20D1F7F777
:201A8000B1FB1DE000F026F8044619E001A821462422082305F074FB06940D4DADF814407A
:201AA00009490794012201AB05F1780005F064FB064A23462C2105F19C00009305F070FB1D
:201AC00020460BB030BDC046C5290100B14C0000B80F002098B5164C94F8E100002710B913
:201AE0001448007860B105F08BFB94F8E310002906BF012184F8E310012705F07DFB0FB133
:201B0000002098BD022003F0C3FB0E20FCF7EEFF094A106848B909494020C8600860012739
:201B2000D761002084F8E20098BD012098BDC046B80F0020320C000004800C402C500C4061
:201B4000F8B516460C46054605F05AFB07461CB3641E1AD0641E15D0641E0FD0601E0BD1EB
:201B6000306828B1012807D1802002F02BF915E0802004F01DFC11E0032410E030780A4998
:201B800008700BE03088688208E00120EE68687406F16000E86001E0306828608324384640
:201BA00005F02AFB2046F8BD080B002038B5042903462BDA05F0CEF90546084605F064F9AE
:201BC000134C5B0002460229195503EB040012BF0329002141706068E9B202F02BFF03F037
:201BE00011FF50B904F12000044605F07BF801280CD1204605F03BFA38BD04F1200004461B
:201C000005F070F810B9204605F02FFA38BDC046D81800202DE9F843174C04F124010868D1
:201C20008846074628B300261D25387D35281BD140463946324602F0F9FD787E30F07F004E
:201C400005D194F82F00401E84F82F0004E094F82E00401E84F82E007D7057F80C9C3846E2
:201C600000F076FB4F4602E03E4657F80C7C002FDBD1BDE8F883C046700D002038B5164D43
:201C800095F8B41001290FD003280BD013480078812804DB8428B8BF49F6404419DB4FF46C
:201CA000FA5416E0002414E0032844F6206410D00B48006890F8690058B105F055F90A22DB
:201CC0004FF4FA6390FBF2F15143401A58432418A4B2A5F8B64038BDD0290020870F002084
:201CE000700D0020164880B507683FB315498B6803EA5300C00E21D2134A106880081DD2B5
:201D0000486880081AD21068096810F0050F4FEA114101F0F00101F5E0710AD1B9420DD239
:201D2000190F38BF40F00100D90E38BF40F0040003E0B94202D920F00500106080BDC046C0
:201D400028500940AC3F0050000009402DE9F04180461748243007680E46ADF1300DBFB170
:201D60003869A8B1B8F1000F12D08EB106208DF828000125ADF82A500022ADF82C2002ACB7
:201D800000943C690AAB93E803001A23A04708B100200AE002A940460C22FDF773FE05A97E
:201DA00030460E22FDF76EFE28460CB0BDE8F081D4110020F8B50646B06801687568886B8E
:201DC00020F4FA6088631349086820F40070086005F016FA104C0746207820B1022003F0C6
:201DE00015F800202070384605F006FA05F008FAA96B11B905F000FAF8BD0021A96305F018
:201E0000FBF9686B296BEB68091A29636A6B30469847F8BD30100040882D0020F8B58446BA
:201E200040F6FF741CF8013B002210E0481B401E10F8015B7F1E01F8015BF9D103E01CF8BF
:201E4000010B01F8010B521C5B08082AEADA5808F5D21CF8010B1CF8015B05F00F07FF1CCD
:201E6000C5F30315122F45EA001508D11CF8016B300A24BF1CF8010B60F3DF16F719AC4231
:201E8000D4D1F8BDB0B5184C05460F46101C28D00DE03868E06397F82700394640F0040022
:201EA00087F8270004F14C0002F0CAFFE76BD7B1F8688542EDD014E0386888B13868C0682D
:201EC00085420DD139680868386091F8270040F0040081F8270004F14C0002F0B1FF00E06D
:201EE0003F68002FE8D1B0BDA00A0020084610B500F0005100F00400084321D0012003F084
:201F000071FB114C012813D00E4801683220B0FBF1F2012A8CBFB0FBF1F101212046A0F131
:201F20002404204605F024F9204605F05DF910BD064804F06DFF06492046D8380839086067
:201F400010BDC046B00C00008C0B00204D2D0000081004409EB5144C606880472146134C5D
:201F60002289E38893421CD0114B1F78CFB9114B89681F7837F07F0714D1E2808847102731
:201F8000E088ADF8007001A9ADF8040009880DF10203198008480068426AE0686946904712
:201FA0009EBD896888479EBDB4150020C4190020922D0020942D0020201700202DE9F8435D
:201FC000DFF85880044608EB440000F11805008B894603F0DBFE074611480678AFB12A8867
:201FE0003846002105F04DF800253C7041467D700A5D381D494604F077FC3046394600F02C
:2020000055FC40B92846BDE8F8838DF8004068461A21FEF77FF81A20BDE8F88388030000E9
:202020003C16002010B5164A144C92F83D0094F8401048B91348006860B9012082F83D0051
:20204000202004F067FE05E0481CC0B2042884F840000DD00C49A1310A784FF4707304F1A3
:20206000200003FA02F101F2636104F065FA10BD202002F081FBFCF70BFB10BD782C002041
:202080001C190020700D0020A00E002010B5044600212822ADF1280D6846FFF724F8134917
:2020A00011226846FDF7EEFC05208DF812008DF8114000218DF8151001208DF816100B220B
:2020C0008DF81700FF208DF8180009208DF8130003208DF814000DF11900FFF704F80449D5
:2020E00018206A460DF07CF80AB010BDFF07000009E800002DE998430446A76E9946904604
:2021000007B1B8470020022100EA090701EA0801002F08BF002917D104F1600106C909EAB8
:20212000020708EA0101002F08BF00290CD161680978022910D100EA09000821002801EA21
:20214000080108BF002907D004F1700080E8000304F1400005F04CF8BDE89883C8B50146ED
:20216000164AC87AB8B992F83170906B2FB3401F401DC6781EB1CA7F03799A4202D07F1E6B
:20218000F6D1C8BD8A7FC270CA880280CA7F0271097B8170C8BD92F83070506B6FB12038D1
:2021A0002030867F3EB1CA7FC37F9A4203D12022FDF768FCC8BD7F1EF2D1C8BDCC100020A0
:2021C00038B5012003F00EFA012820D0114DD5F82401C4681048342101220023A04700285F
:2021E00008BF002014D0286803F0F8FB04F068FA0B4A0A4D93681168D060C01AA1EB910100
:2022000005FB00F3180C884228BF011C1160012038BDC0468000001000A00C4040420F003F
:20222000442D002098B50446207B00F00F00022824D100F0B9FEA168081A8108114800F118
:202240000C021768002F14BFFB6840F6C41303F57A728A4212D20A4A12686FF050448C425C
:202260000CD3C91AB1FBF2F3012B8CBFB1FBF2F10121C83004F07CFF012098BD002098BD91
:20228000B00C0000A00A0020001F06B480B290B5082803AFADF10C0D22DB3A78B0F5805F9C
:2022A0001EDA00F18851091F0C686B461C6049685960BDF800108A420BD17988BDF80230D4
:2022C000994206D1B988BDF80430994208BF012007D0BDF80610401A083880B20828DDDA0A
:2022E000002003B0BDE8904002B0704710B50446012002F041FA208900280CBFEB20002009
:202300001249607091F83F00C20824BF20F0040081F83F00820809D2400813D32B202070E3
:20232000EB236370204600F00FFD0BE091F83F0000F0FD0081F83F00217C6078C1F30011C8
:2023400004F05AFA204604F0DDFC10BD942B002080B501460A7D012A05D0152A03D0252AF2
:2023600018BF352A02D1087E000919D3087EC3091BD2012A18BF152A01D1000909D24F78DC
:202380001B2F04D0094807B10E30805C02E0232000E0312008700648007800F087FA80BDBA
:2023A0004A7808461146FDF7B5FE80BD870800003C16002030B5174C054605F12801ADF181
:2023C000140D04F1AA0003F0FFF908B3EF2309208DF801306B688DF800005A781978181DB6
:2023E00001EB0221ADF802102A890178082A8DF8041014BF94F8E600C07805F11C018DF80B
:2024000005000DF1070004F015FE6846FBF73AFA05B030BDA00E002010B504460320ADF197
:20242000180D04F128018DF8020000208DF8030001A804F002FE6068007804F11C018DF8B6
:202440000C000DF10D0004F0F5FD04F1280003F015FB58B14FF6FF7453206946ADF8004097
:20246000F4F7B2FC044920460A3108800DF10200FBF708FA06B010BD4A0F002070B5164DD5
:20248000286808B104F00CFD144C606880470C3DE9690A68002616710968E961A1688847BA
:2024A0000A4A0B49107810B90846007860B1167008460670FCF77CFE06480078012803D0D3
:2024C00030460146F4F77CFB70BDC046902D0020922D0020A21B0020F02C0020B4150020EC
:2024E000F8B50025114C1348A5604FF4700665600068E660C06B80470D49C0F1FF30086091
:202500000D48C76865700FB90C49C1600C480570012001F00BFE08B104F0CCFB304601F065
:2025200081F9E068FFF768F8F8BDC046241B0020083004402017002094190020212A01007D
:20254000932D002070B5164604460D1C08BF052426D034F07F0001D003F0ACFE002C18BFAD
:20256000032407D155F80C0C18B915F8020CFF2804D00524284604F062FB11E0012E0948B7
:2025800005F8024C03D0294602F010FD02E0294603F0AAFD20464FF40041FCF753FF002471
:2025A000204670BD9C19002030B50446606800252062ADF1140DA5657820A4F84C0094F840
:2025C0002C0025650F2807D004F12C0120460122F7F736F908B116E0284694F83C10FF2952
:2025E00001D1A16D21B104F13C012046FBF7EAFC48B92B4601208DF80C30032101AA009006
:202600002046F0F7B9FF05B030BD70472DE9FC41144C154F06468846700809D320684568A2
:20262000002101220B461FFA88F000903846A847B00809D3206845680021022201231FFA2C
:2026400088F000903846A847F00809D320681FFA88F600210C220223446800963846A047F7
:20266000BDE8FC81A401001000A00C400246F8B5084611464C68203821D0401E1CD0401E58
:2026800018BF6FF001001ED18D6804F0B9FD0E4E07463068016928688847B0F1FF3FF8D1C3
:2026A0000025A564606C401EE06425653846A56304F0A2FD2846F8BD0021084601E0012146
:2026C000002084F82D10F8BDD0010010012898B523D1012002F086FF01281ED004F008F87E
:2026E000114C012104F1D800017004F0B5FB800915D20C4800683222B2FBF0F707B90F4650
:20270000083C3034204603F02FFD2046394604F02FFD204604F068FD01E002F043FB002097
:2027200098BDC046B00C0000C00F0020F8B51549154A134D36395B320B681778E91C097845
:20274000002F0CBF1C695C6901EB810164182679002101E0491CC9B28E42D8BF4FF6FF70AF
:202760000DDD23680A4602EB42029B1893F900209042EFD1B3F801002881B3F80100F8BDBC
:20278000C4190020521700205A0F002038B5154C04F1180005461C3000F0EAFE03F0AEFAC5
:2027A000042003F0CFFAA07E032801D1607EA0B105F14501E120F4F707FB05F14601E72081
:2027C000F4F702FB084894F85F100078884204D005F14701E820F4F7F7FA2846FBF752F8E4
:2027E00038BDC0460C2C0020870F00202DE9B841DFF85080144CFC224146AC3CAC392046E2
:20280000FDF740F9002102220B46181903278D3000F8031F41707F1E8170F9D1521E03F156
:202820000903F2D104F1AC05032728464146182204F05AF818357F1EF7D10220A070BDE8FB
:20284000B881C046D0050000F027002038B50120124C114D94F8A11085F83D000F2917D04D
:202860000F490870202004F055FA94F8A1200E490C4835F81220886201F1200091F84010D9
:20288000491C5143490001F2A32103F01FF938BD02F03EFB38BDC0461C190020A00E0020F6
:2028A00014150020B1ED0000782C002070B502460D4632F07F0004D110460022FFF742FE89
:2028C00070BD04F005FB104908398C78A5F10C06FF2802D0C96A40184478FF2C02D103F060
:2028E000E9FC0DE0104603F035FE01462A46FF20B072204602F008FA20B1284604F09FF96D
:20290000012070BD002070BD9C19002000B5ADF1240DADF80000ADF80210116801A80160E4
:2029200051684160002002460D490690887D8DF80C200D318DF80D000B680DF10E00036081
:202940004B684360097A017218208DF81C2005498DF81D206A460CF043FCC0B209B000BD4F
:20296000E8070000D957000098B5154B1B1D18680004070C21D002F0F5FF104991F90720DB
:20298000824205DD10F1800FB8BF6FF07F00C8718C88BC4210D80A68D3F8D40F801A801C23
:2029A0001F2888BF1F203F1B4008C7404FF6FF70E719B84238BF071C8F8098BD782D0020B0
:2029C0003010094008B51348134A14490078801E0A2807D8DFE800F018141006141006143E
:2029E000100609C004F0D0FB11E010688008FCD250688008FCD20AE008688008FCD306E0D5
:202A000008688008FCD202E010688008FCD3F6F7E9FB08BD9C10002034600C4038600C4019
:202A200070B5134C6068804712490025064648784D70A168820808D2C00816D330468847D7
:202A400028460146F4F7BCF870BD304688470A480078012803D001202946F4F7B1F86068FE
:202A600080470646FBF7AEF8A1683046884770BDB4150020241B0020A21B0020B0B50F4651
:202A8000044604F0BDFB05461148EC3890F8C710C90803D390F8C610A14215D0B0F8C430B0
:202AA000012101FA04F21A430A4BA0F8C420181D026804F10C0399408A430260006818B9F1
:202AC00017B1022001F07EF9284604F095FBB0BD8C0B0020081004401549096821280ADC34
:202AE000212819D00C380FD00D380FD0001F0FD0C01E0FD01AE0253810D0001F10D0401E0E
:202B000010D0401E10D011E0086870474868704788687047C86870470869704748697047FA
:202B200088697047C8697047086A704700207047F0010020F8B50646B08815460F46FDF71F
:202B40009DFA0446002D02D4281B0A2806DB3368291B38460BA201F045FA0419B08978B182
:202B6000002D06D4B06803F0F7FF291B401D884206DCB368291B384603A201F033FA041943
:202B80002046F8BD257000C02827257327290000F8B50746C81D01F00705C610002F4FF06E
:202BA000010000FA05F0A0F1010C14BF0029002019D00020BEB17F1E33460246941B17F8D7
:202BC000011FB4F1FF3F08D10DB10CEA010104E001F1FF04401C2140C0B20029F8D15B1EF0
:202BE00002F10102EAD1F8BD70B5F1F7EDF9124D68688047064603F02FFE104C94F9D6005B
:202C000003F082FF02F09EFD03F074FF03F018FE03F00AFEA9683046884794F8D70000F0A0
:202C20007FFC04F1BD015220F4F7CEF804F03EF908B9FFF755FC70BDB4150020A00E00202C
:202C400038B50C4620B141680122A240114201D1022038BD914341600E480025231800EB64
:202C60008401C1F8945003F140010978FF291ABF406850F8211044F020410548FAF732FA5B
:202C800020464FF0FF3103F05BFB284638BDC046007FC767342600201248134908B54FF4D0
:202CA0002C72FCF7EFFE4FF00451002081F89003012081F87903022081F87503032081F811
:202CC0007703042081F8AE03052081F8AB03062081F88103072081F84D030448C1F8C00305
:202CE00008BDC0461C04002108720100CD05002198B5124CE2685168496839B110B102F05E
:202D000087FCE268506840688047E2685268906808B9D7688FB10A491C310F68002FFCD071
:202D200000230B6010B18047E0684268D06800B180470448503802F029FE98BDA00A0020CF
:202D40000010044051000706144BB0B5997B03EB81010A69017801F07F014D000170AC189A
:202D60005219527803EB82052F6907B19A732278141103EB84031F6C2FB90C290CDA182151
:202D8000FDF7C8F9B0BD02F00F0257F8221011B903F090FFB0BD8847B0BDC0463C16002020
:202DA00038B50546012001F0E7FC124C2046143000F0DEFB288900280CBFEB20002068706E
:202DC00094F83F00C10824BF00F0FB0084F83F0080080BD394F83F0000F0FD0084F83F00FD
:202DE000297C6878C1F3001103F006FD284603F089FF38BD942B00202DE9F04105461248EA
:202E00000E46002100782960012802D00120F3F7D7FE0E4C606880473768804630463FB1AD
:202E20006A687968914203DC38463F68002FF8D1056030682F60854201D1FDF747FDA168AA
:202E400040468847BDE8F081A21B0020B4150020134A38B5B2F8C4504FF6FF71A9421BD0AE
:202E60000024012000FA04F32B4212D05940B2F8C4300C4D1940A2F8C410291D0A6804F1C9
:202E80000C03984010430860022003F091FA204638BD641C0F2CE5DB6FF0010038BDC046BF
:202EA000A00A00200810044038B5044642F209000DF1020100F0F8FB9DF8020050B19DF867
:202EC000020002281AD1A08894F82710FEF77CFC054606E042F20D00694600F0E5FB9DF8FD
:202EE0000050284600F01CFB0020A4F87C5094F82130607013B1102003F014FF38BD38B5FC
:202F0000046845682068002808BF4FF0FF301FD004F076F92168002954BF491E0021216093
:202F200004F06AF9206890B904F12C0004F008F904F1480004F010F904F1640004F00CF9C7
:202F40006868FBF7E9FA04F1180003F06DF8002038BDFEE72DE9B841124C0546201D006810
:202F60008047804603F000F86F7E002F08BF6B6807D069682A69AF68091A5218B9180B4622
:202F80006960E968286105F11402184601F0D6FE012768686F76A168A86040468847BDE877
:202FA000B881C046B415002010B504F029F9104C217829B10F490C6804F01EF9204610BD35
:202FC00004F01AF903F046FD0B4A002303F0B0FC626A002314001B184FF07A024FF090508D
:202FE00044EB0104C11842EB04021046001C10BDA00A00200430044000093D00B0B5134C06
:203000006068628800B325880021AA42C8BF01210B46AA42C6BFA91A01F58061A91A8FB288
:203020008FB1012B03D0A1183A46083109E0A118C2F58062083103F083FF606804F1080130
:203040002A4603F07DFF6580B0BDC0469406002038B51248104C0168114D0C40E143016044
:20306000A10907D34068800904D328464FF4005103F08EFC14F4602F0DD02846EC3800F14E
:20308000C0010A6804F4602400F5907014430C60002103F07DFC38BD20000E0008100440BD
:2030A0008C0B0020134910B5044691F83F00ADF1180D40F0020081F83F00012002F0E4FF83
:2030C000607890B9211D02A803F08AFA03F088FB01460120009004F110030193E38902AA4E
:2030E0000520F4F76FFA607010B1002103F084FB06B010BD942B00201FB5014604208DF80D
:20310000000048788DF80100B1F896000DF10203ADF80C008C31184603F062FA02F0AEFC70
:2031200060B14FF6FF7453200DF10E01ADF80E40F3F74AFE044920460A3108806846FAF70C
:20314000A1FB00901FBDC0464A0F0020134A3D321278812A01DB842A0FDB00F1100249081F
:2031600092B224BF00F129018AB21228CCBF05200220801880B2C0000DE04201490802F5C3
:20318000C67292B224BF02F21E218AB21228CCBF28200C20801880B27047C0464A0F002028
:2031A0002DE9F0410120104E104D307028781F469046022801D003F07DFD0024022114EAC4
:2031C000070001EA080108BF002902D103F072FD07E0074991F90000401E08702C7003F0A9
:2031E0005FFB3470BDE8F081A21B0020A31B00209E1B0020C8B5071C01D103F05BFD796889
:203200004878C6111FD03B89F96400204A78C2F3C3020F2A09D00A781018801C80B25218B7
:20322000834202F10201F1DC01E0801C80B2834206DB79683E8941187960311A398100E0F2
:203240000020A7F85000C8BD10B5044600211C22ADF1200D6846FDF746FF60788DF800005D
:20326000A0788DF80100E0788DF8020020791122611D8DF8030001A8FCF704FCA07D8DF8C1
:20328000150008B1A06906900348006881696846884708B010BDC046741B0020F8B5044676
:2032A0000D46084611220021FDF71DFF94F800C0BCF1000F1AD0641C00214FF0010EE078D0
:2032C000A37843EA0023207809E0C610AF5D00F00702401C0EFA02F2C0B23A43AA5583421C
:2032E000F3DA491C241DC9B28C45E8DCF8BD80B502465378107840EA0320C7130F7007BF5A
:20330000C0F3062300F0FF00C0F3C323C0F30A004B70802848800DDA02280BDB012B0CD062
:20332000022B0AD0042B08D0052B06D0062B04D0072B02D00022104600E0921C4A6080BD83
:2033400070B5114C2068E8B1104D686880470646216894F82F00022806DBA96830468847E5
:20336000F120F6F7D7F870BD04F1240002F0BCFE002394F82F00A9682360401C84F82F0015
:203380003046884770BDC046700D0020B415002038B5044642F208000DF1020100F084F94E
:2033A0009DF8020040B19DF80200022817D1204601F096FA054606E042F20C00694600F0E5
:2033C00073F99DF8005094F8200030B9284600F0A7F8A4F87C50002000E00120207038BDFC
:2033E000F0B5124D00260C460746ADF1140DC5F8B061012003F000FE2868C00FF9D3286AA8
:203400000090686A0190A86A0290E86A03903FB13846694611F8012B401E04F8012BF9D18E
:20342000032005B0C5F838023046F0BD5045024010B50446012001F09FF92078212804BF66
:20344000EB2060700D4991F83F00C20824BF20F0040081F83F00800805D22B20207020465A
:20346000FFF772FC10BD91F83F0000F0FD0081F83F006078002103F0BFF910BD942B00205E
:2034800070B5114D95F8A100B5F8C6400F2810D00E483430066801F075FB2018864208D848
:2034A00095F8A1104FF4707088402418A41B04F57074044D284600F05BF82146284603F041
:2034C0003BF870BDA82B0020A00E00201C190020114898B501210170022111400F4A4FF031
:2034E000E0471F4008BF002903D092F90010491E1170044692F9000030B192F90000002897
:2035000006DC03F0D7FB03E000200146F3F758FB0020207098BDC046A21B00209E1B0020BC
:20352000B0B50546802D01DD03F0C4FB0D4C606880470D4B0D490A4A1F780A390D701FB985
:203540001778A1682FB907E01778A16837F07F0702D088470120B0BD8847FEF787F8B0BDE0
:20356000942D0020B41500204C150020D019002070B505460F480078012803D0012000217A
:20358000F3F71EFB0C4C201D006880470B49064628460B4602F063FE18B9191D284602F04B
:2035A0005EFE1869A84201D1FDF790F9A1683046884770BDA21B0020B4150020801B0020F9
:2035C00070B540680C46054600F5847002F0CCFD0D482A7F0168687F8018AA69C01D80B2D5
:2035E00044430A4805F584766043B0FBF2F008186330B0FBF1F1491C304603F0B9FD304694
:2036000003F0F2FD70BDC046B00C000040420F000F4838B50078C8B10E4D0F4C95F82E1092
:203620006420503C4843206604F15C00FFF792FCE08EE26B95F82E10401C80B28918E08679
:2036400000B900210020E16300F0CCF938BDC0465D0F00208C2A0020202A0020F8B5114CA6
:2036600060680D4680470E4BA16893F830705A6B97B10024203A2032967F4EB1D37F9D42B9
:2036800006D100239377FF23D37788472046F8BD7F1E04F10104EED18847FF20F8BDC046D1
:2036A000CC100020B4150020F8B50E4602F0F4FD05464FF6FF70A84208BF682013D00A4CD0
:2036C0006068804709490A4B0746680000EBC50008180278991842783046FCF7D3F9A1680C
:2036E000384688470020F8BDB4150020C40000008C2A0020042838B51CD1104CEC3C04F1A6
:20370000C800054603F0C3FCA0B1284603F034F909490968484364280CD2284602F024FDCC
:20372000052001F0B5FD2046012181720421EC3003F02EF9002038BDB00C00008C0B002063
:203740001149D0B524310F68ADF1180DCFB17E69BEB1B0B106218DF810100226ADF81260B9
:203760000024ADF814404388ADF8003042680192816802917C6904AE96E803000C226B46DC
:20378000A04706B0D0BDC046D411002038B5EB2002F033FF0D48002505700B480078862870
:2037A00002D1284600F064F8094C6068804709490C39CA6913681D711268CA61A168884748
:2037C00002F0F2FE38BDC046942D0020922D0020B4150020F02C002038B50D4C6068804752
:2037E00005460C48007870B90B48007830F07F0009D10A48007830B90948007830F07F002A
:2038000001D103F014FCA1682846884738BDC046B4150020912D0020902D0020922D00200F
:20382000942D0020F8B506460F4800680D4CC06B80476168401A21788900B0FBF1F0B042E1
:2038400001D303F037FA094D243D686880470746A6603046FDF74CFBFAF7B4F9A9683846F1
:203860008847F8BD241B002020170020D815002038B50F49104C088D401C08856068804753
:2038800005460C480178862903D0A1682846884738BD8721017003F00FFBA16828468847F7
:2038A000082002F04FFAE920FDF798F838BDC046241A0020942D0020B4150020F8B50646FC
:2038C0000F4D104F7388002417E0A00000EBC400321851689068D26852B9AF420BD00A783A
:2038E00055F822200346491C08461946904701E0FCF7C8F87388641CA4B2A342E5DCF8BD47
:203900004480010050800100F8B5034600208C460446074613E01CF8015B082685F001018A
:2039200001F001014018C0B2411E994206D0641C761E4FEA6505E4B2F0D100E00127A242C0
:2039400003DC27B903F083FB01E0002FE3D02046F8BD3EB5054615F8060C03281DD12B6850
:203960001869009058690190986902906C6859689A681868DB68A0472968086015F8080CF6
:2039800001F02EFD0446012002F000FA011C04D0422008702046FEF789FF3EBD2DE9F041C4
:2039A00017468846064603F0D7F80D4C0546002128222046FDF797FB31462A462046FCF793
:2039C00061F840463A46291900F0C0F8204602F021FE02A002F01EFEBDE8F0810D0A00C08A
:2039E000BC2C002070B50F4C05462179E079814217DD6179A94214DDA3680B4E23B12946ED
:203A000032469847E0796179A07101FB0050216800EB800009180878E071D1F80110304689
:203A2000884770BDAC170020042A0020F8B502F0F8FB0D4607463B2F08BFF42012D00B4CA9
:203A4000606880470646BA0007480949835C801842784E39C918284602F046FFA168304673
:203A600088470020F8BDC0469C020000B4150020820F002038B50D460E49144660390A6868
:203A8000AA4205D901EB8501D1F89410884201D0022038BD03F0B4FB074B103B1A68AC401E
:203AA0000121A9408A4314431C6003F0A5FB002038BDC04694260020E0200240104880B504
:203AC0000C3000688769B7B10C49B94213D0816800E039464F681FB100F12802BA42F8D108
:203AE000497B11F00F0F06D1408D40F60901814208BF012000D0002080BDC046C7820000D8
:203B0000A00A002070B50E4614460546082300212422ADF1280D684603F032FB00200690D4
:203B20000590ADF81000084800684FF47A716B46B1FBF0F080B2314604FB00F2284603F01D
:203B40001BFB28460AB070BDB00C0000FEB50746052400266B4697FBF2F05043381AC0B273
:203B60000A28ACBF372530254019187097FBF2F5AFB22FB1641E03F1010306F10106EAD129
:203B8000761C13F80109761E01F8010BF9D100200870FEBD10B50F4C94F83F00ADF1180D1A
:203BA000B0B940F0010084F83F00012002F06CFA02A801F077FF343401200090064B019427
:203BC00003F1BA000388032102AA0520F3F7FAFC06B010BD942B0020A00E002070B5104C26
:203BE0000546606880470B49064691F83D0000F0F00040F0010081F83D000848006883691A
:203C0000054800682A464FF0FF319847A1683046884770BDD8120020D0190020201700204C
:203C2000B41500200E4808B50178081C05D0401E12D0801E01280FD908BD02F03DFF38B14B
:203C40000948084900680968884238BF002004D31C20FCF7C3FE08BD0846F0F707F808BD83
:203C6000261A002010130020281B00201FB5144600900A79487940EA02208A7942EA00229F
:203C8000C87940EA022001900A78487840EA02208A7842EA0022C87840EA0220029068465C
:203CA00000F0E4F9B0FBF4F16143401AC0B200901FBDF8B5051C0E4606AF04D0012D0CBF27
:203CC0000624002400E002240EB9A41CA4B2012A06D0022A0ED15889C01D04EBE00008E032
:203CE0003878002814BF022101210020FBF762F9001984B22046F8BD0F4800B50068ADF1EB
:203D0000240D69466C30F4F729FF10B99DF80B0008B900200DE0684601F027FF9DF808106B
:203D20004FF47A73B0FBF1F24A43801A091A03FB01F009B000BDC046700D002038B504463C
:203D4000642C13DA0D4D6868804703466946722001F0F4FD0099E00000EB04104018A968A8
:203D60000090184688470098001D38BD0248643CE1B200EBC10038BD08110020B41500209C
:203D80002DE9F04103F0B6F80D4D603D2B688046A3B105F194060024012707FA04F018EAC4
:203DA000000F07D056F8240020B1026812B1214690472B68641CE4B29C42EED3BDE8F08111
:203DC0009426002010B5044603F01AFA0C4A117819B903F011FA012010BD11460B7884F008
:203DE000FF0213400B70097811B103F005FA05E003F002FA0348082102F0CAFD832010BD4E
:203E00008A2D00208C0B002038B50D46044603F022F96368A1688B4204D103F0EDF94FF0EE
:203E2000FF3038BDE168491CB1FBF3F25A432368891ACD54E1606269A168491C8A42A160EC
:203E400038BF616103F0D8F9A06838BD0C4885460C4885446F4607208743BD460A486F46FC
:203E600007600A48002803D07946491D8E460047FBF77AFC02F050FD03F042F9FEE7C0468E
:203E8000004B002000050000381C0020016F01000F48B0B507680025ADF1180DADF81050B5
:203EA00097B106208DF808000223ADF80A30ADF80C5004AC00943C6902AA92E803002A4680
:203EC000A04708B1ADF81050BDF8100006B0B0BDF811002010B50446012000F04DFC20782B
:203EE000212804BFEB2060700A4991F83F00C20824BF20F0040081F83F00800809D391F85A
:203F00003F0000F0FD0081F83F006078002102F073FC10BD942B002008B564206946FFF7D1
:203F200085FD09490948C1F8D8000B483830C1F8DC009DF8000000280CBF05480548C1F8A0
:203F40008000C1F8C00008BDD8120020002D00204E9055550E7A55550017002030B50E4D1B
:203F600095F8A100ADF1AC0D0F280CD10B4C3F3C04F11400FFF7FCFAB5F8C61004F1140055
:203F800002F0DAFA05E02F208DF800006846FEF7DBFE2BB030BDC046A00E0020D32B00206C
:203FA00038B50F4C0546083C204602F037FFA8B9204603F052F80446A068054209D0E368DB
:203FC0002269284600219847002818BF4FF0FF3005D1204603F043F8041CEDD1002038BD1E
:203FE000C00F00200CB4F0B505AF061C0C4627F00303ADF1040D03F1040304D030680028EA
:2040000018BF051C00D100253A68284602F0BAFE844238BF601E15B131684118316001B0C3
:20402000BDE8F04002B0704708B50B4602F0B4FB5989418199898181997B8173D97BC1733B
:20404000197C002201B10122597C417459694161197E0274002201B10122027603F119015C
:204060000B221930FBF70EFD08BDFEE7416882680D4B0068C91AD21AC01A4A40A2EBB1421D
:204080005040A0EB72504140A1EBF0114A40A2EB31425040A0EB32704140A1EBB04181EA85
:2040A0000200A0EB31207047054152210B4A08B502F10C000068C00A01D200F04BFC1068ED
:2040C0004008FCD30648006841680220884705490A6882420CBF0448086008BD08800240E7
:2040E000CC010010802D0020EFBEADDE10B50821ADF1180DADF800100A4C04901B21ADF8AD
:204100000210606A0290012101910549064803910168684688470299616206B010BDC04680
:204120009D57010094190020D815002010B5ADF1180D0C4C01900A4808210390002004907D
:204140002069ADF800101B2102900748ADF802100168684688470299216106B010BDC046C1
:2041600071570100241B0020D81500200D4808B50068020F0C48036803F0FF03802B28BF39
:20418000002302F0B3F801464FF0FF30012907D1111C04D0891E04BF143358B208BD0A20FD
:2041A00008BDC04618130050A01000501CB50E4C0020042260706946207000F0D9FF0098D9
:2041C000B0F5801F0CD020B901F07AFAF6F74AFE08E000F06BF802F0DDFC0420608001E061
:2041E00001F06EFA60781CBD281C00200D4938B5CA68824210D1087801280DD103F000F8C5
:204200000546094801F0C2FB0446284602F0F4FF04F0FF00012802D06FF07F0038BD4FFAAD
:20422000A4F038BDA00A002001000304B0B502F012FF05460A48017801290DD00121094F24
:204240000170387840B1084C074620688168204688470C347F1EF8D1284602F0CDFFB0BDC6
:204260004A1C0020C80C0000A40B00000B4B80B51F7800227FB10A4B1B7883420BDD8A4260
:2042800008BF0849084F820002EBC002B8180268D26890470246104680BDC0464A1C0020CC
:2042A000C80C0000200B0000A40B0000F8B50D4C201D00688047054600F0F6FD0646002044
:2042C00001F0F2FD02F02EF80746304602F0C4F81FB10548012141700170A16828468847CE
:2042E000F8BDC046B4150020281C002030B50E4D2868ADF1240DA0B10024FFF7D7FE04EBE8
:204300000D020021CB00491C20FA03F3042902F8013BF7DB241DE4B2202CEEDB29686846CD
:20432000884709B030BDC046301C002010B50446012000F021FAEB200B49607091F83F0064
:20434000C20824BF20F0040081F83F00800809D391F83F0000F0FD0081F83F00607800211A
:2043600002F04AFA10BDC046942B0020F8B5071C01D102F09FFC0C4C201D006880473E68BC
:2043800005465EB107498A68A6F10C00964204BF00228A600021396001F096FDA168284682
:2043A0008847F8BD3C160020B415002038B50E4B05460C46281D03F1480102F0C6FD188F5D
:2043C0002880B3F8460003F13E016880201D02F0BCFD93F83A00207300206073188F2080AF
:2043E000988F608038BDC046701400201CB50A1C17D000230124E407A04238BF041C944237
:2044000001D95200FBE790425B41904228BF801A914201D25208F6E7191C021C081C111C4C
:204420001CBD00B1C843FBF7DEFA1CBDB0B50D46044602F010FEA76897B121692268515C2A
:20444000297063682169A768491CB1FBF3F25A43891A2161791EA16002F0CEFEA068B0BDDC
:2044600002F0CAFE4FF0FF30B0BD704738B50D4D04462868ACB178B9281D05F11001FBF703
:2044800035FC1D212F22286001F0D8F828681E21302201F0D3F8286804F001021C2100F082
:2044A000C9FA38BDE41A00200D4910B509780446A1B1617871B9217839B194F8201021B9D2
:2044C000FEF766FF0020207010BD94F87C00FFF727F810BDFEF7E8FC0020607010BDC0467F
:2044E0005D0F0020F8B50C4E0446706880470B4DC7B205F15C0002F04DFC410001EBC001F4
:204500004FF47A70B1FBF0F0E96B20604018B168206038468847F8BDB4150020D029002019
:2045200070B50446606810F07F4F18BF6FF0020011D10BF02AFA084D0646287828B1686853
:2045400000F0F6FF606801F00AF86068686030460BF045FA002070BDB81B002000B5ADF1E8
:20456000140D8DF808000A4A039112788DF804200823ADF800300748ADF8023024301822BE
:204580000168ADF806206846884705B000BDC0466C1B0020B415002010B5ADF1180D019049
:2045A00009480A4C0390606A0491082202900848ADF8002013220168ADF8022068468847AF
:2045C0000298606206B010BD9D57010094190020D815002000B50221ADF11C0D8DF81410E5
:2045E0000A488DF81810828FADF80C20008F0649ADF816006A4600208DF8190018200AF0A1
:20460000EFFD07B000BDC046376F0100701400200D4938B5D1F8EC3209681B3800FB00F40C
:2046200009060A1643F3072100FB01F519066043091661434243891201EBE50101EBA240B7
:2046400000EB234038BDC046A41000500C49086820F0020040F4007008600A48032140F87C
:20466000041C41F230018160012101605022826001604FF4CA628260016040F80C1C7047D4
:20468000000004600C41044098B50D4C2778002F18BF012013D16188C1F5805189B2884260
:2046A00000DC58B902F046FB00206070F6F7DAFB20B9607800280CBF0127071C384698BD66
:2046C000281C002070B502F09BFD06460B48E030007848B107480068C568074800243421FB
:2046E00001222346A84700B10124304602F084FD204670BDA401001000A00C40B80F002065
:20470000B0B502F07DFD0546FDF75AFD0A48094C0021E0300170A168022088470746102072
:20472000FFF73EFC17B1A16803208847284602F063FDB0BD240C0000B80F002038B50C4CFD
:2047400001462C3CCB8AE2682068DB080ED204F1240001F0C9FC074D6868804794F82F103B
:20476000491C84F82F10A968884738BD904738BD9C0D0020B415002038B50B4C054660686F
:2047800080470A4B1A7885F0FF010A40A1681A708847FFF721F806480078012803D0002059
:2047A0000146F2F70DFA38BDB4150020912D0020A21B002002460C4808B5007800F0F8FD73
:2047C0004168006802FB0103084A4FF47A70B3FBF0F189B2D18400FB113040037D21B0FB61
:2047E000F1F0108508BDC046870F0020D81200200C4800B50268ADF1140D53681189106AB7
:2048000000910190C01A091A88B2029006480390916A506A92F888201530F8F7C5F805B03F
:2048200000BDC046700D0020780F0020F8B50D4C0646201D006817460D4680473168A9427F
:2048400019BF55F80C1C47F80C1C55F80C1C3160FF2705F8027C002145F80C1CA16888479F
:20486000F8BDC046B415002038B5044602F0C8FC05460B48007868B1204601F087F8044658
:20488000284602F0B9FC04F0FF04012C0CBF8120022038BD284602F0AFFC012038BDC04635
:2048A000A00A002000B500211822ADF11C0D6846FCF719FC0849088F6A46ADF80A00022038
:2048C0008DF80800888F0549ADF8000018200AF087FC07B000BDC046701400207B6F010083
:2048E00010B50446E220ADF1200D05A9FFF79EF8608894F8262005A9FFF7B8F9044669469A
:2049000042F20200FEF7D0FE01F01CF9024669462046FEF7F9FF08B010BD08B502460B4673
:204920000846002102F039FB012102F8010B184602F033FB022102F8010B184602F02DFB9B
:20494000032102F8010B184602F027FB02F8010B104608BD0949086820F480600860000478
:20496000000C40F480300860054848600549012008600549002008607047C04614800240AA
:2049800004010100A8025042802D002030B5054608200C46ADF1140DADF800000020ADF835
:2049A0000200182102900648ADF804100168684688479DF80C0028700498206005B030BD46
:2049C000D81500201FB58DF800000A48006868B144695CB1084902A80A688988026002AB57
:2049E000818093E8030001226B46A04702F050F800901FBDF81100209C0C000003B490B50A
:204A000003AF3968ADF10C0D68460160B98881809DE803001C46FBF715FF28B1B9682246E9
:204A200000F0A6FB002000E0012003B0BDE8904002B0704780B517460A4A603A13688B426B
